:100000000C94340E0C945C0E0C945C0E0C945C0EF0
:100010000C945C0E0C945C0E0C945C0E0C945C0EB8
:100020000C945C0E0C945C0E0C945C0E0C9440676B
:100030000C94D66A0C946D670C945C0E0C94D617D5
:100040000C94C4170C945C0E0C94F16D0C945C0E23
:100050000C945C0E0C945C0E0C945C0E0C945C0E78
:100060000C94966A0C9432180C94D8670C94A5687A
:100070000C945C0E0C945C0E0C945C0E0C945C0E58
:100080000C945C0E0C945C0E0C945C0E966C9A6C4A
:10009000A26CAC6CC36CDD6CF26C016D166D2D6DD9
:1000A000376D556D5B6D606D666D6C6DC66DD06D39
:1000B000756D7B6D816D8A6D8E6D936D9B6DAD6D74
:1000C000B36DB96DBE6D9E6C9E6DA36DA86D5370C2
:1000D0006C617368008040000000000000000000B8
:1000E0000000000000000000000000000000000010
:1000F0000000000000000000000000000000000000
:1001000000000000000000000000000000000000EF
:1001100000000000000000000000000000000000DF
:10012000000080C0E0E0F0F8F8FCFCFCF8F8F8F023
:1001300040000000000080808000000000000000FF
:1001400000000000000000000000000080C0C0E0CF
:10015000E0E0F0F0F0E0C00000000000C0F8FFFFB9
:100160009F8783838383838383838383838383833F
:1001700083838383838383830383808383838383D2
:10018000838383838383838383838383838383833F
:100190008383C3E3733F1F0000000080E0F0F8FC9E
:1001A000FEFFFFFFFF7F3F1F1F0F0783C3E1E1E05B
:1001B000E0C0000E1F3F7F7FFFF3E0E08000000003
:1001C0000000000000000080F0FCFEFFFFFFFF7F4A
:1001D0003F0F0301010100000080F0FEFFFFC7C1D7
:1001E000C1C1C1C1C1C1C1C1C1C1C1C1C1C1C1C1FF
:1001F000C1C1C1C1C101C1F0FEFF3F0F070F0D0D0D
:100200000D1D191919193131313171616161E1C166
:10021000C1C18100000080E0F8FCFFFFFFFF2F1745
:100220000F038180C0E0F0F8FCFEFFFFFFFFFFFF3F
:100230007F010000000000000001010307070E1EFF
:100240001C3870E0F0F8FEFFFF7F1F0F0300010075
:10025000000000000000000000000000000000009E
:10026000000000000000000000000000000000008E
:10027000000000000000000000000000000000007E
:10028000000000000000000000000000000000006E
:1002900000000000007EFFFFFFFFFFFFFBF8FCFCFB
:1002A000FEFF7F3F1F0F07C3FFFFFFFFFFFF7F071B
:1002B0000000000000000000000000000000C0E09E
:1002C000F8FEFFFF7F1F0F1F3D7CF8F8F0E0800075
:1002D000000000000000000000000000000000001E
:1002E000000000000000000000000000000000000E
:1002F00000000000000000000000000000000000FE
:1003000000000000000000000000000000000000ED
:1003100000000000000000010101010103070707C0
:100320000301000000E0FCFFFFFFFFFF1F030000D0
:10033000000000000000000000C0F078DE27130974
:100340000E0703000000000000000001030F7FFF04
:10035000FC7878F800000000000000000000008039
:10036000808080808080808000808000808000008D
:1003700000000000008080808080808080808080FD
:1003800080808080808080000000000000000000ED
:10039000000000000000000000000000000000005D
:1003A000000080F0FEFFFFFFFF3F0F010000000094
:1003B00000000000C0E0381E0F0300010000000034
:1003C000000000000000000000000000000000002D
:1003D0000000030301000000000000000000000E08
:1003E0000E02020202020303000F0F000F0F0808A3
:1003F00008080808080F0F08080808080F0F000071
:1004000000000F0F000000000000000000000000CE
:1004100000000000000000000000000000000000DC
:10042000C0F8BFFFFFFF1F7F0100000000000000B9
:1004300000F0FCFF7F7830000000000000000000AA
:1004400000000000000000000000000000000000AC
:10045000000000000000000000000000000000009C
:10046000000000000000000000000000000000008C
:10047000000000000000000000000000000000007C
:10048000000000000000000000000000000000006C
:100490000000000000000000000000000000301C10
:1004A000070E0F0701000000000000000000000020
:1004B000000000000000000000000000000000003C
:1004C000000000000000000000000000000000002C
:1004D00000000000000000001B1E272D36394B4E87
:1004E000636C7278878D939CB1B4C6C9D2D8E1E4AD
:1004F00001020304010302040402030104030201D4
:1005000003010200040506076D656E75537461638F
:100510006B206F766572666C6F77006D656E7553D4
:100520007461636B20756E646572666C6F770070C2
:100530007265737320616E79204B657900414C457B
:100540005254004D455353414745004C4F41444997
:100550004E47002020202020202020202020202066
:1005600020202020202020202000506C6561736511
:1005700020526573657420537769746368657300EE
:100580005377697463686573205761726E696E672B
:1005900000204F6C642056657273696F6E2045456C
:1005A00050524F4D202020434845434B2053455443
:1005B00054494E47532F43414C494200416C6172AC
:1005C0006D732044697361626C6564005265736584
:1005D00074207468726F74746C65005468726F7400
:1005E000746C65206E6F742069646C650050726570
:1005F000737320616E79206B657920746F20736B43
:10060000697000414C45525400454550524F4D20B1
:100610006C6F77206D656D004F46464142535255D1
:1006200073525525454C73454C2554487354482501
:10063000414C73414C2550312050312550322050CF
:1006400032255033205033250054485252554445EA
:100650004C4549443049443149443241494C47456D
:100660004154524E535731535732535733535734E3
:1006700053573553573653573753573853573953C2
:100680005741535742535743004F4646004F4E2061
:10069000002D2D2D004348002D2D2D2000525544B6
:1006A00020454C45205448522041494C20005031AF
:1006B000202050322020503320204D4158204655D4
:1006C0004C4C4359433143594332435943335050BF
:1006D0004D3150504D3250504D3350504D3450509C
:1006E0004D3550504D3650504D3750504D38434891
:1006F0003120434832204348332043483420434884
:100700003520434836204348372043483820434863
:10071000392043483130434831314348313243482E
:100720003133434831344348313543483136002D65
:100730002D2D2D00564552533A2056312E35343941
:10074000352D6572657A00444154453A2031312E89
:1007500030322E323031320054494D453A2031305A
:100760003A31303A3139002053564E3A20657239C9
:10077000782D7237303800204D4F443A204A455486
:10078000492020200012081200081C0808081C0834
:100790000000082200490022080000000000227F1B
:1007A0002200000008220049002208000008220060
:1007B00049002208000000227F22000000000008FB
:1007C0002200490022080000081C0808081C080034
:1007D00064319F438342E82BD024CD54AF51D3489A
:1007E0006D4AD650124BD01D8B1FC11F6120DC21DA
:1007F00054546D00457870457846466E654D656485
:1008000043727300544F540053544B1153542500FA
:10081000544D45115453570053544154004A4554C4
:1008200049005B4D454E555D20746F2072656672C0
:1008300065736800537461636B0F6200746D616966
:100840006E0F6D7300746D7231204A697474657235
:100850000F757300746D72314C6174206D696E0F89
:10086000757300746D72314C6174206D61780F7511
:1008700073005354415432004D6F64650042616E01
:100880006447617000506F745363726F6C6C004109
:100890006C61726D205761726E696E67004D656D97
:1008A0006F7279205761726E696E670054524530DD
:1008B000313241470054524530313241470044659E
:1008C0006661756C74205377005377697463682090
:1008D0005761726E696E67005468726F74746C65EC
:1008E000205761726E696E670053706C6173682087
:1008F0004E616D650053706C61736820736372653F
:10090000656E004F4646004C69676874206F6E2024
:1009100053746B204D76004C69676874206F66666F
:10092000206166746572004C69676874207377692A
:1009300074636800466C617368206F6E2062656541
:1009400070004265657020636F756E74646F776EBA
:10095000004D696E7574652062656570005468723B
:100960006F74746C652072657665727365005349A7
:100970004E474F534D5046494C540046696C746580
:10098000722041444300496E6163746976697479E9
:1009900020616C61726D00426174746572792077B8
:1009A00061726E696E6700436F6E7472617374007A
:1009B00048617074696320537472656E677468006F
:1009C000537065616B65722050697463680042659D
:1009D00065706572506953706B7200536F756E6409
:1009E000204D6F6465005175696574204E6F4B65CD
:1009F00079207853686F727453686F7274204E6FE9
:100A0000726D20204C6F6E672020784C6F6E6720CF
:100A100000426565706572004F776E6572204E61A9
:100A20006D6500524144494F205345545550004391
:100A3000616C004D756C7469706C696572006368F7
:100A400031636832636833636834006F6666202BF5
:100A50003D203A3D006D6F64650A25207372632066
:100A600020737700536C61766500545241494E45BE
:100A7000520000030303030056455253494F4E00F2
:100A80005472696D2D202B00204D656E75204578C0
:100A9000697420446F776E20202055705269676812
:100AA00074204C6566740044494147004247004148
:100AB0004E41005B4D454E555D205748454E204404
:100AC0004F4E45004D4F564520535449434B532FED
:100AD000504F545300534554204D4944504F494EB4
:100AE00054005B4D454E555D20544F2053544152A8
:100AF000540053544152542043414C4942524154B2
:100B0000494F4E0043414C4942524154494F4E00D7
:100B100066726565004D4F44454C53454C00434F4C
:100B20004C20446972656374696F6E0041494C20C2
:100B3000446972656374696F6E00454C4520446971
:100B400072656374696F6E005377617368205269D0
:100B50006E6700436F6C6C656374697665002D2D5C
:100B60002D202020313230202020313230582020DA
:100B7000313430202020393020202020005377616C
:100B8000736820547970650048454C49205345549A
:100B90005550000044454C455445204D4F44454C6C
:100BA0000F5B4D454E555D00543254685472696771
:100BB00000547261696E657200452E204C696D6942
:100BC000747300504F534E45470053686966742054
:100BD00053656C004C50342F4C5035202044534DFD
:100BE000326F6E6C792044534D322F44534D580070
:100BF00044534D20547970650053656E64205278DB
:100C0000204E756D626572205B4D454E555D0050FE
:100C1000504D2046724C656E0D6D53656300205239
:100C2000784E756D00344348203643482038434899
:100C30002031304348313243483134434831364320
:100C40004800755300755365630050504D202020B7
:100C500050585820202044534D32202050504D31C0
:100C600036200050726F746F005245544131323358
:100C7000004265657020436E74005472696D2053A4
:100C80007700457870202020457846696E65466972
:100C90006E6520204D656469756D436F6172736583
:100CA000005472696D20496E6300542D4578706F51
:100CB00000542D5472696D00436F756E7420446F3B
:100CC000776E436F756E7420557020200054696DE7
:100CD00065722000547269676765720054696D65BA
:100CE00072004E616D650053455455500000090176
:100CF0000000000000000602004475706C6963612A
:100D000074696E67206D6F64656C005B4D454E5570
:100D10005D20205B455849545D005945530B4E4FAB
:100D20000044454C455445204D4F44454C004455E6
:100D3000504C4943415445204D4F44454C002041BF
:100D400042434445464748494A4B4C4D4E4F50510B
:100D500052535455565758595A61626364656667D1
:100D600068696A6B6C6D6E6F70717273747576778B
:100D700078797A303132333435363738395F2D2E41
:100D8000006578702020252020737731207377321A
:100D9000004558504F2F44520000034452204869E8
:100DA0006768004452204C6F77004452204D6964BC
:100DB00000447253773200447253773100576569AB
:100DC000676874004578706F004558504F2F445243
:100DD00000002B2A52004D4958455200507265734D
:100DE00073205B455849545D20746F2061626F72B7
:100DF00074004D6178206D69786572732072656149
:100E000063683A200044454C455445204D495820DC
:100E10005B4D454E555D00536C6F7720205570003B
:100E2000536C6F772020446F776E0044656C617956
:100E30002055700044656C617920446F776E0041E5
:100E4000646420202020204D756C7469706C795288
:100E500065706C61636520004D756C747078004F2F
:100E60004646005761726E696E6700537769746316
:100E70006800437572766573004F4E204F464600FA
:100E80005472696D004F46464F4E2000466C4D6FC0
:100E900064657472696D004F666673657400466DB3
:100EA0005472696D56616C005765696768740053C8
:100EB0006F757263650045444954204D49582000C0
:100EC000494E53455254204D495820002D2D2D2D6B
:100ED000202020763E6F66732020763C6F6673205C
:100EE000207C767C3E6F66737C767C3C6F667341BB
:100EF0004E44202020204F522020202020584F52A6
:100F00002020202076313D3D7632207631213D76FD
:100F1000322076313E7632202076313C76322020E7
:100F200076313E3D76322076313C3D76322000539C
:100F30005700435553544F4D205357495443484548
:100F400053000002534146455459205357495443D6
:100F5000484553000002434C454152204D495845F5
:100F600053205B4D454E555D002052455441004392
:100F700068616E6E656C204F726465720054454DF9
:100F8000504C4154455300434F5059205452494D01
:100F9000205B4D454E555D002D2D2D494E56004C84
:100FA000494D4954530000030303030303030303A0
:100FB00003030303030303004356004355525645FE
:100FC000530050524553455400454449542D3E006A
:100FD00043555256450009002D2D2D494E56004FC0
:100FE00046464F4E20002D2D2D783E30783C307CEB
:100FF000787C663E30663C307C667C6331206332B0
:101000002063332063342063352063362063372028
:1010100063382063392063313063313163313263A7
:1010200031336331346331356331360045455052D5
:101030004F4D206F766572666C6F77004545505254
:101040004F4D206F766572666C6F770067656E77BF
:1010500072697465206572726F7200454550524F17
:101060004D20466F726D617474696E6700426164F1
:1010700020454570726F6D2044617461004D4F448E
:10108000454C2020202020004D45202020202020DD
:1010900020200050085000000000000000006F00F9
:1010A0000007000700147F147F14242A7F2A1223CC
:1010B0001308646236495522500005030000001CE5
:1010C0002241000041221C0014083E081408083E7A
:1010D0000808005030000008080808080060600098
:1010E000002010080402003E49453E0000427F40B7
:1010F00000625149460041494936001814127F00E8
:1011000027454539003E494932000179050300363B
:10111000494936000649291E0000363600000056AF
:101120003600000814224114141414144122140827
:1011300000020151090600060909067E0909097E17
:101140007F494949363E414141227F4141221C7F2E
:10115000494949417F090909013E4149497A7F08C6
:1011600008087F00417F41002040413F017F081473
:1011700022417F404040407F020C027F7F040810E4
:101180007F3E4141413E7F090909063E4151215EB2
:101190007F09192946264949493201017F01013F4A
:1011A0004040403F1F2040201F3F4030403F6314DD
:1011B00008146307087008076151494543007F41DF
:1011C000410002040810200041417F000402010296
:1011D0000440404040400001020400205454547830
:1011E0007F484444383844444420384444487F3895
:1011F00054545418087E0901020C5252523E7F0882
:1012000004047800447D40002040443D007F1028C5
:10121000440000417F40007C041804787C080404EA
:101220007838444444387C14141408081414187C86
:101230007C080404084854545420043F4440203C93
:101240004040207C1C2040201C3C4020403C442846
:101250001028440C5050503C4464544C4400083610
:10126000410000007F000000413608000808221CF1
:1012700008081C220808A060800000000000000090
:1012800000000000000000FFFF0000000000001F41
:101290003F00003F1F00003030FFFF3030FFFF30C5
:1012A000303078CCCCFFFFCCCC8C0C060F0F86C036
:1012B000E070381C0C3CFEC7E3F33B1E0C00000042
:1012C00000333B1F0F000000000000F0F81C0E0769
:1012D000030000000003070E1CF8F000003030E0AF
:1012E000C0FCFCC0E03030C0C0C0C0FCFCC0C0C00E
:1012F000C000000000000000000000C0C0C0C0C06E
:10130000C0C0C0C0C000000000000000000000001D
:10131000000080C0E070381C0C00000000000000DD
:10132000000000000000003838000000000000004D
:101330000000000000000003033F3F03033F3F03A2
:10134000030C0C0C0C3F3F0C0C07030C0E070301A5
:1013500000183C3C180F1F383133331E1E33330046
:10136000000000000000000000000003070E1C3811
:10137000300000000030381C0E070300000303019A
:10138000000F0F00010303000000000F0F0000001A
:10139000000000333B1F0F000000000000000000B1
:1013A00000000000000000183C3C18000000000C89
:1013B0000E07030100000000000000FCFE87C3E3ED
:1013C00077FEFC00000C0EFFFF0000000000000C88
:1013D0000E0783C3E77E3C00000303C3C3C3E7FEDD
:1013E0003C0000C0E070381C0EFFFF00003F3F33A0
:1013F000333373E3C30000FCFEC7C3C3C78E0C00C6
:10140000000303C3E3733B1F0F00003CFEE7C3C3AD
:10141000E7FE3C00003C7EE7C3C3E7FEFC0000188B
:101420003C3C18000000000000183C3C1800000084
:10143000000000C0E0F0381C0E07033030303030C0
:10144000303030303003070E1C38F0E0C000000CA4
:101450000E07030383C3E77E3C00000F1F3B3130C0
:10146000381F0F000030303F3F3030000000003C9C
:101470003E37333130303000003030303030391FBB
:101480000F00000303030303033F3F00000C1C385D
:101490003030381F0F00000F1F383030391F0F0059
:1014A0000000003F3F0000000000000F1F393030F7
:1014B000391F0F0000000030381C0E070300000623
:1014C0000F0F06000000000000333B1F0F0000005C
:1014D000000000000103070E1C3830030303030360
:1014E000030303030330381C0E0703010000000050
:1014F00000000033330100000000003C7EE7C3C35E
:10150000E77E3CF0F8DCCEC7C7CEDCF8F0FFFFC3C7
:10151000C3C3C3C3E7FE3CFCFE0703030303070E7C
:101520000CFFFF030303070E1CF8F0FFFFC3C3C348
:10153000C3C3C30303FFFFC3C3C3C3C3C30303FCCA
:10154000FE0703C3C3C3C7CECCFFFFC0C0C0C0C02B
:10155000C0FFFF00000303FFFF03030000000000C3
:10156000000303FFFF0303FFFFC0E0F0381C0E077A
:1015700003FFFF0000000000000000FFFF0E1CF84A
:10158000F81C0EFFFFFFFF3870E0C08000FFFFFC7B
:10159000FE070303030307FEFC0000000000000039
:1015A0000000003F3F0000000000003F3F3F3F3091
:1015B00030303030391F0F0F1F3830303030381C8A
:1015C0000C3F3F303030381C0E07033F3F30303087
:1015D00030303030303F3F00000000000000000F8E
:1015E0001F3830303030303F3F3F3F0000000000B8
:1015F000003F3F000030303F3F303000000C1C38CF
:101600003030381F0F00003F3F000103070E1C3829
:10161000303F3F30303030303030303F3F0000001E
:101620000000003F3F3F3F0000000103033F3F0F2A
:101630001F3830303030381F0FFFFFC3C3C3C3C360
:10164000E77E3CFCFE070303030307FEFCFFFFC32A
:10165000C3C3C3C3E77E3C3C7EE7C3C3C3C3C78EDB
:101660000C03030303FFFF03030303FFFF0000005A
:10167000000000FFFFFFFF000000000000FFFFFF71
:10168000FF000000000000FFFF0F1F38F0E0E0F057
:10169000381F0F3F7FE0C08080C0E07F3F0303031F
:1016A00083C3E3733B1F0F0000FFFF03030303002B
:1016B000000C1C3870E0C080000000000003030331
:1016C00003FFFF000030381C0E07070E1C383000E7
:1016D0000000000000000000003F3F00000000008C
:1016E0000000000F1F383033371E1C3F333F3F00D0
:1016F0000003070E1C38300C1C3830303030391FD6
:101700000F000000003F3F000000000F1F38303086
:101710003030381F0F03070E1C38381C0E07030F1C
:101720001F38381F1F38381F0F3C3E0703010103C5
:10173000073E3C000000013F3F010000003C3E37F7
:101740003331303030303000003F3F303030300007
:101750000000000000000103070E0C0000303030D4
:10176000303F3F000000000000000000000000309B
:10177000303030303030303030000003070E1C384D
:101780003000000000303030303070E0C0FFFFC06B
:10179000E070303070E0C0C0E07030303030300089
:1017A00000C0E070303070E0C0FFFFC0E07030304B
:1017B000303070E0C0C0C0FCFEC7C303070E0CF0A1
:1017C000F89C0C0C0C0C0CFCFCFFFFC0E0703030E3
:1017D00070E0C000003030F3F300000000000000B3
:1017E000003030F3F30000FFFF0080C0E0703000F5
:1017F0000000000303FFFF00000000F0F03070E085
:10180000E07070E0C0F0F0C0E070303070E0C0C058
:10181000E0703030303070E0C000000000000000A8
:101820000000000C1E3F33333333333F3F3F3F3024
:1018300030303030381F0F0F1F3830303030381C08
:101840000C0F1F3830303030303F3F0F1F3B3333E9
:10185000333333030300003F3F000000000000006B
:101860000133333333333B1F0F3F3F000000000091
:10187000003F3F000030303F3F303000000C1C384C
:101880003030381F0F00003F3F03070F1C38300077
:1018900000000030303F3F303000003F3F00000389
:1018A0000300003F3F3F3F0000000000003F3F0FAC
:1018B0001F3830303030381F0FF0F03030303030DB
:1018C000F0E0C0C0E0F0303030E0C0F0F0F0F0C048
:1018D000E070303070E0C0C0E0F0303030303000C8
:1018E000003030FFFF303000000000F0F00000005A
:1018F000000000F0F0F0F0000000000000F0F0F058
:10190000F0000000000000F0F03070E0C08080C007
:10191000E07030F0F0800000000000F0F030303077
:101920003030B0F0F070300000C0E03C3E07030003
:101930000000000000FFFF00000000000003073E61
:101940003CE0C00000C0C0C0C00C1CF8F0E0C0C04B
:10195000E0F0F81C0CC0C0C0C03F3F03030303030A
:1019600003010000010303030303033F3F3F3F0064
:1019700000000000000000303133333333333F1EAA
:101980000C00000F1F383030381C0C0F1F3830305F
:10199000381C0C3F3F03070E1C38381C0E07030F82
:1019A0001F38381C1C38381F0F30381C0F07070F22
:1019B0001C3830000133333333333B1F0F30383C96
:1019C0003E373331303030000000010F1F38300017
:1019D00000000000003F3F00000000000030381F02
:1019E0000F01000000000000000C0E0703010000C2
:1019F0000103070E0C0000000040800804201002C4
:101A000001111A1D1A231A301A371A441A4F1A5A7A
:101A10001A53696D706C6520342D434800542D4372
:101A2000757400537469636B7920542D4375740089
:101A3000562D5461696C00456C65766F6E5C44652B
:101A40006C74610048656C6920536574757000475B
:101A500079726F20536574757000536572766F20CC
:101A600054657374000000891112239B322446AD23
:101A7000573665BF74488CC19D5AAFD3BE6CCAE55A
:101A8000DB7EE9F7F88110080193331A22A5562C62
:101A900047B7753E64C99C408DDBBF52AEEDDA643A
:101AA000CBFFF976E802218B30100299132667AF3D
:101AB000763444BD554AADC3BC588ED19F6EEBE71A
:101AC000FA7CC8F5D983310A2091121803A7772E22
:101AD00066B5543C45CBBD42ACD99E508FEFFB66FA
:101AE000EAFDD874C904428D5316619F702004A981
:101AF000153227BB364CCEC5DF5EEDD7FC6888E1DA
:101B0000997AABF3BA85520C4397711E60A11428E1
:101B100005B3373A26CDDE44CFDFFD56ECE99860B9
:101B200089FBBB72AA06638F7214409D512225ABBC
:101B3000343006B9174EEFC7FE5CCCD5DD6AA9E399
:101B4000B8788AF19B87730E6295501C41A3352AA1
:101B500024B1163807CFFF46EEDDDC54CDEBB96279
:101B6000A8F99A708B088481951AA793B62CC2A500
:101B7000D33EE1B7F04008C919522BDB3A644EED71
:101B80005F766DFF7C899400859BB712A6ADD22449
:101B9000C3BFF136E0C1184809D33B5A2AE55E6C51
:101BA0004FF77D7E6C0AA583B4188691972EE3A724
:101BB000F23CC0B5D14229CB38500AD91B666FEF31
:101BC0007E744CFD5D8BB502A499961087AFF32609
:101BD000E2BDD034C1C3394A28D11A580BE77F6E11
:101BE0006EF55C7C4D0CC685D71EE597F42880A168
:101BF000913AA3B3B2444ACD5B5669DF78600CE9F1
:101C00001D722FFB3E8DD604C79FF516E4A99020C8
:101C100081BBB332A2C55A4C4BD7795E68E11C68D0
:101C20000DF33F7A2E0EE787F61CC495D52AA1A3A3
:101C3000B03882B193466BCF7A5448DD59622DEBB0
:101C40003C700EF91F8FF706E69DD414C5ABB12288
:101C5000A0B9923083C77B4E6AD5585C49E33D6A90
:101C60002CF11E780F00BD1911241FBECFEFD0E15B
:101C7000DEBFCDBF11E0A0E0B1E0E6EAFEED02C0BC
:101C800005900D92A434B107D9F71EE0A4E4B1E0A9
:101C900001C01D92AC39B107E1F71CE1C8E6DCE1F7
:101CA00004C02297FE010E940C6FC636D107C9F707
:101CB0000E94ED180C94516F0C9400003091B70401
:101CC00022B78091B7043817C9F7932F80E030E02E
:101CD000282B392BC901089529E282029001112491
:101CE000359527953595279587FD815C86FB880F6F
:101CF000880B80F9992787FD9095281B390BC9011E
:101D00000895F8942091D70D3091D80D7894C90199
:101D10000895482F50E09A01220F331F63E0440FCB
:101D2000551F6A95E1F7240F351F22543E4FC90114
:101D3000089590E09C01220F331F220F331F280FBC
:101D4000391F22503D4FC9010895AF92BF92CF92E3
:101D5000DF92EF92FF920F931F93CF93DF93C82EE2
:101D6000162FEA01F22ED02E57FF10C022FF02C01C
:101D70008CE101C08FE09C2D981B892F612F4DE2D3
:101D80002F2D0E942C5DD095C195DF4F2D2D2F2139
:101D90008C2D612F4AE30E942C5D8F2D90E0B4E0E2
:101DA000AB2EB12CA822B922F2FE02C0E2E001C0A3
:101DB000E0E0CE016CE370E00E94BA6E9B01442724
:101DC00037FD4095542F0F2D00618E2F8C0D612F04
:101DD000A2E0EA2E0E942C5FA114B10411F0ECE104
:101DE00001C0E1E1CE016CE370E00E94BA6E9C019B
:101DF000442737FD4095542F0D2D00618E2F8C0DFB
:101E0000612FF2E0EF2E0E942C5FDF91CF911F91A6
:101E10000F91FF90EF90DF90CF90BF90AF9008951B
:101E20000F931F93062F122F206250E00E946260D2
:101E300017FD07C08091A90D602F46E7212F0E9452
:101E40002C5D1F910F910895242F409108010E944D
:101E5000100F08950F93022F442319F44FE257E017
:101E600020C04530A8F4E0918801F0E0EE0FFF1F9C
:101E7000EE0FFF1F3197E40FF11DE051FB4F44912E
:101E800050E0440F551F440F551F4756594F09C086
:101E9000453250F450E0440F551F440F551F46562D
:101EA000594F24E00E94EF5D0F910895FF920F9328
:101EB0001F93182FF62E022F442321F448E956E0F1
:101EC00024E00EC08A5E4A3008F485506F2D50E041
:101ED000202F0E946260812F6F2D45E956E022E09D
:101EE0000E94EF5D1F910F91FF9008950F931F9334
:101EF000DF93CF9300D0CDB7DEB7382F162F942FB6
:101F0000022F442329F0463139F04A3E81F408C0BB
:101F10008A5F41E956E007C08A5F4DE856E003C09A
:101F20008A5F49E856E0202F0E941F5E28C0409536
:101F3000441F4427441F81E2841B482F832F398389
:101F40009A830E942C5D3981832F8A5F9A81E92FC1
:101F5000FF27E7FDF095F7FF03C0F095E195FF4FF0
:101F6000FF27E7FDF0953197AF01440F551F4E0F46
:101F70005F1F475B594F612F23E00E94EF5D0F9079
:101F80000F90CF91DF911F910F91089589E496E012
:101F90000895DF92EF92FF920F931F93D82EE62EB3
:101FA000F42E1091AF01E12FFF27E7FDF095F7FF29
:101FB00003C0F095E195FF4FE031A4F483E0E8021F
:101FC000F0011124E85EF94F8D2D6E2DAF0123E055
:101FD0000F2D0E94EF5D1F3F3CF58D2D86506E2D1D
:101FE00041E21FC08D2D8650E53264F411161CF4B9
:101FF000412F4F5002C0412F415F6E2D2F2D0E9467
:10200000760F12C011161CF4412F445202C0412F0A
:102010004C5D6E2D2F2D0E94760F8D2D8E5E6E2DB8
:102020004DE62F2D0E942C5D1F910F91FF90EF9098
:10203000DF9008958C3038F4E82FF0E0EE0FFF1FAA
:10204000EF50FB4F2AC0803198F4E82FF0E0DF0119
:10205000AA0FBB1FA257BB4FEE0FFF1FE25AFE4F46
:102060002D913C91119780819181281B390B0AC0D9
:10207000843158F4E82FF0E0EE0FFF1FE257FB4FDA
:1020800020813181220F331F0DC0843248F4E82FA4
:10209000F0E0EE0FFF1FE952FB4F2081318102C0BB
:1020A00020E030E0C9010895AF92BF92DF92EF9235
:1020B000FF920F931F93DF93CF9300D0CDB7DEB77E
:1020C000F82E463008F0DEC0882309F4DEC08631E1
:1020D00019F08A3E19F4D6C061E0D7C0992787FD70
:1020E00090959C0197FF04C022273327281B390BAA
:1020F0002A307CF41F144CF02DE030E0A901481B7D
:10210000590BCA010E94CC61BAC00D960E94CC61E5
:10211000BBC02A50A22EBB249501220F331F2A0DCB
:102120003B1D2C553E4FF901E85AFD4F5081552378
:1021300009F4A8C0453029F4F501EE57FB4F808122
:102140009CC0F901EA5AFD4FD080295A3D4FF90150
:10215000E080553008F4A6C0583060F08D2D8150D5
:102160004A8359830E941A108C018E2D81500E943F
:102170001A10A2C020E030E000E010E0583088F4EF
:10218000553088F5523009F462C0533020F4513094
:1021900009F06EC057C05330D1F0543009F068C018
:1021A0001CC05A3009F44EC05B3038F4583009F482
:1021B0003FC0593009F05CC040C05C3009F44CC0ED
:1021C0005C3008F444C05D3009F052C04AC017FFCB
:1021D00039C0109501951F4F35C017FF38C01095B5
:1021E00001951F4F34C0142F1F5F8D2D60E0412FCC
:1021F0000E945410082F8E2D60E0412F0E94541031
:10220000F501EE0FFF1FEA0DFB1DE450FC4F90811E
:10221000953029F4002361F1882341F52AC09630D6
:1022200029F4002319F5882319F120C0802721C043
:1022300081E002171307E1F41CC081E002171307C5
:10224000C1F416C081E0201731079CF011C081E075
:102250000217130774F00CC081E0021713074CF447
:1022600007C081E02017310724F402C081E001C0DB
:1022700080E0F501EE57FB4F80831F142CF061E0E6
:10228000682703C060E001C0682F862F0F900F9071
:10229000CF91DF911F910F91FF90EF90DF90BF9052
:1022A000AF9008958D2D81504A8359830E941A1052
:1022B0008C018E2D0E946C0E9C014A8159815ECF4B
:1022C00086B380958E7708950E9460118823E1F788
:1022D0000E943B6108958091750160E040E00E949A
:1022E0005410882331F480919F049091A0040097AA
:1022F00011F0C79A0895C79808950F931F93CF932D
:10230000DF93EC018B010E94C25C82E260E043E05B
:1023100056E024E00E941F5E80E2BE010E94465EFD
:1023200088E2B8010E94465E80E36DEE75E00E948F
:10233000465E0E94CC60809172010E94C2600E9441
:102340006411DF91CF911F910F9108950F93AB010D
:1023500060E123E000E00E94EF5D0F910895DF92BD
:10236000EF92FF920F931F93CF93DF93809187019A
:1023700081FD83C080E895E06AE675E00E947D11EA
:1023800090919F01892F887341F0883131F0883214
:1023900021F0803311F0883329F4892F877C8860FD
:1023A00080939F0100E010E065E1E62EF12C08C06B
:1023B000C701801B91090E94CC61110F182B0F5F80
:1023C0000830B0F3D0909F01D12680E060E143E572
:1023D00055E026E100E00E94EF5DCD2DD0E0CE017A
:1023E00080FF05C082E069E476E00E94A611C1FF8B
:1023F00005C087E16CE476E00E94A611C2FF05C02B
:102400008CE26FE476E00E94A611CE018873907092
:102410000097B1F0012F13FF05C081E462E576E07B
:102420000E94A61104FF05C081E465E576E00E94E4
:10243000A61105FF05C081E468E576E00E94A611BB
:10244000C6FF05C086E56BE576E00E94A611D7FEC3
:1024500005C08BE66EE576E00E94A6110E94CC6076
:1024600080919F01181749F00E946011882329F478
:102470000E946B1100E010E09BCFDF91CF911F9184
:102480000F91FF90EF90DF9008951F93CF93DF930C
:102490000E94601120E030E011E0482F50E02F5FF3
:1024A0003F4FBA01022E02C0759567950A94E2F774
:1024B00060FD03C01F5F183091F71150163030F5E2
:1024C000812F0E943D57882309F110937101812FBC
:1024D0000E94415781E00E9410580E94C25C86E130
:1024E00060E04BE455E024E00E941F5EC4EAD1E0C6
:1024F0001AE04991812F68E124E00E942C5D155F6C
:102500001837B9F70E94CC600E946411DF91CF9117
:102510001F910895CF93DF93EC010E94C25C82E289
:1025200060E043E455E024E00E941F5E88E1BE01C4
:102530000E94465E0E94CC60809172010E94C2603F
:10254000DF91CF9108951F93CF93DF93EC01162F66
:102550000E94C25C82E260E04DE355E024E00E940C
:102560001F5E88E1BE010E94465E8CE168E34FE297
:1025700055E00E944E5E0E94CC60112319F48091B8
:10258000720101C089E10E94C26082E10E94EA6D8D
:102590000E9464110E9460118823C9F480916B0E1F
:1025A000833019F4A89510926B0E8091750160E04C
:1025B00040E00E945410882331F480918C018823DC
:1025C00011F4112311F0C79AE5CFC798E3CFDF913B
:1025D000CF911F91089580918104882351F081E962
:1025E00095E060E00E94A312809181048E7F809329
:1025F000810408958091870187FD07C0887329F4BD
:102600008CEB95E060E00E94A31208958091870111
:1026100082FD0AC00E943159883C910528F489E066
:1026200096E060E00E94A3120895EF92FF92CF938C
:10263000DF93A82FAF70A6509091B601923074F03E
:10264000292F332727FD309521503040C1E0D0E0BD
:1026500002C0CC0FDD1F2A95E2F79C2FA83008F0AE
:102660009CC06A2F659570E0FB01EE0FFF1FE050E4
:10267000FF4F0190F081E02DB081992379F4CB2FA9
:10268000DD27C7FDD095D7FF03C0D095C195DF4F9B
:102690009C2FC7FD9D5F959595959F5F4091880103
:1026A00050E04170507022E030E0241B350B2617BB
:1026B000370769F42091B5012F7009F473C021E048
:1026C00094E030918A0130FF03C0919501C020E071
:1026D0004B2F552747FD5095C92FDD27C7FDD095B6
:1026E000A0FF03C0C40FD51F04C0BA016C1B7D0B33
:1026F000EB01209729F07E019F2D9B2797FF0BC0B0
:10270000222349F4BB2339F010820E942B6286E118
:102710000E94EA6D41C0CE0184589F4F893F9105C8
:10272000B8F4C08386E00E941058CE0183589F4FB2
:102730008B3F910588F5D7FF03C0D095C195DF4F3A
:10274000D595C795D595C795BE01645C462F1FC02A
:102750001C161D0614F48DE701C083E8808386E013
:102760000E941058CE0183589F4F8B3F9105A0F4D3
:10277000CE01D7FF03C0909581959F4F64E070E034
:102780000E94BA6E709561957F4F462F445C89E434
:1027900094E065E10E94776C80E0DF91CF91FF903B
:1027A000EF90089520E08DCF8F929F92AF92BF92CD
:1027B000CF92DF92EF92FF920F931F93CF93DF930D
:1027C000182FEB015A016901802E84FF06C01F708B
:1027D000106694E0992E05E003C085E0982E04E091
:1027E000802F8066181761F0802F8064181741F0E1
:1027F00080912005882369F0133611F0133449F4D1
:102800007E010894E11CF11C83E10E94EA6D892D90
:1028100018C0992D9066191761F0992D90641917B9
:1028200041F0882309F474C0123619F0123409F00B
:102830006FC07E010894E108F10884E10E94EA6D0E
:10284000802F90E00E94CC61882351F0EE24FF2479
:10285000EC1AFD0A892D0E942B62802F0E942B62A8
:10286000A114B10491F481E0C816D10471F41036BA
:1028700061F41092200501E0E02EF12C209711F078
:10288000EE24FF2480E60E942B6220919C0430916C
:102890009D04E21AF30ACE14DF0444F4812F0E944F
:1028A0002B6283E10E94EA6D76010AC0EA14FB0400
:1028B0003CF4812F0E942B6284E10E94EA6D750135
:1028C000EC16FD06A9F0E114F10451F4812F0E94E9
:1028D0001C62D7FF02C083E101C084E10E94EA6D5F
:1028E000882D83700E94105881E08093990402C063
:1028F00010929904C701DF91CF911F910F91FF9022
:10290000EF90DF90CF90BF90AF909F908F90089501
:102910007E01A6CF0F93772767FD7095552747FD5A
:102920005095332727FD30950E94D4130F910895B9
:102930000F93772767FD7095552747FD50953327EF
:1029400027FD309502E00E94D4130F9108950F9354
:10295000772767FD7095552747FD5095332727FD4D
:10296000309501E00E94D4130F910895E0919804EE
:10297000F0E0EE0FFF1FE057FB4F8081918108953B
:1029800090919804992319F4882331F418C088236E
:1029900019F4892F815001C080E08093980487E169
:1029A0000E94EA6DE0919804F0E0EE0FFF1FE257FD
:1029B000FB4F0190F081E02D8EEB099508958BE19E
:1029C00095E060E00E94A3120895FC01A091980494
:1029D000B0E0AA0FBB1FA257BB4F8D939C938FEB08
:1029E000099587E10E94EA6D0895CF93DF93EC018A
:1029F00080919804982F9F5F90939804953040F0B1
:102A00008093980488E095E060E00E94A3120FC0D4
:102A100087E10E94EA6DE0919804F0E0EE0FFF1F5D
:102A2000E257FB4FD183C0838FEBFE010995DF9105
:102A3000CF91089589E494E00E94766B882311F089
:102A400084E105C08091B804882321F081508093EF
:102A5000B80407C09091630081E091FF80E080930B
:102A6000B9048091B90408951092A3041092A504AA
:102A70001092A4041092A204089520919F04309112
:102A8000A0042115310531F0215030403093A004CD
:102A900020939F04882369F040918C0150E084EFDB
:102AA00091E0489F9001499F300D589F300D1124AF
:102AB00002C020E030E08091A104882369F0609199
:102AC000940170E044EF51E0649FC001659F900D58
:102AD000749F900D112402C080E090E040919F040B
:102AE0005091A0044217530720F43093A004209380
:102AF0009F0420919F043091A0042817390720F4E7
:102B00009093A00480939F040E946B110895E82F76
:102B1000F0E0E050FB4FE491F0E0EE0FFF1FE454D3
:102B2000FB4F20813181C9010895CF92DF92EF924E
:102B3000FF920F931F93DF93CF930F92CDB7DEB722
:102B400020E0CC24DD24822F29830E948715092FC1
:102B500010E0C00ED11E29812F5F2430A1F7C601DD
:102B60000F90CF91DF911F910F91FF90EF90DF9029
:102B7000CF9008951F930E94810E41E02091EF04B1
:102B80003091F0048217930709F440E040939E04CB
:102B90000E94810E9093F0048093EF0485E295E00B
:102BA00060E00E94A63580919E04882309F4CBC082
:102BB0008091A20480FF14C08091A304982F9F5F8E
:102BC0009093A304943660F083568093A30480917D
:102BD000A4049091A50401969093A5048093A40465
:102BE00080E00E941E580E94C25C0E943E610E94CA
:102BF0001513182F0E943D152091FD043091FE04FD
:102C000080919A0490919B04821B930B60E270E088
:102C10000E94BA6E70939D0460939C0461157105C7
:102C200091F08091ED049091EE04821B930B62E091
:102C300070E00E94BA6E70939D0460939C04309380
:102C40009B0420939A043093EE042093ED0480912A
:102C50008A0185FF04C010929D0410929C04E091AB
:102C60009804F0E0EE0FFF1FE257FB4F0190F08158
:102C7000E02D812F09950E94CC600E941A158823AF
:102C800021F0809165008F7E03C080916500806196
:102C9000809365000E94810E8F7190708230910543
:102CA00009F04FC087E00E9487159C01E4E0220FE5
:102CB000331FEA95E1F768E070E00E94BA6E409138
:102CC0007401552747FD50954A5F5F4F649FC001CF
:102CD000659F900D749F900D1124820F931F20917A
:102CE0008A0126FD05C06091090170910A0102C0A8
:102CF00060EF70E02091080130E02F5F3F4F0E94AD
:102D0000A66E260F371F35952795209308018091D1
:102D1000EC04805E8093EC04882399F48091730125
:102D2000281778F4223368F081E10E94EA6D8091DF
:102D30008A0183FF06C082E390E09093A004809311
:102D40009F041092A1041F910895ACEBB4E0ECEC49
:102D5000F4E060E0862F806487B9369A4089518913
:102D60008D919C91119796958795840F951F8E7FD5
:102D700011969C938E9320813181C901840F951FF8
:102D800096958795918B808B349BFECF349A84B136
:102D900095B1820F931F96958795819391936F5F5D
:102DA00012966830B9F60895EF92FF920F931F9331
:102DB000CF93DF9380918A0184FD44C00E946B1100
:102DC0000E94C25C80E060E045ED50E020E000E061
:102DD0000E94CD5C8091900184FD08C080E068E392
:102DE00045E951E02AE000E10E94EF5D0E94CC60DD
:102DF000809172010E94C2600E94641100E20E94F0
:102E0000A5160150E1F70E9495158C010E94810ED4
:102E1000EC01C057DE4F0DC00E94A5160E9495150B
:102E20007C010E946011882369F4E016F10651F4D8
:102E300006C00E94810EC817D90771F703C00E940F
:102E40006B11F7CFDF91CF911F910F91FF90EF9012
:102E50000895ECEBF4E040E012C067B9369A349B79
:102E6000FECF349A24B135B1820F931F5150A9F788
:102E700096958795819391934F5F483031F054E058
:102E800080E090E0642F6064E8CF0895ECEBF4E01C
:102E900020E0822F806487B9369A349BFECF349A23
:102EA00084B195B1880F991F819391932F5F28303A
:102EB00081F70895FF920F931F93CF93DF93809133
:102EC000870180FD3AC08091880190E08170907008
:102ED00002E010E0081B190BF801EE0FFF1FEC5B7E
:102EE000FE4FC181D281609687859089C81BD90B1E
:102EF0000E944617F02E802F0E948715C817D90709
:102F0000E4F40E9460118823C1F40DC00E944617AA
:102F10008F2D0E948715C817D9077CF40E94601175
:102F2000882341F00AC08BED95E06CEC75E00E94BF
:102F30007D11ECCF0E946B11E9CFDF91CF911F91F2
:102F40000F91FF9008958EE587B9369A349BFECF96
:102F5000349A84B195B104964091090150910A01C7
:102F60009A0163E0220F331F6A95E1F7241B350BAA
:102F7000820F931F23E0969587952A95E1F790930A
:102F80000A0180930901089578941F920F920FB659
:102F90000F9211248F938091B7048F5F8093B704B1
:102FA0008F910F900FBE0F901F90189578941F92DD
:102FB0000F920FB60F9211242F933F934F935F936D
:102FC0006F937F938F939F93AF93BF93EF93FF93F1
:102FD000F89487B78D7F87BF789481B78E5F81BF64
:102FE00090914B0480914D04882379F08091930156
:102FF000882349F0813051F480919B0E890F809392
:103000009B0E87FF02C01B9A01C01B9880910B0189
:10301000982F915090930B01882371F48DE4809345
:103020000B0189E494E00E948A6B0E943C628091CB
:103030006B0E826080936B0EF89487B7826087BFB7
:103040007894FF91EF91BF91AF919F918F917F9174
:103050006F915F914F913F912F910F900FBE0F9005
:103060001F90189578941F920F920FB60F9211240B
:103070001F932F933F934F935F936F937F938F9300
:103080009F93AF93BF93EF93FF9320918000309174
:103090008100F89480917D008F7D80937D007894ED
:1030A0008091BA049091BB04A901481B590BCA0135
:1030B000969587953093BB042093BA041091B6047B
:1030C000212F2150283058F59C012152334055E0E2
:1030D0002737350708F5E12FF0E0EE0FFF1FEC551D
:1030E000FB4FAC014C5D554020918E01332727FDED
:1030F0003095265F3F4F429FC001439F900D529FE6
:10310000900D11246AE070E00E94BA6E71836083B2
:103110001F5F1093B6040CC01092B60409C0815A08
:103120009F402EE28F3D920718F481E08093B60411
:10313000F89480917D00806280937D007894FF9167
:10314000EF91BF91AF919F918F917F916F915F911F
:103150004F913F912F911F910F900FBE0F901F9095
:103160001895EDE9FEE09F0181918535E1F32C5939
:103170003E40C9010895CF93DF930E945E0EEC019B
:1031800080918B01813019F40E94A51607C082300E
:1031900019F40E94291702C00E9446178EE587B9CC
:1031A0000E94BA150E94A31780916B0E833019F408
:1031B000A89510926B0E0E945E0E8C1B9D0B2091A9
:1031C000C7063091C8062817390720F49093C8061F
:1031D0008093C706DF91CF9108951F938FEF8ABB2D
:1031E0001BBA91E897BB9EE798BB9EE394BB91EC1A
:1031F00095BB11BA82BB88E082B987EF83B9109280
:1032000061001092620084E1809364008BEF8093F0
:1032100065000E948C600E942E6E80E487B985E86C
:1032200086B987E083BF8CE981BF87B7836087BF9A
:103230001FBC8AE08EBD10928B0082E880938A00CA
:1032400080917D00806280937D00EDB7FEB732975C
:1032500085E502C0808331979EE0EC39F90709F0DB
:10326000C8F7789484E89FE390938F0480938E044A
:1032700089E10E94C2600E94C957109171010E94A9
:103280004512809172010E94C26050918C01409160
:103290009401451778F4652F70E024EF31E0629FC8
:1032A000C001639F900D729F900D11249093A00414
:1032B00080939F04541770F450E024EF31E0429F54
:1032C000C001439F900D529F900D11249093A00434
:1032D00080939F040E946B1180919301813039F497
:1032E00080918A0184FD03C087E00E94EA6D0E94FC
:1032F000D4160E9406130E9446170E945A170E9475
:10330000AF110E94FA120E94EB120E94641180EF2A
:1033100090E090930A01809309010E94E1692DE0F9
:1033200088E190E00FB6F894A89581BD0FBE21BD4D
:1033300085E295E060E00E94A63584E691E30E9474
:10334000F51481E00E94C014809172010E94C26055
:1033500080917101181729F081E00E9410580E9495
:10336000AC5880ED97E09BBD8ABD80E186BF87B7F2
:10337000806187BF0E94BB18FDCF89E494E00E9462
:10338000736B089529E282029001112435952795E7
:103390003595279587FD815C86FB880F880B80F922
:1033A000992787FD9095281B390BC90108959C0129
:1033B000E5E035952795EA95E1F7AC01440F452FF7
:1033C000441F550B280F391F892F990F990B85958D
:1033D000280F391F241B350BC9010895F89420913B
:1033E000D70D3091D80D7894C9010895AC0180E0D3
:1033F00060E021E00E941F5E08950F931F93CF931A
:10340000DF93182F88E198E00E94F619113658F0E2
:10341000133628F0133639F48BE19BE102C084E8BF
:103420009FE30E94E51486E068E040E158E00E94D6
:103430004E5E40913F06509140068AE268E020E0EF
:1034400000E00E94A50E40914106509142068EE494
:1034500068E020E00E94A50E86E060E148E058E0C8
:103460000E944E5E40914306509144068AE260E11C
:1034700020E00E94A50E4091450650914606F4E0DA
:1034800056954795FA95E1F78EE460E120E00E94B9
:10349000A50E86E660E044E058E00E944E5E409152
:1034A0003D0650913E068EE460E020E00E94A50EAD
:1034B0008091C3069091C4068937910528F08091C8
:1034C000C206C82FD0E002C0C0E0D0E082E06CE3CA
:1034D0004EE70E94CC5E85E06CE143E20E94D05E44
:1034E0001BE0812F6BE343E00E94D05E1A5F13382C
:1034F000C1F716E00CE3FE01E65BF94F4081602F57
:10350000641B812F0E94D05E2196C837D10510F030
:10351000C0E0D0E02091C20630E0C217D30719F016
:103520001F5F1E3741F7DF91CF911F910F910895D3
:103530001F93CF93DF93182F8DE198E00E94F61927
:10354000113631F40E94496E84E89FE30E94E5142D
:10355000C9E7DEE01CE04991812F68E120E10E948B
:103560002C5D812F60E24F8520E10E942C5D1A5F67
:103570001C3689F78091990E882309F458C00E945F
:10358000476E83E090E00E94CC61882351F08091E7
:10359000410190914201807D90709093420180930F
:1035A000410182E090E00E94CC61882351F080913B
:1035B000410190914201807B9070909342018093F1
:1035C000410185E090E00E94CC61882351F0809118
:1035D00041019091420180779070909342018093D5
:1035E000410184E090E00E94CC61882351F08091F9
:1035F000410190914201807E9070909342018093AE
:1036000041011092990E80914101909142010E94D6
:103610004F6E8FE99FE00197F1F700C000000E9414
:10362000456E80EF90E09093420180934101DF91DD
:10363000CF911F9108951F93182F82E798E00E9461
:10364000F6191236E1F0133628F4103631F011363F
:10365000E9F418C01336D1F415C08FEF97E09093BA
:103660000D0180930C011092C6061092C5061092AF
:10367000C8061092C70687E10E94EA6D07C08DEF69
:1036800099E102C084E89FE30E94E51488E063E6C4
:1036900078E00E94465E4091C5065091C606569558
:1036A000479584E568E00E94726080E164E578E017
:1036B0000E94465E40910C0150910D015695479530
:1036C00084E560E10E94726088E165E478E00E9430
:1036D000465E4091C5065091C60680910C019091BE
:1036E0000D01481B590B5695479584E568E10E94EA
:1036F000726080E26CE378E00E94465E2091C7062B
:103700003091C80684E690E0289FA001299F500DC3
:10371000389F500D1124A4E056954795AA95E1F7DE
:1037200084E560E220E30E94626088E264E378E07E
:103730000E94465E0E94B118AC018FE368E20E94CD
:10374000525E82E168E342E258E00E944E5E1F91C1
:10375000089586EE9FE008950F9393E0499FA0019E
:1037600011244152504F01E0222309F400E023E0EC
:103770000E94EF5D0F9108950F9393E0499FA00180
:1037800011244852504F01E0222309F400E023E0C5
:103790000E94EF5D0F910895FF920F931F93F82EF3
:1037A000062F142F80E860E0402F50E0212F0E9468
:1037B00062600A3010F00FE601C005E7802F60E07C
:1037C0004FE2212F0E942C5D4F2D50E04F5F5F4F45
:1037D000802F60E0212F0E9462601F910F91FF9067
:1037E00008956F927F928F929F92AF92CF92DF92C5
:1037F000EF92FF920F931F93CF93DF93EC01162F5D
:10380000D42E49016090F9047090FA048091C808A0
:103810009091C9088619970920E430E0B9010E9407
:10382000BA6E462F60932305E091FB04F091FC04EF
:103830008091C6089091C7088E1B9F0BB9010E940A
:10384000BA6E862F60932405442321F07092C90834
:103850006092C808882321F0F093C708E093C60857
:1038600080912205882321F480918A0185FF06C07A
:1038700010922305109224051092220560912305D1
:10388000662351F480912405882331F480919C04AF
:1038900090919D04009781F040918C0150E024EFBD
:1038A00031E0429FC001439F900D529F900D112423
:1038B0009093A00480939F048114910409F456C04E
:1038C0008881882309F04BC0662331F1809120055F
:1038D000882311F5ED2DE61BE7FDE0E0202F30E019
:1038E0008E2F992787FD90958217930714F0E02F6C
:1038F000E150FF27E7FDF0958D2D90E0E817F907DF
:1039000049F0EE0FFF1FE80DF91D25913491C90113
:103910000E94E51410922305153641F4DD2011F0C4
:10392000ED2D01C0E02FF0E031970FC01436C9F43F
:103930002D2D30E0802F90E00197281739071CF4D7
:10394000ED2DEF5F01C0E0E0F0E0EE0FFF1FE80DAE
:10395000F91D25913491C9010E94E51402C040E08F
:1039600001C041E08D2D602F0E94CC1BE114F104B9
:1039700051F098818C2D9C1508F4892FF701E80FE0
:10398000F11D549101C050E080912005882309F079
:103990004FC080912405882329F14881481B47FDA9
:1039A00040E0242F332727FD30958A2D90E02817FB
:1039B00039070CF04A2D48838981E114F10459F04C
:1039C000C41608F44C2DF701E40FF11DE4918E1795
:1039D00018F4E82F01C0E0E0E98380E68093D90D78
:1039E000109224058881882319F190912305992349
:1039F000F9F04981E114F104B1F0491B47FD40E0C1
:103A00009C2D8C1508F4982FF701E90FF11DE49116
:103A1000242F332727FD30958E2F90E02817390764
:103A20001CF04E2F01C040E0498380E68093D90D01
:103A3000103651F1113690F4133409F480C0143467
:103A400030F4113279F1123409F09CC06AC0143498
:103A500009F43FC0153409F095C04FC01436E9F1A0
:103A6000153638F4123609F45FC0133609F08AC0EF
:103A700069C01138A1F01F3B21F0153609F082C052
:103A800040C01982188212C0552309F47BC081E01E
:103A900090912005911180E08093200573C01092D1
:103AA00020050DC080912005882319F01092200573
:103AB00069C08881882319F08114910421F480E081
:103AC0000E94C0145FC087E10E94EA6D19821882CB
:103AD00056C08981851709F455C0E114F10409F431
:103AE00051C080912005882309F04CC08981851739
:103AF00010F48F5F12C0198242C08981882309F4B3
:103B000041C0E114F10409F43DC0809120058823EF
:103B1000C9F58981882319F08150898330C0598380
:103B20002EC088818A1571F180912005882351F576
:103B300088818A1510F48F5F0DC018820EC08881AD
:103B4000882301F1809120058823E1F4888188236E
:103B500019F08150888301C0A8828981E114F104A1
:103B600061F098819C1508F4C92EEC0CF11CF7014A
:103B70009491891718F4982F01C090E0998380E6FA
:103B80008093D90DDF91CF911F910F91FF90EF900E
:103B9000DF90CF90AF909F908F907F906F9008951F
:103BA0004F925F926F927F928F929F92AF92BF924D
:103BB000CF92DF92EF92FF920F931F93DF93CF93F9
:103BC0000F92CDB7DEB7D82E8AE69AE00E94F6199A
:103BD0008AE498E06D2D41E024EE37E006E052E7FC
:103BE000E52E5AE0F52E15E0C12EB6E0AB2E0E9470
:103BF000F11B80904A0890904B088091630081FFF0
:103C000007C08AE268E144E65AE00E944E5E60C165
:103C100082E168E045E55AE00E944E5E8A94809118
:103C20002005882319F0A2E0CA2E02C0CC24C39438
:103C3000EE24FF2410E1A82CBB24A7FCB094F4E0F0
:103C40006F2E712C2701440C551C8EE791E0480E15
:103C5000591E4E2D4F5F80E0612F20E00E942A0FF9
:103C6000AE14BF0411F491E0911090E0F2012181B3
:103C7000229526952695237030E0A901440F551F03
:103C8000420F531F455B554F992311F400E001C0CB
:103C90000C2D88E1612F23E099830E94EF5D9981CB
:103CA0009923C1F0809120058823A1F0F201618160
:103CB00062956695669563708D2D40E022E00E94C6
:103CC000A7148295880F880F807CF20191819F73E1
:103CD000982B9183AE14BF0421F401E0F92DF1304B
:103CE00009F000E0F2018181880F880F85958595A4
:103CF000FDE08F02C0011124B3010E94BA6EAB0136
:103D0000002311F420E001C02C2D82E4612F0E94D9
:103D100062600023A9F080912005882389F0F201D8
:103D20006181660F660F659565958D2D41EE2FE1DA
:103D30000E94A7148F73F2019181907C982B91833C
:103D4000AE14BF0421F491E0F92DF23009F090E0B7
:103D5000F2012081277030E0A901440F551F420F66
:103D6000531F425C554F992311F400E001C00C2D04
:103D700088E4612F23E099830E94EF5D9981992364
:103D800091F080912005882371F0F20160816770C5
:103D90008D2D40E023E00E94A7148770F2019081EE
:103DA000987F982B9083AE14BF0421F401E0F92D85
:103DB000F33009F000E0F2014081459545954595C5
:103DC000002311F420E001C02C2D8AE5612F0E9410
:103DD000760F0023B1F080912005882391F0F20145
:103DE00060816595659565958D2D4AEE26E10E9469
:103DF000A714880F880F880FF20190819770982B75
:103E00009083185F0894E11CF11C103309F01ACF5D
:103E100080E363E37AE00E94465E40918E0155277D
:103E200047FD5095465F5F4FF82DF43011F421E2C5
:103E300001C020E28EE460E30E946260282D2430FD
:103E400049F48D2D60918E0146EF28E20E94A7145F
:103E500080938E01EE24E394882D853009F0EE24C2
:103E600080E068E34FE25AE02E2D0E941F5E46EA92
:103E7000A42E44E0B42E06E711E090E3F501419151
:103E800051915F01F801219131918F01421B530B38
:103E9000440F551F892F68E320E299830E946260D6
:103EA0009981985E903951F7EE2091F0FD2DF03612
:103EB00079F4A6E7B1E0E6EAF4E088E001900D923B
:103EC0008150E1F781E00E94105887E10E94EA6D7D
:103ED0000F90CF91DF911F910F91FF90EF90DF90A6
:103EE000CF90BF90AF909F908F907F906F905F909A
:103EF0004F900895AF92CF92EF92FF920F93AE2C16
:103F0000EE24FF24CC240E94F11B0F91FF90EF9030
:103F1000CF90AF900895EF920F93DF93CF930F92CE
:103F2000CDB7DEB7682F88E79AE069830E94F6195B
:103F30008CE498E0698142E024EE37E006E0EE246C
:103F40000E947A1F80E167E677E00E94465E88E182
:103F500064E377E00E94465E80E267E477E00E94D7
:103F6000465E88E268E577E00E94465E80E367E7A8
:103F700077E00E94465E0F90CF91DF910F91EF9016
:103F80000895CF92DF92EF92FF920F931F93DF93EA
:103F9000CF9300D0CDB7DEB7682F87EA9AE0698368
:103FA0000E94F6198EE498E0698143E024EE37E040
:103FB00006E0EE240E947A1FEEE0CE2ED12C00E027
:103FC00010E0143020F078EFF72EF00E01C0F02E44
:103FD000C6010E94CC61E82E1F5F8AE26F2D412F3F
:103FE00020E00E94760F4E2D405D84E46F2D2E2D33
:103FF0000E942C5D085F0894C11CD11C193009F780
:1040000008E3CC24DD2410E0812F90E00E94CC61F5
:10401000F82EA6014857554F80E0602F25E00E94FA
:10402000195E4F2D405D80E2602F2F2D0E942C5D88
:104030001F5F85E090E0C80ED91E0850163021F7AA
:1040400084E568E140E85AE027E00E94195E66E0F6
:10405000E62EF12C10E230E084E5612F45E857E0D0
:10406000232F00E03A830E94CD5CC7010E94CC61FF
:10407000282FC701019629830E94CC61082F29812E
:10408000422F405D8CE6612F0E942C5D402F405DE9
:1040900088E7612F202F0E942C5D3A813F5F185FD7
:1040A000E2E0F0E0EE0EFF1E3430B1F60F900F901C
:1040B000CF91DF911F910F91FF90EF90DF90CF9004
:1040C00008958F929F92AF92BF92DF92EF92FF92EC
:1040D0000F931F93CF93DF93D82E8FEA9AE00E941D
:1040E000F61980E598E06D2D44E024EE37E006E017
:1040F000EE24E3940E947A1FF0905008C1EFD4E0C0
:1041000010E000E0812CF4E09F2EA12CB12C88E17E
:10411000612F41E40E94EB5D402F4F5C8EE1612FE7
:104120000E94EB5D802F0E948715AC018AE2612F0F
:104130000E94525E0730B1F068817981882777FD4F
:104140008095982F24E630E040E050E00E947B6E9E
:10415000A50194010E94EF6E8AE5612FA9010E94DA
:1041600072600AC08F2D813011F040E201C041E23F
:104170008AE5612F0E94240F0F5F185F2296083096
:1041800031F68CE668E24CEA5AE022E00E94195EC1
:104190004091090150910A0188E760E320E00E9404
:1041A00062608F2D813059F4F09222058D2D60913F
:1041B000740141E82FE70E94A71480937401DF91F6
:1041C000CF911F910F91FF90EF90DF90BF90AF9034
:1041D0009F908F900895EF920F93E42E40E020E09F
:1041E00030E000E00E947A1F0F91EF900895AF92A7
:1041F000BF92CF92DF92EF92FF920F931F93DF93C4
:10420000CF9300D0CDB7DEB78FE161E247E10E94E6
:10421000D05E8FE167E347E10E94CC5E85E361E217
:1042200047E10E94D05E8FE161E247E10E94CC5EEF
:104230008BE461E247E10E94D05E8BE467E347E1F3
:104240000E94CC5E81E661E247E10E94D05E8BE491
:1042500061E247E10E94CC5E8AE26BE243E00E94A9
:10426000D05E89E26CE243E00E94CC5E86E56BE2C0
:1042700043E00E94D05E85E56CE243E00E94CC5EA4
:104280008091F1049091F20451E7C52ED12CB60132
:104290000E94BA6E262F8091F3049091F4040FE8E7
:1042A0001FEFB8010E94BA6E362F48E2E42EE20EEC
:1042B0009AE2F92EF60E8E2D6F2D45E02A83398372
:1042C0000E94D05E3981632F625D8E2D45E00E9491
:1042D000CC5E2A81822F845D6F2D45E00E94D05EE6
:1042E0008E2D6F2D45E00E94CC5E8091F704909159
:1042F000F804B6010E94BA6E262F8091F5049091C1
:10430000F604B8010E94BA6E062F84E5F82EF20E6C
:10431000162F165D8F2D612F45E02A830E94D05EF7
:10432000602F625D8F2D45E00E94CC5E2A81822F36
:10433000885A612F45E00E94D05E8F2D612F45E0A5
:104340000E94CC5E19EFA12E14E0B12EBAE3FB2E31
:104350000DE510E0A8E3EA2EF501819191915F014E
:1043600080509C4FB8010E94BA6ED62ED394CE2CAA
:10437000CD188F2D6C2D4D2D0E94D05E8F2D8F5F0F
:104380006C2D4D2D0E94D05E8F2D8E5F6C2D4D2D8E
:104390000E94D05EF5E0FF0E8F2D8934E9F60F9074
:1043A0000F90CF91DF911F910F91FF90EF90DF90D1
:1043B000CF90BF90AF9008954F925F926F927F928F
:1043C0008F929F92AF92BF92CF92DF92EF92FF9225
:1043D0000F931F93DF93CF930F92CDB7DEB7B82E15
:1043E00084E09BE00E94F6198DE798E06B2D45E094
:1043F00024EE37E006E0EE24E3940E947A1F109248
:104400007D0811E6E12E18E0F12EB3E5CB2EB8E0E1
:10441000DB2E8601470160E0862F69830E948715A5
:10442000D4014D915C911197282F392F6981421742
:1044300053070CF49A01F401219331934F01D801F1
:104440004D915C911197282F392F241735070CF4C3
:104450009A01F801219331938F016F5F6730E1F684
:104460008091520880932205FB2DF03219F0FF3B1A
:1044700071F40BC08F5F80935208833041F487E161
:104480000E94EA6D81E00E941058109252088091BB
:1044900052088130B1F0813020F0823009F0A4C0A0
:1044A0003FC08CE060E142EF5AE021E100E00E9471
:1044B000EF5D82E168E142EE5AE02FE00E94EF5D9D
:1044C00093C08EE160E145ED5AE02CE000E00E94EF
:1044D000EF5D82E168E143EB5AE020E10E94EF5D8D
:1044E000AFE68A2EA8E09A2E20E008E91AE3F8E663
:1044F000AF2EF5ECBF2ED7010D931D937D01F60174
:10450000A192B1926F01822F29830E948715D40155
:104510008D939D934D0129812F5F273061F764C0F2
:1045200082E160E144EC5AE020E100E00E94EF5DAE
:1045300082E168E143EB5AE020E10E94EF5DEFE6A3
:10454000AE2EE8E0BE2E75E4472E71E0572EF20144
:1045500060E4862E912CD7018D919D917D01D6012D
:104560006D907D906D019C012619370937FF03C0BE
:10457000309521953F4F23333105DCF0D5012D9146
:104580003C91318320838901081B190BC801B401B8
:104590000E94BA6E061B170B17870687C301821B82
:1045A000930B9C01B4010E94BA6E261B370B358F0A
:1045B000248FA2E0B0E0AA0EBB1E3296BFE6EB1637
:1045C000B8E0FB0641F680E090E0F20121913191E4
:1045D0002F01820F931FFDE54F16F1E05F06A9F74B
:1045E0009093700180936F010E94F7200F90CF91FC
:1045F000DF911F910F91FF90EF90DF90CF90BF90D0
:10460000AF909F908F907F906F905F904F900895A4
:10461000282F30E0C901880F991FA90163E0440FDA
:10462000551F6A95E1F7840F951FA9014F5F5F4FF2
:10463000BA01660F771FA3E0440F551FAA95E1F753
:10464000640F751F62547E4F20953095205E3F4F5A
:10465000A901440F551FE3E0220F331FEA95E1F74C
:10466000420F531F82549E4F0E941F6F8AE0E4EF57
:10467000F2E0DF011D928A95E9F782E00E9410586E
:104680000E94AC5808950F931F93CF93DF93282F68
:1046900030E0E901CC0FDD1FC90113E0880F991F3D
:1046A0001A95E1F7C80FD91F8E0102541E4FA901B8
:1046B0004F5F5F4FCA01880F991FA3E0440F551F3A
:1046C000AA95E1F7840F951F20953095205E3F4F06
:1046D000A901440F551FE3E0220F331FEA95E1F7CC
:1046E000420F531F82549E4FB8010E941F6F8AE0F1
:1046F000D8011D928A95E9F78091A108CC55DE4F2B
:104700008A8F8B8F84E68C8F82E00E9410580E94E3
:10471000AC58DF91CF911F910F910895FF920F93A5
:104720001F9385EFE5E4F5E0DF011D928A95E9F737
:1047300080913A06AEEBB1E050E021E030E060E07D
:104740007C91772311F0472F01C040E1641738F5C1
:10475000F22E032F162F1F5F802F90E0FC01EE0F2B
:10476000FF1FEE0FFF1FE80FF91FEB5BFA4F912FB2
:104770009F738081807C892B80648083F182F39495
:1047800053830F5F141738F3962F9095642F822F61
:104790008F5F890F390F340F290F240F840F772370
:1047A00059F1832F90E0FC01EE0FFF1FEE0FFF1F6A
:1047B000E80FF91FEB5BFA4F4F738081807C5483C5
:1047C000842B8068808322832F5F1A968C911A979E
:1047D000781719F41182138205C021832F5F852F6A
:1047E0008F5F8383822F5F5F1A96503219F4209374
:1047F0003A0604C03F5FA4CF80933A061F910F9101
:10480000FF900895EEEBF1E080E0908191509031BF
:1048100008F48F5F3A9692E0EE3FF907B1F70895FA
:104820001F93182F80E162EF7DE00E94465E0E9498
:104830000224482F88E760E150E020E00E94626097
:1048400080E26CED7DE00E94465E113651F481E617
:104850000E942B6281E00E94C01480ED94E20E94CD
:10486000F5141F9108950E940224803230F080E1F7
:1048700094E20E94F51481E0089580E00895EF929B
:10488000FF920F931F93DF93CF9300D0CDB7DEB786
:10489000182F813208F07BC0882319F4442341F497
:1048A00076C0803219F4442331F071C0442319F0EA
:1048B000012F0F5F02C0012F0150812F4A836983AE
:1048C0000E94890E7C01802F0E94890EFC01D70175
:1048D0008C91982F91504A816981903108F057C08E
:1048E0002081213108F053C06623A1F10E943324B6
:1048F000882309F04CC0212F30E0A9014F5F5F4FA2
:10490000CA01880F991F13E0440F551F1A95E1F74C
:10491000840F951FB901660F771FA901A3E0440F0B
:10492000551FAA95E1F7640F751F62547E4F2095BD
:104930003095205E3F4FA901440F551FE3E0220F41
:10494000331FEA95E1F7420F531F82549E4F0E9496
:104950001F6F1DC0281759F0442331F08031B8F47F
:104960008F5FF701808313C0D7019C9310C0D701DC
:10497000CF010A9604C020813C9131932D93E81712
:10498000F907C9F782E00E9410580E94AC580F90B6
:104990000F90CF91DF911F910F91FF90EF900895AD
:1049A0006F927F928F929F92AF92BF92CF92DF923F
:1049B000EF92FF920F931F93CF93DF93182F86ED03
:1049C0009DE00E94F619E0903A06EA9484EA98E0A5
:1049D000612F44E020ED37E00AE00E947A1FC0908A
:1049E000A408CC2011F41092A3081236D9F1133682
:1049F00070F41334A9F1143420F4123409F070C0A7
:104A000031C01036C1F0113609F06AC045C0103807
:104A100009F452C0113820F4133609F061C020C0E7
:104A20001E3BB9F11F3B09F05BC081E08093A208F7
:104A30001092A3082EC01C143CF481E09091A308AE
:104A4000911180E08093A3088091A3088093A2082D
:104A500080919F08882309F443C01092A30840C0A6
:104A60001092A2088091A3088823D1F141E0123668
:104A700009F040E08091A0086091A2080E943F24C4
:104A80008091A208882319F0133609F4CA94109271
:104A9000A2080E948E2324C08091A308882301F1DC
:104AA0008091A0080E9408231092A3080E948E23E0
:104AB00081E60E942B6214C01C1494F480919F081C
:104AC000882341F00E943324882321F48091A00898
:104AD0000E9443231092A30886E892E50E94F514F1
:104AE00038E0D32E77247A9423E6822E9924BB24AF
:104AF000BA9466246394E0901F05E90CFF24F70143
:104B0000EE0FFF1FEE0FFF1FEE0DFF1DEB5BFA4FC9
:104B10004081842F807C09F462C146FF06C04F7338
:104B200080E06D2D20E00E94560F1C14E4F4E70194
:104B3000CC0FDD1FCC0FDD1FCE0DDF1DCB5BDA4FA1
:104B40008981C81681F46D2D695F80E048E10E947B
:104B5000CC5E8B818093A00888818F738093A1089D
:104B600060929F08B92CF701EE0FFF1FEE0FFF1F99
:104B7000EE0DFF1DEB5BFA4F808187FF05C194812D
:104B8000C92FDD27C7FDD095AA24A3949281C9120D
:104B9000AA2486FD1FC0FE01EE0FFF1FCE01A3E079
:104BA000880F991FAA95E1F7E80FF91FEB53FE4F05
:104BB00040814695477050E04E52524F8091A30875
:104BC000882311F400E001C00A2D82E16D2D21E05F
:104BD0000E94EF5DFE01EE0FFF1FCE0163E0880F24
:104BE000991F6A95E1F7E80FF91FEC55FE4F448DC8
:104BF000552747FD50958DE26D2D2A2D0E9462604C
:104C00008091A308882311F420E001C02A2D8DE2B1
:104C10006D2D45E20E942C5DFE01EE0FFF1FCE01BF
:104C200043E0880F991F4A95E1F7E80FF91FEC550B
:104C3000FE4F438D8091A308882311F420E001C02A
:104C40002A2D86E36D2D0E942A0FFE01EE0FFF1F15
:104C5000CE0123E0880F991F2A95E1F7E80FF91F8D
:104C6000EC55FE4F458D442359F08091A3088823CD
:104C700011F420E001C02A2D8EE46D2D0E94760FE4
:104C8000FE01EE0FFF1FCE01B3E0880F991FBA950A
:104C9000E1F7E80FF91FEC55FE4F468D442391F0E4
:104CA00023E0429FA00111244A51504F8091A30854
:104CB000882311F400E001C00A2D86E66D2D23E063
:104CC0000E94EF5DFE01EE0FFF1FCE0173E0880F23
:104CD000991F7A95E1F7E80FF91FE254FE4F21E0A2
:104CE0008581882309F420E0FE01EE0FFF1FCE012D
:104CF00053E0880F991F5A95E1F7E80FF91FE25426
:104D0000FE4F8681882329F0222309F498C04AE2C5
:104D100003C0222361F044E480912005882311F42C
:104D200020E001C02A2D89E76D2D0E942C5D8A2D7F
:104D3000813051F55E01AA0CBB1C33E0CC0FDD1FA6
:104D40003A95E1F7AC0EBD1EE4EAF1E0AE0EBF1EEF
:104D5000812FF501648D43E82DE70E949814F50139
:104D6000848FF701EE0FFF1FEE0FFF1FEE0DFF1DEB
:104D7000EB5BFA4F84818093A00880818F738093CE
:104D8000A10810929F08B92CF701EE0FFF1FEE0F3C
:104D9000FF1FEE0DFF1DEB5BFA4F8181882331F081
:104DA00088150CF4882E87150CF0782EF701EE0F7D
:104DB000FF1FEE0FFF1FEE0DFF1DEB5BFA4F828111
:104DC000882331F088150CF4882E87150CF0782E86
:104DD0009394F8E0DF0E292D273009F08CCECC20FB
:104DE000A1F08B2D8F3FF9F4C81464F480911F0556
:104DF00090E00197EFEF8F3F9E0711F480E090E085
:104E000080931F057C14ECF414C0FB2DFF3F59F474
:104E100080911F0590E001972FEF8F3F920761F47B
:104E200080E090E009C08B2D86305CF0992D9830A1
:104E300040F080911F058F5F80931F0502C043E5FE
:104E40006BCFDF91CF911F910F91FF90EF90DF908B
:104E5000CF90BF90AF909F908F907F906F9008956C
:104E60002F923F924F925F926F927F928F929F927A
:104E7000AF92BF92CF92DF92EF92FF920F931F9368
:104E80005C01CC24DD243B018824992464E6262E91
:104E9000312C412C512CC201B101661977098809C6
:104EA0009909A60195010E947B6E7B018C0182E32A
:104EB00090E0A0E0B0E0E80EF91E0A1F1B1FC6013B
:104EC000B5010E947B6E0E947B6EBC0188279927EA
:104ED000A40193010E947B6E44E096958795779597
:104EE00067954A95D1F7E60EF71E081F191FC801EE
:104EF000B701A20191010E94CD6EC9011F910F91CE
:104F0000FF90EF90DF90CF90BF90AF909F908F90E9
:104F10007F906F905F904F903F902F9008951F93D8
:104F2000CF93DF939C016115710511F1132F111FB0
:104F30001127111F19F0309521953F4F77FF0EC0B3
:104F4000C0E0D4E0709561957F4FCE01821B930B3A
:104F50000E9430279E01281B390B05C0C9010E9401
:104F60003027282F392F112319F0309521953F4FE5
:104F7000C901DF91CF911F9108956F927F928F9217
:104F80009F92AF92BF92CF92DF92EF92FF920F93D8
:104F90001F93DF93CF93CDB7DEB7982E962F322F86
:104FA000802F6E2D222359F0442361F440919C04FC
:104FB00050919D044115510539F421E001C020E0D4
:104FC000FF2405C022E001C021E0FF24F394332335
:104FD00011F0911121E04A2D433679F44C2D50E027
:104FE000440F551F8A0173E0000F111F7A95E1F7F6
:104FF000041B150B065A1C4F11C0FA2DF236D9F4BA
:105000004C2D50E0440F551F8A0193E0000F111FF3
:105010009A95E1F7041B150B055A1C4FF8014081C6
:105020000E94760FFF2009F463C0F8016081892D8A
:105030004AEE26E159C069887724BB24882051F5BF
:105040004C2D50E0440F551F6A01B3E0CC0CDD1C21
:10505000BA95E1F7C41AD50AAA0CBB1CAA0CBB1C52
:10506000CA0CDB1CC60CD71C4EE453E0C40ED51E84
:10507000F6014081552747FD50950E946260FF2050
:10508000B9F1F6016081892D4CE924E60E9498145B
:10509000F6012DC0DD24AA0CBB1CA601E3E0440FE1
:1050A000551FEA95E1F74C195D09A40EB51EA80C31
:1050B000B11CAA0CBB1CF301EA0DFB1DE25BFC4F0B
:1050C0004081552747FD50954C595F4F0E946260C3
:1050D000FF2071F08501060D171D025B1C4F892D05
:1050E000F80160814CE920E00E949814F801808367
:1050F000CF91DF911F910F91FF90EF90DF90CF90B4
:10510000BF90AF909F908F907F906F9008952F9257
:105110003F924F925F926F927F928F929F92AF9247
:10512000BF92CF92DF92EF92FF920F931F93DF9384
:10513000CF93CDB7DEB72A970FB6F894DEBF0FBE78
:10514000CDBFD82E89EC9DE00E94F6198DE998E03C
:105150006D2D40E020E030E000E071EDE72E7DE0D5
:10516000F72ECC2453E0A52E0E94F11B4091950808
:105170004F5F80E360E020E00E942A0FF0909D08DE
:105180008091950890E0880F991FFC0123E0EE0FB5
:10519000FF1F2A95E1F7E81BF90BE65AFC4F8081C7
:1051A00060E040E00E9454108823C1F0809195088F
:1051B00090E0880F991FFC0113E0EE0FFF1F1A9576
:1051C000E1F7E81BF90BE55AFC4F808160E040E015
:1051D0000E945410882321F411E003C010E001C0A4
:1051E00012E060919508462F50E0FA01EE0FFF1F84
:1051F000EF50FB4F808191818A3191051CF0109214
:105200009C0807C02FEF873E92071CF481E0809333
:105210009C082091880130E02170307082E090E09D
:10522000821B930B8417950741F4643030F480910E
:10523000B501807F11F010929C0880E164EC7DE064
:105240000E94465E0F92EDB7FEB7319621E0F11055
:1052500020E080919C0880838D2D61E041E006E391
:10526000A0E1EA2EC0909508A12E88240E94BD27B7
:105270000F9088E16DEB7DE00E94465E0F92EDB7E6
:10528000FEB7319621E03F2D313009F020E08091CA
:105290009C0880838D2D61E041E006E3F8E1EF2E6C
:1052A000C0909508A12E882483940E94BD270F905A
:1052B00080E267EB7DE00E94465E0F92EDB7FEB79D
:1052C000319621E08F2D823009F020E010828D2D63
:1052D00061E041E00EE1E0E2EE2EC090950873E659
:1052E000A72E88240E94BD270F9088E261EB7DE005
:1052F0000E94465E0F92EDB7FEB7319621E09F2DDA
:10530000933009F020E010828D2D61E041E00EE144
:1053100058E2E52EC090950832E6A32E88240E941C
:10532000BD270F90113019F0123049F404C080E30A
:105330006AEA7DE007C080E363EA7DE003C080E3C2
:105340006BE97DE00E94465E00919508402F50E099
:10535000812F90E0880F991F880F991FBA01660F5F
:10536000771F9B01B3E0220F331FBA95E1F7261B8D
:10537000370B820F931F8C559E4FFC01E655FE4F55
:10538000A081A983FC01E555FE4FB081BA83FC01E1
:10539000E455FE4F9080E4E69E0E83559E4FDC015F
:1053A0008C908E0E2091880130E02170307082E068
:1053B00090E0821B930B8417950709F062C00430BC
:1053C00008F05FC08091B501807F09F45AC0EE24D7
:1053D000FF24870120E030E0B9816B2E772467FC41
:1053E0007094A1E24A2E512C292C332427FC3094AE
:1053F000F0E4CF2ED22ED801C701B595A795979589
:105400008795B30129873A870E948F27880F991FB4
:10541000B2010E94BA6E629DC001639D900D729DA3
:10542000900D11246FE3A62EAD0C64E670E00E948F
:10543000A66EEC2DE61B6E2F8A2D0E94805E2985BC
:105440003A85C90183709070009761F48A2D6FE3EB
:105450000E94805E6D2D6695605E8FE30E94805E87
:105460003A8529852F5F3F4F81E290E0A0E0B0E0D0
:10547000E80EF91E0A1F1B1F2E33310509F0BACFA3
:105480007CC0DD249981492E552447FC509401E2CB
:1054900010E0A92DBB27A7FDB095BC83AB8354E6D4
:1054A000652E712C40E2A42EBA812B2E332427FCCA
:1054B0003094E82DFF27E7FDF095FE83ED83FD2D69
:1054C00021E2F29F70011124C701B2010E948F27CF
:1054D000B8010E94BA6EAB81BC816A9FC0016B9F0C
:1054E000900D7A9F900D11243EE5C32ECD0CB30193
:1054F0000E94A66EBA2DB61B6B2F8C2D0E94805E6B
:10550000ED2DF0E0E370F070F887EF83309749F409
:105510008C2D60E20E94805E6D2D605E8EE50E94A3
:10552000805EC701B1010E948F27B8010E94BA6E48
:105530002D813E81629FC001639F900D729F900DEF
:1055400011242EE5F22EFD18B3010E94A66E605EB6
:105550008F2D0E94805E8F819885009749F48F2D52
:1055600060E20E94805E6A2D6D198EE50E94805E69
:10557000D3949D2D9F3109F0A2CFE0919508F0E0E2
:10558000EE0FFF1FEF50FB4F408051805201CC24A3
:10559000B7FCC094DC2CC601B50121E230E040E04C
:1055A00050E00E94EF6E822F825A61E04EE30E942B
:1055B000D05E409195082091880130E021703070D4
:1055C00082E090E0821B930B242F30E08217930738
:1055D00009F050C0443008F04DC08091B501807F83
:1055E00009F448C0C601B50160507C4F8F4F9F4FF2
:1055F00022E030E040E050E00E94EF6EA9816A2F87
:10560000772767FD7095C9010E948F27BC01660F3F
:10561000771F882777FD8095982F292D97FC2D5F80
:1056200025952595332727FD3095432F532F0E942D
:105630007B6E29E130E040E050E00E94EF6E79019E
:105640008A01CA01B9012FED3FEF4FEF5FEF0E94D2
:10565000EF6E622F605C8FE34EE30E94CC5EC80168
:10566000B70122E030E040E050E00E94EF6E7901A7
:105670008A013CC01A141B041C041D0414F4698123
:1056800001C06A81772767FD7095C2010E948F274C
:105690009C01442737FD4095542F1A141B041C0409
:1056A0001D0414F4692D01C0682D67FD6D5F6595BB
:1056B0006595772767FD7095872F972F0E947B6EE2
:1056C00029E130E040E050E00E94EF6E79018A016C
:1056D000CA01B9012FED3FEF4FEF5FEF0E94EF6E70
:1056E000622F605E8FE34EE30E94CC5EC601B5017F
:1056F00029E130E040E050E00E947B6E612CB1E097
:105700007B2E812C912CA40193010E94EF6E82E7E5
:1057100060E3A90120E00E946260C801B70129E1AD
:1057200030E040E050E00E947B6EA40193010E94B3
:10573000EF6E84E568E0A90120E00E9462601A141F
:105740001B041C041D0474F4B9816B2F772767FDBB
:105750007095C20144970E948F27F701E81BF90B4F
:10576000CF010BC0FA816F2F772767FD7095C201BB
:1057700044960E948F278E199F099C01220F331F88
:10578000220F331F280F391F442737FD4095542F10
:1057900084E560E100E3F3E0EF2E0E942C5F2A969F
:1057A0000FB6F894DEBF0FBECDBFCF91DF911F9132
:1057B0000F91FF90EF90DF90CF90BF90AF909F90B0
:1057C0008F907F906F905F904F903F902F900895B3
:1057D0002F923F924F925F926F927F928F929F9201
:1057E000AF92BF92CF92DF92EF92FF920F931F93EF
:1057F000DF93CF93CDB7DEB72F970FB6F894DEBF08
:105800000FBECDBF982E81E99DE00E94F6198AE96E
:1058100098E0692D43E020ED37E00AE0F9E9EF2E4A
:10582000FDE0FF2ECC24C394E4E0AE2E0E94F11BD9
:10583000F0909A08FA9430909B08292D203841F472
:10584000F7FC06C0F092950887E898E20E94F514EC
:1058500085E168E041E85DE00E944E5E8AE593E004
:105860009C838B8376E9472E78E0572EE1EFF4E0B6
:10587000FB87EA8710E1662477242F2D332727FD45
:1058800030953A832983C901880F991FFC0153E0A1
:10589000EE0FFF1F5A95E1F7E81BF90BFE83ED832E
:1058A000F62CEB81FC81808160E040E00E94541086
:1058B000882361F0EB81FC81818160E040E00E94FF
:1058C0005410882329F4BB24B39404C0BB2402C021
:1058D00042E0B42E2B2D30E038872F83C901880F8A
:1058E000991F880F991FA301440F551F9A0103E0C8
:1058F000220F331F0A95E1F7241B350B820F931FEC
:105900008C559E4FDC01A355BE4FFC01E455FE4F64
:105910003C912081321751F4FC01E555FE4F86552C
:105920009E4F41E02081FC018081281340E0EA8500
:10593000FB8581919191FB87EA879C0197FF04C0C9
:1059400022273327281B390B2A3131050CF040E080
:10595000242E8A3191051CF0F201108207C0FFEF5E
:10596000873E9F071CF421E0F2012083809188018B
:1059700090E081709070E2E0F0E0E81BF90BE61532
:10598000F70551F48091B501807F31F0F301EA56BB
:10599000F74F1082222423944F2D4F5F80E0612F18
:1059A00020E00E942A0F5D864C86F2013081F1E0F2
:1059B000F9873111198680912005882351F4DD245F
:1059C000D39480919C0490919D04009721F4DD2450
:1059D00002C0DD24D39489819A818615970511F43C
:1059E00021E0311020E00F92EDB7FEB73183892D11
:1059F00060E04D2D07E2E12ECF2CAB2C88240E94D5
:105A0000BD270F9029813A812615370509F0D2C0AC
:105A1000332009F0CBC0DD2009F4CCC0222009F4EA
:105A2000C9C08F819885880F991F880F991FED81B4
:105A3000FE818E0F9F1F8C559E4FF9858F0F911DF4
:105A400086559E4F9F878E87892DEE85FF856081C5
:105A50004CE924E60E949814EE85FF858083AAC055
:105A600021E00F92F2018081EDB7FEB78183892D8D
:105A700060E04D2D09E3E12ECF2CAB2C88248394DC
:105A80000E94BD270F9029813A812615370509F01C
:105A900097C0332D313009F08FC0DD2009F490C05C
:105AA000222009F48DC08F819885880F991F880F57
:105AB000991FED81FE818E0F9F1F8C559E4FF9859A
:105AC0008F0F911D84559E4F98878F83892DEF816D
:105AD000F88560814CE920E00E949814EF81F885F8
:105AE00080836EC021E00F92EDB7FEB71182892D41
:105AF00060E04D2D0FE3E12ECF2CF3E6AF2E88248E
:105B00000E94BD270F9029813A812615370521F47F
:105B100021E0332D333009F020E00F92EDB7FEB7CE
:105B20001182892D60E04D2D07E5E12ECF2CE2E6B4
:105B3000AE2E88240E94BD270894411C511C0F9052
:105B4000EC85FD858081882319F4222031F008C07E
:105B5000222031F48AE34FE705C08BE34EE702C011
:105B60008AE34DE2612F0E94EB5DFB2DF13019F0CD
:105B7000F23049F404C085E7612F4DE407C085E7A2
:105B8000612F4CE403C085E7612F48E40E94EB5D80
:105B90000894611C711C2B813C81225F3F4F3C8328
:105BA0002B83185F103309F07BCE0CC0332D3130BE
:105BB00009F456CF20E055CF832D823009F492CFDF
:105BC00020E091CF2F960FB6F894DEBF0FBECDBF69
:105BD000CF91DF911F910F91FF90EF90DF90CF90C9
:105BE000BF90AF909F908F907F906F905F904F90FD
:105BF0003F902F90089520E030E0F901E25CF24FF1
:105C0000E491E81711F4822F08952F5F3F4FEE23A0
:105C1000A1F780E00895823430F4E82FF0E0E25CF0
:105C2000F24F8491089580E20895EF92FF920F93CE
:105C30001F93182FF62EE22E862FBA010E94465E81
:105C400086E66F2D412F2E2D0E94AC1BEE2039F0E1
:105C5000802F612F40E021E00E94A714182F812F90
:105C60001F910F91FF90EF900895FF920F931F9354
:105C7000F82E1091AF01212F332727FD309537FFE4
:105C800003C0309521953F4F022F25320CF43DC0C3
:105C90002091440830914508809142089091430832
:105CA000282B392B8091460890914708282B392BB7
:105CB0008091410890E0282B392B40913E0850E01C
:105CC000242B352B2115310531F4812F881F88278E
:105CD000881F80933E0811161CF4812F845202C045
:105CE000812F8C5D60E040E00E945410882359F0C1
:105CF00090913E08992339F491E0209141082111B7
:105D000090E09093410880933E08209144083091A0
:105D100045082F5F3F4F309345082093440820915A
:105D20004208309143082F0D311D309343082093D2
:105D300042080E94810E2091460830914708821B3C
:105D4000930B8436910508F471C12C593F4F309361
:105D50004708209346082091420830914308E0917B
:105D60004408F0914508C901BF010E94A66EF62EB5
:105D7000462F50E04E9FC0014F9F900D5E9F900DAB
:105D80001124281B390B30934308209342081092AA
:105D900045081092440800311CF4109241080FC0CD
:105DA00005326CF411161CF4812F8F5002C0812F24
:105DB000815F60E040E00E94541080934108809130
:105DC0003D0690913E06019690933E0680933D06D7
:105DD00040913F06509140064F5F5F4F5093400601
:105DE00040933F06FF2049F080914306909144067E
:105DF000019690934406809343068091410888233E
:105E000049F0809141069091420601969093420696
:105E100080934106F69420914506309146062F0D59
:105E2000311D30934606209345068091B101909133
:105E3000B20190934906809348066091AF0177279D
:105E400067FD709577FF03C0709561957F4F66235E
:105E500019F4109247061EC0613019F4841B950B8B
:105E600015C0603168F460FF06C0A4E03695279540
:105E7000AA95E1F709C0209143063091440604C079
:105E80002091410630914206821B930B9093490664
:105E90008093480680914706813051F0813018F098
:105EA000823049F514C08091AF01882321F120C0D0
:105EB000809148069091490618161906E4F08091E1
:105EC000B1019091B2010097B1F082E012C08091CF
:105ED0004806909149062FEF853C92071CF483E019
:105EE000809347068091B1019091B201009719F417
:105EF00081E0809347068091480690914906209161
:105F00003F08309140082817390709F479C02091DB
:105F10004706213009F065C020918A0122FF45C063
:105F20002091B1013091B20121153105F1F18E318D
:105F3000910519F489E10E94EA6D809148069091DB
:105F400049068431910519F48AE10E94EA6D809135
:105F50004806909149068A30910519F48BE10E9418
:105F6000EA6D8091480690914906843091051CF4B1
:105F70008CE10E94EA6D80918A0183FF16C08091B6
:105F80004806909149068E31910549F0843191057A
:105F900031F08A30910519F08430910534F482E3B0
:105FA00090E09093A00480939F0480918A0181FFE8
:105FB00027C08091B001209148063091490680FFAA
:105FC00007C08091B1019091B201821B930B01C077
:105FD000C9016CE370E00E94A66E009789F480E02E
:105FE00003C0223069F48CE10E94EA6D80918A013D
:105FF00083FF06C082E390E09093A00480939F0407
:1060000020914806309149063093400820933F087C
:106010008091B00180FF0AC08091B1019091B201DE
:10602000821B930B90934906809348061F910F9112
:10603000FF9008958091AF01992787FD909597FF74
:1060400003C0909581959F4F982F823034F1803115
:1060500024F585959A3024F40E944F6390E003C0A4
:10606000992787FD90950197FC01EE0FFF1FEF50D8
:10607000FB4F208131818091AF0187FF05C080E017
:1060800094E0821B930B03C0C90180509C4F26E013
:10609000969587952A95E1F702C080E090E00E94EE
:1060A000352E83E00E944F63E82FF0E0EE0FFF1FD4
:1060B000E151FB4F8081918180509C4FB6E09695D5
:1060C0008795BA95E1F72091B00122FF0AC085308B
:1060D000910538F02091A204222319F423E02093A3
:1060E000A20420913A0830913B082F5F3F4F309334
:1060F0003B0820933A082091380830913908280F3E
:10610000391F30933908209338080E94810E20915E
:106110003C0830913D08821B930B23E0883E920798
:10612000E8F10E94810E90933D0880933C08809195
:10613000B301823051F485E160E040E00E945410E8
:10614000882319F087E00E94EA6D809138089091C9
:10615000390860913A0870913B080E94A66E10922F
:1061600039081092380810923B0810923A08809132
:10617000C3069091C40601969093C4068093C3060B
:106180008091C206E82FF0E0E65BF94F60838F5FF5
:106190008093C206883710F01092C20608951092BC
:1061A00047061092400610923F0610924406109245
:1061B0004306109242061092410610924606109233
:1061C000450608950F931F93182F80913B0688234F
:1061D00019F06EE27DE002C061E27DE088E00E949D
:1061E000465E81E060E144EA51E02AE000E10E947D
:1061F000EF5D82E460E14FE30E94EB5D82E168E2E3
:106200004AE15DE00E944E5E82E160E34BE05DE0CA
:106210000E944E5E113609F44AC01F3B21F0103631
:1062200009F04FC004C080E00E94EA6D4AC080912E
:106230003B068823A9F089EF9CE00E948A12809196
:106240003C060E947857882339F087E10E94EA6D66
:1062500082E080933B0629C080E00E94EA6D25C061
:10626000809171018F5F0E943C5A1091710108C0AA
:106270001150113108F01FE080917101181739F0A9
:10628000812F8F5F0E94EF59882391F301C010E0A6
:106290001093710181E00E9410580E94AC588091C7
:1062A00071010E9441570E94CF3080E601C081E613
:1062B0000E942B6281E00E94C01484E691E30E9458
:1062C000F5141F910F910895AF92BF92DF92EF9254
:1062D000FF920F931F93CF93DF93182F85E19BE0DD
:1062E0000E94F619809120058823A1F4E0912305EE
:1062F000E7FF10C0E195EA3008F0E9E0F0E0EE0FCA
:10630000FF1FE053F84F25913491C9010E94E51415
:1063100010922305F0908F088FE898E0612F4FE0EE
:106320000E94EB2086E360E040E15BE00E944E5E6D
:106330000E943159AC0186E660E020E00E94626074
:1063400080E06AE041E00E94CC1BD0908F088091F1
:106350003B06823021F410928E0810923B061636CE
:1063600048F4143690F5103609F456C0113609F089
:1063700075C00AC0113809F456C01F3B09F465C046
:10638000103809F06BC053C080918E088823E9F063
:1063900010928E0887E10E94EA6D81E60E942B62CE
:1063A0000E94AC5880918F08809371010E944157E0
:1063B0000E94CF3081E00E9410580E94AC5882E0C9
:1063C0000E9410580E94AC5849C0809171018D15EF
:1063D000B9F0812F0E942B6280918F088093710108
:1063E0000E94AC58809171010E9441570E94CF30A9
:1063F00081E00E9410580E94AC5881E00E94EA6D32
:10640000153619F486ED90E504C0143639F58FE998
:1064100093E40E94E51422C081E080938E0887E116
:106420000E94EA6D1BC081E00E94C01417C08091D9
:106430008E08882399F081E080933B06D0923C0639
:1064400082EE90E30E94F51409C010928E088091AC
:10645000710180938F0881E00E941E5880918E0800
:10646000882341F0FD1431F06D2D6F5F8F2D8F5F0C
:106470000E94FD59CD2DDD27C7FDD09580911F05C8
:106480009E01281B3109C901181619065CF0CE01BE
:10649000019797FF02C080E090E080931F0510E114
:1064A000DD240BC025303105D4F3CE0104978B30A9
:1064B00091059CF38AE090E0F0CFF0901F05FD0C71
:1064C000AF2CBB2495012F5F3F4F442737FD4095EC
:1064D000542FCA15DB0511F401E101C000E182E18E
:1064E000612F72E0E72E0E942C5F80917101F816F7
:1064F00029F481E0612F4AE20E94EB5D8F2D6FE766
:1065000078E04FE00E94F956CA15DB0531F480911E
:106510008E08882311F001E101C000E188E1612FBC
:106520004FE758E02FE00E94EF5DD394185F3D2DB8
:10653000363019F6DF91CF911F910F91FF90EF90B8
:10654000DF90BF90AF900895AF92BF92CF92DF924D
:10655000EF92FF920F931F93CF93DF935B016C0138
:1065600010E1E12EF12CC0E0D0E800E010E89E013F
:1065700040E050E0CA01B9010E947B6EA616B70642
:10658000C806D90610F4C027D12716950795089498
:10659000E108F108E114F10461F4CE01DF91CF913B
:1065A0001F910F91FF90EF90DF90CF90BF90AF9031
:1065B0000895C02BD12BDBCFE1E0683068F4E0E038
:1065C00070E09B01220F331F220F331F260F371F4E
:1065D000A90146575C4F0EC070E0685070409B01A7
:1065E00053E0220F331F5A95E1F7260F371FA901F9
:1065F0004E545C4FDA012C9180509C4F97FD0FC098
:10660000B8E080309B078CF0EE2319F028E030E0F2
:1066100002C024E030E0240F351FF9012081332728
:1066200027FD3095322F222730C0EE2329F0692F25
:106630009070880F991F03C0692F66959170262F5F
:1066400030E0FA01E20FF31F6181772767FD709553
:10665000AC0155954795649F9001659F300D749FDF
:10666000300D11246081772767FD709540E052E07E
:10667000481B590B55954795649FC001659F900D28
:10668000749F900D1124280F391FC90169E170E032
:106690000E94BA6ECB0108952F923F924F925F9263
:1066A0006F927F929F92AF92BF92CF92DF92EF92C2
:1066B000FF920F931F93DF93CF9300D00F92CDB72C
:1066C000DEB7182F992493948091A608883008F497
:1066D000992480ED9FE00E94F619992011F05AE06C
:1066E00001C056E084EC98E0612F40E020E030E00B
:1066F00000E076EDE72E7FE0F72ECC24C394A52EA4
:106700000E94F11B4091A60850E04F5F5F4F84E26A
:1067100060E021E00E9462608091A608992079F0F3
:1067200090E008977C0103E0EE0CFF1C0A95E1F76E
:10673000E80EF91E22EB33E0E20EF31E0CC090E0EF
:106740007C01EE0CFF1CEE0CFF1CE80EF91E8AE823
:1067500093E0E80EF91E0091C4080150D090C508DE
:10676000113661F0123628F41434D1F0153471F575
:106770000EC01436A9F0153649F509C0DD2031F1F7
:106780001092C50881E60E942B62DD241FC0809113
:1067900020058823D9F01D14CCF48D2D815014C010
:1067A00080912005882391F02D2D332727FD3095EA
:1067B000992019F089E090E002C085E090E0281768
:1067C000390724F48D2D8F5F8093C5088091C5080B
:1067D00080932005CE2C4F2C6E2C7F2C90E1222410
:1067E0003324A02EBB24A7FCB094F30141913F01B8
:1067F000552747FD509521E0A214B30409F020E08D
:1068000088E1692F99830E9462600894211C311CE1
:106810009981985F983349F7992001F1A5E06A2E94
:10682000712C6E0C7F1C90E1F5E02F2E312CF301C2
:1068300041913F01552747FD509521E0A214B30433
:1068400009F020E080E3692F99830E946260089438
:10685000211C311C9981985F903349F70F3F11F447
:1068600021E0D11020E08CE068E049EC5FE00E947C
:106870001F5E992019F089E090E002C085E090E069
:1068800021E0A816B90609F020E08CE068E342ECAC
:106890005FE00E941F5E992019F089E090E002C03D
:1068A00085E090E0A816B90694F407FD4EC0A02E2E
:1068B000BB24A7FCB094AE0CBF1C812FF5016081F6
:1068C0004CE924E60E949814F50180833EC010161E
:1068D000E4F5812F6091C3084CEF24E000E00E94B2
:1068E0008A148093C30890919904992371F1992097
:1068F00021F050E194E049E003C058E092E045E027
:1069000024E6820230011124892F90E09095819530
:106910009F4F869D9001879D300D969D300D1124CF
:10692000EC2DF42DA52E00E0C9016A2D702F0E94D8
:10693000BA6E6193260D371D8E2F8C198417A0F324
:1069400082E00E9410580E94AC5880912005882354
:1069500051F0AA24ECE92E2EEFEF3E2E4D2C5524BB
:1069600047FC5094A5C000E01CEFAA24BB2470E2B1
:10697000D72EACC0C90165E0880F991F6A95E1F771
:10698000992019F064E070E002C062E070E00E94BB
:10699000BA6E462F062F055C37016A0C711CF30195
:1069A0008081992787FD909555E0880F991F5A950A
:1069B000E1F7B1010E94BA6E562F90E2D92ED60EA1
:1069C0002F5F3F4F8D2D90E09B838A8342165306A5
:1069D00009F050C082349105ACF48AE3C82EC40E8D
:1069E000625E8C2D45E059830E94CC5E5981EA811C
:1069F000FB81E134F10531F0652F615E8C2D45E0BE
:106A00000E94CC5EFD2DF03430F4802F81506D2D2E
:106A100045E00E94CC5E2A813B812F33310594F4FE
:106A200001506D2D6F5F802F45E00E94CC5E8A8102
:106A30009B818E33910531F06D2D6E5F802F45E087
:106A40000E94CC5E80919C0490919D04009741F43B
:106A5000123631F0133621F0123411F0133439F5B7
:106A6000812FF30160814CE924E60E949814F30120
:106A700080831DC02A813B81213431052CF4615E65
:106A8000802F43E00E94CC5E3D2D303428F4802FCF
:106A90006D2D43E00E94CC5E8A819B818F339105EE
:106AA00034F46D2D6F5F802F43E00E94CC5EA39481
:106AB0002A2D30E0992019F089E090E002C085E0AD
:106AC00090E0281739070CF455CF4DCFC8016091DD
:106AD000A6080E94DC32BCE3EB2EEA0C9C01A5E088
:106AE00036952795AA95E1F76D2D621B8E2D0E9494
:106AF000805E9501237030702115310521F48E2DB3
:106B000060E20E94805E0894A11CB11C005E1F4FD1
:106B100090E4A916B104D1F68CE560E040E40E944F
:106B2000D05E0F900F900F90CF91DF911F910F913A
:106B3000FF90EF90DF90CF90BF90AF909F907F90AD
:106B40006F905F904F903F902F9008952F923F92BB
:106B50004F925F926F927F928F929F92AF92BF926D
:106B6000CF92DF92EF92FF920F931F93DF93CF9319
:106B7000CDB7DEB7A2970FB6F894DEBF0FBECDBF7C
:106B80008F8F98A36A8B80919E04882309F474C028
:106B900080912105882319F08150809321058091EF
:106BA000CB069091CC062091C9063091CA06820F7F
:106BB000931F2091CD063091CE06820F931F209116
:106BC000CF063091D006820F931F20915407309149
:106BD00055072C01421A530A920157FE03C0309503
:106BE00021953F4F41E0213034073CF09093550709
:106BF0008093540781E08093A10480918901863FAE
:106C0000D9F1909108019233B8F1909151079F5FAB
:106C100090935107903160F02091520730915307C3
:106C20002F5F3F4F30935307209352071092510725
:106C30009091A104992321F01092530710925207CA
:106C40002091520730915307992787FD90950A9616
:106C500067E771E0869FA001879F500D969F500DBA
:106C600011244217530740F423703070213031054E
:106C700019F480E10E94EA6D80918801582F5170CB
:106C80005F5F598781FF02C01D8602C063E06D8788
:106C90006090BC01662009F44AC08985E82FF0E0C5
:106CA000EE0FFF1FEF50FB4FA080B180CC24B7FC4C
:106CB000C094DC2C9D85E92FF0E0EE0FFF1FEF5014
:106CC000FB4F20813181442737FD4095542FCA0165
:106CD000B9010E947B6E7B018C01C601B501A60142
:106CE00095010E947B6EE60EF71E081F191F662D88
:106CF00070E080E090E0EAE0660F771F881F991F40
:106D0000EA95D1F724E630E040E050E00E94EF6ED3
:106D1000B901CA010E947B6E6E157F05800791073D
:106D200030F4C801B7010E94A4324C0102C088248B
:106D30009924B40180E090E024E630E040E050E0A7
:106D40000E947B6E6B8F7C8F8D8F9E8F64E4662E8E
:106D500061E0762EA9ECB6E0BE8BAD8BFE013196DC
:106D6000F88FEF8B50E0252E51E0352E24EA31E0EC
:106D70003F872E8741EF54E05A8F498F2901F98BC5
:106D8000E88BBC8BAB8BEE24FF241B865A89517099
:106D900059A3AE2C8E2D0E9487159C01D30111960C
:106DA0008D919C911297281B390BB901882777FD8B
:106DB0008095982F4AE0660F771F881F991F4A9584
:106DC000D1F7121613062CF45D962D913C915E9727
:106DD00003C0F301278530892436310514F424E6F5
:106DE00030E0442737FD4095542F0E94EF6E890113
:106DF000FCEF21303F072CF024E00030120724F490
:106E000005C000E01CEF02C000E014E080918A01A0
:106E100080FF0FC08091880190E08170907042E007
:106E200050E0481B590BE416F50619F4109501952E
:106E30001F4FA98DBA8D0D931D93BA8FA98FC801CD
:106E40000F968F319105F0F4B4E0EB16F1047CF469
:106E50008A2D8F5F0E944F6390E00197E1E0F0E0A0
:106E600002C0EE0FFF1F8A95E2F7CF0108C081E054
:106E700090E00E2C02C0880F991F0A94E2F7FB8560
:106E8000F82BFB872A2D243008F07AC139A133234F
:106E900009F05FC08091B00181FF5BC06701CC0C3D
:106EA000DD1C4EE751E0C40ED51ED60111968C9123
:106EB0001197807C09F44DC08C91859585958595B9
:106EC00061E040E00E945410882309F442C0D601DA
:106ED000EC91E770F0E0DF01AA0FBB1FAA55BB4F92
:106EE000EE0FFF1FEA58FE4F8D919C911197208164
:106EF0003181821B930B62E070E00E94BA6EF70151
:106F0000EE0FFF1FE158FE4F2081422F440F440F28
:106F100045954595552747FD5095649FC001659F50
:106F2000900D749F900D11246FE170E00E94BA6E75
:106F3000660F771F660F771F22952695269523707B
:106F4000213019F0223029F403C0060F171F01C0A9
:106F50008B018114910409F1B985AB1619F0ED8507
:106F6000AE16D9F46091BC0170E080E090E04AE098
:106F7000660F771F881F991F4A95D1F798014427FC
:106F800037FD4095542F0E947B6E2B8D3C8D4D8D8F
:106F90005E8D0E94EF6E022F132FF201EA54FE4F16
:106FA000808160E040E00E945410882369F0F20183
:106FB000E954FE4F808160E040E00E945410882335
:106FC00029F4CC24C39404C0CC2402C032E0C32EE4
:106FD0008091880190E08170907022E0A22EB12C07
:106FE000A81AB90AAE14BF0469F58091B501807F73
:106FF00049F1C80180509C4F62E070E00E94BA6E77
:107000009B01EC2DF0E0EE0FFF1FEE0FFF1FA7011D
:10701000440F551FCA01A3E0880F991FAA95E1F7F5
:10702000841B950BE80FF91FE25BFC4F608177270B
:1070300067FD7095C9010E948F27AC01440F551F51
:1070400030E028C031E0101611060CF430E08C2D31
:1070500090E0A701440F551FFA0163E0EE0FFF1FF8
:107060006A95E1F7E41BF50B880F991F880F991FAC
:10707000E80FF91FEC55FE4FE30FF11DE655FE4FEB
:107080006081772767FD7095C8013AA30E948F271A
:10709000AC013AA1EC2DF0E0EE0FFF1FEE0FFF1F49
:1070A000B701660F771FCB0113E0880F991F1A9560
:1070B000E1F7861B970BE80FF91FEC55FE4FE30F26
:1070C000F11DE455FE4F6081772767FD70956C597F
:1070D0007F4F882777FD8095982FDA019D014427FF
:1070E00037FD4095542F0E947B6E24E630E040E04F
:1070F00050E00E94EF6E022F132FAE14BF0499F5DB
:107100008091B501982F907F09F466C60050144015
:1071100063C6D101ED91FC911197608180918A0144
:1071200080FD6195772767FD7095872F972F6358AE
:107130007F4F8F4F9F4F20E034E0201B310B4427BF
:1071400037FD4095542F0E947B6E20E038E040E0F0
:1071500050E00E94EF6E2030B8E03B07B0E04B07F4
:10716000B0E05B0739F4D101ED91FC912081332728
:1071700027FD3095220F331FE889F9893183208359
:10718000AB89BC890D931D93BC8BAB8B0894E11C20
:10719000F11CE2E0F0E06E0E7F1E288939892E5F37
:1071A0003F4F398B288B2E0E3F1E4EE050E0440E91
:1071B000551E57E0E516F10409F0EBCD0091B90139
:1071C0006B850623809156078095802319F088E10E
:1071D0000E94EA6D0093560780E094E09093D806F1
:1071E0008093D7069093DA068093D906E6EAF4E016
:1071F00026E731E0A1EEB6E0BD0181919191D90180
:107200004D915D919D01841B950B880F991FDB01AA
:107210008D939D93BD01B4E0EE3AFB0771F7809129
:10722000AE049091AF04880F991F9093EA06809363
:10723000E9068091B0049091B104880F991F909352
:10724000EC068093EB068091B2049091B304880F12
:10725000991F9093EE068093ED068091B40490916F
:10726000B504880F991F9093F0068093EF06E1E133
:10727000F7E0FC87EB8721EF36E041915191619176
:107280007191D9014D935D939D01B7E0E135FB0705
:10729000A1F7C090BC01CC2009F47AC0E985AE2EDC
:1072A000BB24AA0CBB1C29EC422E26E0522EA40CB7
:1072B000B51CD5012D903C90442437FC4094542CAF
:1072C000BD850B2F10E0000F111F0753194FF80158
:1072D00020813181442737FD4095542FCA01B901DF
:1072E0000E947B6E3B014C01C201B101A2019101E0
:1072F0000E947B6E660E771E881E991EDD24EE248A
:10730000FF248AE0CC0CDD1CEE1CFF1C8A95D1F713
:10731000C701B60124E630E040E050E00E94EF6E85
:10732000B901CA010E947B6E66157705880599052B
:1073300078F5C401B3010E94A432BC0180E090E062
:1073400024E630E040E050E00E947B6E3B014C01BF
:10735000C201B101A70196010E947B6EA4019301B5
:107360000E94EF6ED5012D933C93F80160817181ED
:10737000882777FD8095982FA70196010E947B6E44
:10738000A40193010E94EF6ED80111963C932E93B5
:10739000E090BA018E2D807E09F4DEC0B9852B2FD6
:1073A00030E0220F331FF901E753F94F408151813B
:1073B000CE010196280F391FD901ED91FC91BD85B1
:1073C0006B2F70E0660F771FDB01A753B94F2D912C
:1073D0003C91860F971FDC018D919C91BA89B1FD7C
:1073E00005C0E40FF51F280F391F04C020E030E06E
:1073F000E0E0F0E0A091BB01AA2349F0B0E0AA0FC1
:10740000BB1FA953B94F0D911C91119702C000E009
:1074100010E0E2FE03C0F095E195FF4FE3FE03C0EC
:10742000309521953F4FE4FE03C0109501951F4F05
:107430008091BA01829586958770823071F1833090
:1074400020F4813009F088C007C0833009F459C0A6
:10745000843009F081C06CC0C90168E070E00E940E
:10746000BA6E7B01C90160E870E00E94BA6E290122
:107470004E185F087201E61AF70AC90160E072E06F
:107480000E94BA6EE61AF70AC8018E1B9F0B9093F2
:10749000DC068093DB06CF0120C0CF0168E070E0FE
:1074A0000E94BA6E7B01CF0160E870E00E94BA6E64
:1074B0003F016E187F087301E61AF70ACF0160E0FA
:1074C00072E00E94BA6EE61AF70AC801821B930B9B
:1074D0009093DC068093DB06C90162E070E00E94B5
:1074E000BA6E600F711FCB018E0D9F1D9093DE064B
:1074F0008093DD066E197F097093E0066093DF06C6
:107500002BC0C8018E1B9F0B9093DC068093DB067B
:10751000E00FF11FCF01820F931F9093DE0680933F
:10752000DD06E21BF30BF093E006E093DF0614C0E8
:10753000C8018E1B9F0B9093DC068093DB06C8016D
:10754000820F931F9093DE068093DD06021B130BC0
:107550001093E0060093DF0680919E04882311F0CB
:107560000E941A3080E4E1E1F7E0DF011D928A9584
:10757000E9F7BA89B1FF2DC08091880190E0817050
:10758000907022E030E0281B390B80E090E0ED891C
:10759000FE89AF89B88D2817390729F0118210822A
:1075A00011961C921E920196329612968430910585
:1075B00091F71092E2061092E1061092E406109202
:1075C000E3061092E6061092E5061092E806109285
:1075D000E70686E893E090930101809300019C0107
:1075E0002F5F3F4F30930301209302019C012E5FD8
:1075F0003F4F3093050120930401039690930701B8
:107600008093060127E1422E28E0522E97E9692E49
:1076100097E0792E87E5282E87E0382E19861D867B
:1076200089850E94890E7C01FC0180818150803116
:1076300008F0ADC2838161E040E00E945410D201A5
:107640009C918823A1F4292F1C92F7019181892F05
:107650008850823008F08AC287818E70843009F4A5
:1076600085C2993009F04BC000E01CEF4AC021E010
:10767000911120E081E0D2018C93D7011196EC9119
:107680003E2F3150832F90E0DC01AA0FBB1FA75380
:10769000B94F0D911C911197343160F0B9853B17AA
:1076A00048F4DC01AA0FBB1FAA0FBB1FAF5EB84F87
:1076B0000D911C91D70117963C911797832F8073DA
:1076C00081F0832F8295837090E0019741E050E034
:1076D00002C0440F551F8A95E2F7CA015D85582BF9
:1076E0005D8736FF0EC0E53060F4F0E0EE0FFF1F5F
:1076F000E250FF4FC70108969183808302C000E0EB
:1077000010E0D7011796CC901797C6FC0BC01896BF
:107710008C911897882331F02AA30E946C0E080FD1
:10772000191F2AA1F7018681882321F485818823E6
:1077300009F458C1D3016D917D918D919C9113975E
:10774000222389F420E031E040E050E00E94EF6E17
:1077500050954095309521953F4F4F4F5F4F4801D1
:10776000820E931E5AC08C2D8E70843051F5D70135
:10777000EC91F0E0EE0FFF1FE151F94F6081718154
:10778000882777FD8095982F20E034E640E050E090
:107790000E947B6EF3016083718382839383D701A0
:1077A00012962C911297222361F0332727FD3095F2
:1077B000432F532F0E94EF6EF301208331834283C6
:1077C0005383D3016D917D918D919C91139720E00E
:1077D00031E040E050E00E94EF6E509540953095CA
:1077E00021953F4F4F4F5F4F4801820E931E8114EA
:1077F000910499F0F701258197FE22952F7030E0D2
:1078000044E650E0249FC001259F900D349F900DC9
:107810001124D10111969C938E93F1018081918165
:10782000009799F020919E04222319F001979183EB
:107830008083D1018D919C911197009731F0F301D4
:107840006081718182819381B7C08114910409F4B0
:10785000C9C0D70116968C911697882309F4B4C035
:1078600080919E04882309F476C012962C91129779
:107870002223B1F0332727FD309537FF03C0309521
:1078800021953F4F332727FD3095432F532F60E03D
:1078900070E080E293E00E94EF6E59016A0106C039
:1078A000A12CB12CF0E2CF2EF3E0DF2EF701868180
:1078B00018141904FCF48F7090E00097F1F144E67D
:1078C00050E0849F9001859F300D949F300D1124CE
:1078D000442737FD4095542FC601B5010E94EF6E35
:1078E000F30180819181A281B381280F391F4A1F42
:1078F0005B1F2CC082958F7090E00097F1F044E6FA
:1079000050E0849F9001859F300D949F300D11248D
:10791000442737FD4095542FC601B5010E94EF6EF4
:1079200059016A01D3012D913D914D915C911397BD
:107930002A193B094C095D0909C09801442737FD04
:107940004095542F542F432F322F2227F3012083A9
:10795000318342835383D3016D917D918D919C91AD
:1079600020E031E040E050E00E94EF6EC801AA271D
:1079700097FDA095BA2F1814190434F482179307B1
:10798000A407B50734F012C0281739074A075B0768
:107990006CF4222717FD2095322F322F212F102F24
:1079A0000027F3010083118322833383D3016D9178
:1079B0007D918D919C91139720E031E040E050E063
:1079C0000E94EF6E89010EC0C801AA2797FDA095FD
:1079D000BA2FBA2FA92F982F8827F301808391837C
:1079E000A283B383D70114966C911497633061F12D
:1079F000643028F4613051F06230A0F444C0653046
:107A000069F1653038F1663081F52BC0F70181816D
:107A1000893029F417FD35C0005012400EC017FF01
:107A200032C02CC0D70111968C911197893041F446
:107A30001016110604F100501E4F000F111F23C035
:107A400010161106DCF01FC017FF1DC01095019520
:107A50001F4F19C01016110674F010C017FF0EC08A
:107A600010C0101611063CF00CC06750C8010E94EF
:107A7000DC328C0108C000E014E005C000E010E03A
:107A800002C000E01CEFF701878180FD13C0E18197
:107A9000EE2381F0E53070F4F0E03197EE0FFF1F38
:107AA00021E030E02C0F3D1FE20FF31F8081918118
:107AB000080F191FB801882777FD8095982FD701E7
:107AC00012962C911297332727FD3095432F532F71
:107AD0000E947B6EF701008110E001501040278169
:107AE00026952770213071F0F801EE0FFF1FEE0F81
:107AF000FF1F223069F5EF5EF84F60837183828348
:107B0000938334C024E630E040E050E00E94EF6E02
:107B1000E22EC32EDA01000F111F000F111F0F5E9E
:107B2000184FF80120813181428153816E2D7C2DC7
:107B3000CD010E947B6E20E034E040E050E00E94E6
:107B4000EF6ED8012D933D934D935C9313970EC028
:107B5000EF5EF84F2081318142815381260F371F1C
:107B6000481F591F2083318342835383B985BF5FE8
:107B7000B9870894411C511CE4E0F0E06E0E7F1EB2
:107B800022E030E0220E331EB03209F049CD0E94CF
:107B9000810E8C01ED84E0FE05C0882319F48EE18E
:107BA0000E94EA6DE1FE0BC0C8019070803491051F
:107BB00019F08834910519F48FE10E94EA6DE2FE14
:107BC0000DC010700038110531F00838110519F09A
:107BD0000039110519F480E20E94EA6DBFEF4B2EC7
:107BE000B4E05B2E3F8D28A1832F922F9A8789873F
:107BF00022243324598A488AAB85BC85ED90FD90B8
:107C00000D911C91C801B70124E630E040E050E03E
:107C10000E94EF6EEB85FC85208331834283538382
:107C2000A889B9892D933D93B98BA88BEE85FF85E3
:107C3000E35AFE4F80819181EE85FF85E55AFE4F24
:107C40002081BAE02B0260011124E8EEF3E0CE0EB1
:107C5000DF1EEE85FF85E65AFE4F20812B02500184
:107C60001124A8E14A2EACEF5A2EA40CB51C9601A3
:107C70004C2D232F8C159D0514F4482F292F842E6D
:107C8000922E8A149B040CF44501E114F1040105C1
:107C9000110569F19401442737FD4095542F1E14B6
:107CA0001F041006110654F4B601882777FD80954D
:107CB000982F621B730B840B950B0DC0C501AA276F
:107CC00097FDA095BA2F29013A01481A590A6A0A64
:107CD0007B0AC301B201A80197010E947B6E20EAD2
:107CE00036E841E050E00E94EF6E79018A01C4015C
:107CF0000E94D7193C01882477FC8094982C6E0C44
:107D00007F1C801E911EC6010E94D7198C01C501DF
:107D10000E94D719222717FD2095322F0615170527
:107D20002805390514F438014901AA2797FDA095C3
:107D3000BA2F84017301681679068A069B0614F42B
:107D40007C018D01EE85FF85E45AFE4F80818823FA
:107D500041F010950095F094E094E11CF11C011D98
:107D6000111DF4EACF2EF1E0DF2EC20CD31CF60178
:107D7000E358FD4F8081882389F060E040E00E9455
:107D80005410882359F0F601E258FD4F80810E947B
:107D90006C0E7C010027F7FC0095102FF894A98544
:107DA000BA85ED92FD92BA87A9877894EB85FC8518
:107DB0003496FC87EB87E2E04E2E512C240C351CC8
:107DC0002E853F852B5F3F4F3F872E8730E223165E
:107DD000310409F011CF04C08F7009F09AC9C3C9EA
:107DE000A2960FB6F894DEBF0FBECDBFCF91DF9144
:107DF0001F910F91FF90EF90DF90CF90BF90AF90C9
:107E00009F908F907F906F905F904F903F902F90BA
:107E10000895EF92FF920F931F93DF93CF93CDB707
:107E2000DEB7C054D0400FB6F894DEBF0FBECDBF52
:107E30008E010F5F1F4FC80163E00E94A63581E2EB
:107E4000E82EF12CEC0EFD1EC70161E00E94A63564
:107E5000E0E0F3E0418152816081D8012D913C91B5
:107E6000D7018D919C911197662329F0B901681B68
:107E7000790BCB0102C0821B930B840F951F73E01B
:107E8000883E97072CF4ACEF89319A0724F005C09F
:107E900088EE93E002C088E19CEF9283818335965F
:107EA0000E5F1F4F62E070E0E60EF71E73E0E035F4
:107EB000F70781F68091880190E08170907022E050
:107EC00030E0281B390B80E090E02817390721F0BB
:107ED000FC01EA57FC4F1082019684309105A9F706
:107EE00086E00E94105881E00E94EA6DC05CDF4F7E
:107EF0000FB6F894DEBF0FBECDBFCF91DF911F91BB
:107F00000F91FF90EF9008952F923F924F925F92C2
:107F10006F927F928F929F92AF92BF92CF92DF9299
:107F2000EF92FF920F931F93DF93CF930F92CDB7F2
:107F3000DEB7109186011F70813809F477C082384E
:107F400088F48332F1F1843230F48032E1F082320D
:107F500009F07EC045C0813609F45DC0803809F063
:107F600077C01BC08438F9F0853838F4823809F4BA
:107F70004AC0833809F06CC040C08538E1F08F3BBF
:107F800009F066C059C0153009F062C08091A204A2
:107F900091E089278093A2044DC00E94B6140E94EC
:107FA000F51480E805C084E691E30E94F51484E8A6
:107FB0000E942B624DC082E19BE40E94F51485E88B
:107FC000F7CF812F8F5F80938601863010F010925B
:107FD000860181E00E94105883E10E94EA6D38C05A
:107FE000112319F0812F815001C085E08093860113
:107FF00081E00E94105884E1F0CF8DEF99E10E945A
:10800000E51483E8D5CF0E944C6E88E99AE10E947E
:10801000E51482E8CDCF80914706823021F483E0D9
:108020008093470607C0153099F402C00E94CF30F4
:108030000E94341587E1D1CF81E00E942B6283E05A
:108040000E942B6282E00E942B6281E080933708BD
:108050008091B80160E040E00E945410882331F024
:1080600080913708882311F40E94093F8091B8015C
:1080700060E040E00E9454108093370880918601B0
:10808000803108F0D3C09091080180917301981756
:1080900010F496E001C094E0B4EAEB2EB1E0FB2EC0
:1080A0000AE0D7014D917D01802F60E024E09983A3
:1080B0000E942C5D055F9981083799F7492F406828
:1080C00084E260E10E94240F84E268E146E50E94B8
:1080D000EB5D80914706882399F0823011F406E029
:1080E00001C004E040914806509149068EE560E1E8
:1080F000202F0E94A50E83E368E140E00E94C90F93
:108100004091B60183E04802A00111244C50584F21
:1081100084E260E123E000E00E94EF5D8091B50120
:108120008F7031F089E360E140EF57E00E944E5ECE
:10813000AEE0EA2EA1E0FA2EF0E0CF2EF1E0DF2E45
:1081400066247724EFE19E2EF70101917F01D6018D
:10815000ED91FD916D01808187FD8D5F8595859500
:10816000843E0CF484EEA82E8D3114F07CE1A72E11
:10817000862D81508230F8F4802F64E046E30E941F
:10818000D05E2091880130E02625372520FD04C0EF
:108190008091B5018F7061F4802F81506EE143E0D2
:1081A0000E94D05E802F8F5F6EE143E00E94D05E20
:1081B000992D9A1914C0802F8B516BE346E30E94CE
:1081C000CC5E802E8A94882D6AE343E00E94CC5EC8
:1081D000882D6CE343E00E94CC5E0A0D9BE36DEFBB
:1081E000862E800E5DEFA52EA90E882D6A2D47E004
:1081F00099830E94D05E9981692F6D5F882D47E039
:108200000E94CC5E802F8D5F6A2D47E00E94D05E79
:10821000882D6A2D47E00E94CC5E0894611C711C79
:10822000B4E06B16710409F08FCF27C080E060E0E6
:1082300044EA51E02AE001E10E94EF5D90910801DB
:1082400080917301981710F442E001C040E084E58A
:1082500060E00E94240F80914706882371F08230ED
:1082600011F402E001C000E0409148065091490637
:108270008FE660E0202F0E94A50E123008F085C026
:1082800045E2E42E45E0F42E00E039E1A32EB12CC6
:108290002BE1922E90E2692E712C80E8482E512C11
:1082A000F701219031907F01113011F1802F8370FF
:1082B000899DC02C1124D02ED694D694DD0CDD0CD3
:1082C000DD0CF8E2DF0EC101B3010E94BA6E9B0122
:1082D000C101B2010E94BA6EAB01421B530B420DA9
:1082E000531D8C2D8F5D6D2D20E20E94626048C071
:1082F000043018F4B2E2CB2E02C0AEE5CA2E802FB5
:108300008370D82EDD0CDD0CD80E26E2D20EC10112
:1083100037FE04C088279927821993098A9DA001F6
:108320008B9D500D9A9D500D112440505E4F452F4E
:10833000550F550B45954595842E4A3114F0E9E1CA
:108340008E2E8C2D89516D2D43E325E50E949E5E76
:108350006D2D62508C2D45E00E94D05E12141304E6
:1083600014F4C39401C0C8186D2D6F5F8C2D482D77
:108370000E94CC5E6D2D61508C2D482D0E94CC5EEC
:108380000F5F083009F08CCF8AC0153008F07DC02F
:108390000E94F720123061F0812F880F810F880F23
:1083A0008950912F9150192F110F190F110F02C0E1
:1083B00080E016E0C82E992787FD90952C01440C8B
:1083C000551C480E591E60E2D62EEE24FF2452E0C2
:1083D000852E912C880E991E3C011AC00E94C60F52
:1083E0005C018C2D60E040E00E945410082FA50134
:1083F000440D551D8AE06D2D23E00E94EF5D089429
:10840000E11CF11C83E090E0480E591E98E0D90E63
:10841000C394C701860D971D88169906FCF6812F17
:10842000992787FD90952C01440C551C480E591E28
:1084300030E2D32EEE24FF2422E0822E912C880EEF
:10844000991E3C011AC00E94C60F5C01812F60E09A
:1084500040E00E945410082FA501440D551D85E6EB
:108460006D2D23E00E94EF5D0894E11CF11CA3E058
:10847000B0E04A0E5B1EB8E0DB0E1F5FC701860D41
:10848000971D88169906FCF60AC04091A4045091E5
:10849000A5048CE368E224E004E00E94A50E0F909E
:1084A000CF91DF911F910F91FF90EF90DF90CF90D0
:1084B000BF90AF909F908F907F906F905F904F9004
:1084C0003F902F90089518161CF010921F050895E4
:1084D000282F332727FD309590911F05291B31093F
:1084E000462F50E04217530724F4861B80931F0544
:1084F0000895465050402417350724F48A5F861BA0
:1085000080931F050895AF92CF92DF92EF92FF9272
:108510000F931F93DF93CF930F92CDB7DEB7182F32
:1085200088E89BE00E94F61981E998E0612F42E01B
:1085300020ED37E00AE073E9E72E7BE0F72ECC244C
:1085400056E0A52E0E94F11BF09091088F2D67E058
:108550000E94634288E06DE77BE00E94465E31E066
:108560008F2D813009F030E08091BA018295869597
:10857000877090E0AC01440F551F480F591F440FFE
:10858000551F425A544F84E568E026E0032F398393
:108590000E94EF5D3981332399F06091BA016295B1
:1085A00066956770812F40E024E00E9498148295C0
:1085B000880F807E9091BA019F71982B9093BA0199
:1085C00080E163E57BE00E94465E01E0EF2DE23052
:1085D00009F000E084E560E14091BB01202F0E949A
:1085E0002A0F002349F0812F6091BB0140E024E273
:1085F0000E9498148093BB0188E168E47BE00E94AC
:10860000465E4091BC01FF2DF33011F421E401C01E
:1086100020E484E568E150E00E9462608F2D8330A1
:1086200049F4812F6091BC0140E024E60E94981437
:108630008093BC010091BA0106950695017080E215
:108640006AE37BE00E94465ECF2CDD24C7FCD09419
:1086500021E0E4E0CE16D10409F020E084E560E2F8
:10866000402F0E94BC1BFF2DF43079F4812F602F26
:1086700040E021E00E9498148170880F880F90914B
:10868000BA019B7F982B9093BA010091BA0106958D
:1086900006950695017088E26CE27BE00E94465EDA
:1086A00021E085E0C816D10409F020E084E568E205
:1086B000402F0E94BC1BEF2DE53081F4812F602FED
:1086C00040E021E00E9498148170880F880F880F85
:1086D0009091BA01977F982B9093BA010091BA01BB
:1086E0000295017080E36EE17BE00E94465E21E02E
:1086F000F6E0CF16D10409F020E084E560E3402FD6
:108700000E94BC1B8F2D863079F4812F602F40E0B2
:1087100021E00E94981481708295807F9091BA0127
:108720009F7E982B9093BA010F90CF91DF911F916C
:108730000F91FF90EF90DF90CF90AF900895AF92A0
:10874000BF92CF92DF92EF92FF920F931F93DF932E
:10875000CF930F92CDB7DEB7D82E87EE9CE00E9464
:10876000F61983E998E06D2D41E020ED37E00AE04D
:10877000ADEEEA2EACE0FA2EFBE0CF2EE0E1AE2E1D
:108780000E94F11B10919308F0909408812F67E0EC
:108790000E9463422091710130E02F5F3F4F4427D8
:1087A00037FD4095542F8AE260E001E172E0E72E48
:1087B0000E942C5F2D2D253451F0263418F42434DA
:1087C00001F511C03D2D343671F03536D1F411303C
:1087D000C1F4FF20B1F080912005882391F08091B1
:1087E000940881500CC0113061F44F2D493048F489
:1087F00080912005882329F0809194088F5F8093D1
:10880000940880911F05882309F088C088E062EEF3
:108810007CE00E94465E113031F481E090E02091CE
:108820002005222311F080E090E0082F00618CE306
:1088300068E044EA51E02AE00E94EF5D8091200563
:10884000882359F48091230587FF07C081E0809336
:10885000200510922305109294088091200588230A
:1088600081F020912305332727FD30958F2D90E04F
:108870008217930734F4109220051092230510926A
:108880009408113009F04DC080912005882309F427
:1088900048C08091940890912305891B8093940887
:1088A00087FF02C010929408809194088A301CF0CF
:1088B00089E08093940810922305AF2CBB24F50126
:1088C000EC55FE4F80810E94FB2D682F20919C0467
:1088D00030919D042115310549F47D2D723631F01A
:1088E000733621F0723411F0733431F48D2D40E081
:1088F00021E40E949814682F862F0E940B2E482F87
:10890000F501EC55FE4F80838F2D880F8F0D880F5A
:10891000845C68E021E00E942C5D03C098E0E92EB1
:1089200002C080E1E82E80911F05823008F084C0EB
:108930008E2D6CED7CE00E94465E4091B10150911D
:10894000B201123099F4FF2039F480912005882378
:1089500009F01AC421E019C48F2D813039F48091B7
:108960002005882329F020E002E004C020E00DC4A7
:1089700020E001E087E46E2D0E94A50E123009F080
:1089800059C080912005882339F480919C049091EE
:108990009D04009709F44EC0FF2029F09F2D9130CF
:1089A00009F048C022C08091B1019091B2010CE35E
:1089B000A02EB12CB5010E94A66E8D2D40E02BE3B8
:1089C0000E9498142CE3482F4203900111248091B7
:1089D000B1019091B201B5010E94A66E280F391F16
:1089E0003093B2012093B10125C08091B1019091E3
:1089F000B2016CE370E00E94A66E082F0E5F8D2D11
:108A0000602F41E02EE30E949814081B602F772707
:108A100067FD70952091B1013091B201261B370B93
:108A20003093B2012093B10137FF04C01092B2011C
:108A30001092B10168E0E60E80911F058330F8F4D2
:108A40008E2D64ED7CE00E94465E01E0133009F05B
:108A500000E08CE36E2D402F0E94C90F002349F0E7
:108A60008D2D6091AF0147EC29E30E94981480930B
:108A7000AF0178E0E70E8E2D893308F088C380912E
:108A80001F058430C8F58E2D6DEC7CE00E94465E9B
:108A900091E0143009F090E08091B001282F21700E
:108AA00030E0A901440F551FA3E0220F331FAA9500
:108AB000E1F7420F531F4854534F8CE36E2D2AE0C9
:108AC000092F99830E94EF5D9981992379F0609134
:108AD000B00161708D2D40E021E00E9498148170FA
:108AE0009091B0019E7F982B9093B00198E0E90E91
:108AF000EE2DE93308F04BC380911F05853030F52A
:108B00000091B5010F708E2D61EB7CE00E94465EF6
:108B100021E0153009F020E08CE36E2D402F0E94FB
:108B2000AC1B153069F48D2D602F40E021E00E94D0
:108B300098148F709091B501907F982B9093B50108
:108B4000F8E0EF0E2E2D293308F021C380911F0588
:108B5000863040F50091B50102950F708E2D6AEABE
:108B60007CE00E94465E21E0163009F020E08CE3B4
:108B70006E2D402F0E94AC1B163071F48D2D602F8E
:108B800040E021E00E9498148295807F9091B50189
:108B90009F70982B9093B50138E0E30E4E2D49332A
:108BA00008F0F5C280911F05873050F58E2D61EADF
:108BB0007CE00E94465E91E0173009F090E0409121
:108BC000B60186E04802A00111244E57534F8CE3B2
:108BD0006E2D26E0092F99830E94EF5D99819923DC
:108BE00049F08D2D6091B60140E024E00E94981478
:108BF0008093B60168E0E60E7E2D793308F0C7C297
:108C000080911F05883008F58E2D6AE77CE00E9470
:108C1000465E01E0183009F000E086E36E2D4091D9
:108C2000B801202F0E94760F002349F08D2D60910E
:108C3000B8014AEE26E10E9498148093B80188E0BA
:108C4000E80E9E2D993308F0A2C280911F0589304D
:108C500008F051C08E2D61E77CE00E94465E9CE3E7
:108C6000AA24BB24A5014759534FFA1411F4193013
:108C700061F02091B90130E00A2C02C035952795AA
:108C80000A94E2F7022F017001C002E0892F6E2DD5
:108C900021E099830E94EF5D0894A11CB11C998189
:108CA0009A5F9636F9F6193001F5ED2DE03631F080
:108CB00080919C0490919D040097B9F08D2D0E94A5
:108CC0002B621092200581E090E00F2C02C0880FEB
:108CD000991F0A94E2F72091B90128272093B9013E
:108CE00082E00E9410580E94AC58F8E0EF0E2E2D42
:108CF000293308F04CC280911F058A3008F0E3C088
:108D00008E2D63E67CE00E94465E4091B30186E0D2
:108D1000489FA0011124465B534F1A3041F4FF20B5
:108D200031F480912005882321F002E003C000E0A7
:108D300001C001E084E26E2D26E00E94EF5D80918B
:108D4000B301882321F0833009F04DC009C086E6C5
:108D50006E2D45E45CE020E00E941F5E9CE308C0AD
:108D600082E76E2D42E45CE020E00E941F5E98E402
:108D70004091B401552747FD5095440F551F440FAE
:108D8000551F435D534F1A3049F43F2D313031F4B4
:108D900080912005882321F002E003C000E001C09B
:108DA00001E0892F6E2D24E099830E94EF5D998167
:108DB000892F865D4091B70192E34902A0011124F9
:108DC000445D5E4F1A3049F46F2D623031F490915A
:108DD0002005992321F022E003C020E001C021E01A
:108DE0006E2D0E9462608091B301813001F582E4B2
:108DF0006E2D4EE15CE020E00E941F5E4091B401C8
:108E0000552747FD50954F5F5F4F1A3049F47F2D2E
:108E1000713031F480912005882321F022E003C0D5
:108E200020E001C021E08EE76E2D0E9462601A30C2
:108E300009F043C080912005882331F480919C047F
:108E400090919D040097C9F18F2D813079F0813088
:108E500018F0823091F522C08D2D6091B30140E071
:108E600023E00E9498148093B30127C08091B3013E
:108E7000882311F0833031F48D2D6091B4014EEFD1
:108E800024E007C08130C9F48D2D6091B40140E029
:108E90002CE70E9498148093B4010FC08091B30115
:108EA000882311F0833049F48D2D6091B7014CEF88
:108EB0002AE00E9498148093B70198E0E90EEE2D05
:108EC000E93308F064C180911F058B3008F07AC047
:108ED0008091B301882311F0833019F58E2D6FE056
:108EE0007CE00E94465E4091BD0185E04802A00101
:108EF00011244F515F4F1B3011F421E201C020E2D9
:108F00008EE46E2D0E9462601B3009F055C08D2DDD
:108F10006091BD014CEE24E10E9498148093BD0144
:108F20004BC08130B9F401E01B3009F000E080E073
:108F30006E2D49EF5BE0202F0E941F5E0023E1F1C0
:108F4000FD2DF038C9F581E080936D0E80E00E9420
:108F5000EA6D32C08E2D60EF7BE00E94465E80910C
:108F6000B40187FD03C083301CF403C080E001C05E
:108F700082E08093B40149E08402A00111244C52A4
:108F8000544F1B3031F480912005882321F002E0FA
:108F900003C000E001C001E08CE36E2D29E00E94D7
:108FA000EF5D1B3049F48D2D6091B40140E022E06B
:108FB0000E9498148093B40128E0E20E3E2D3933CC
:108FC00008F0E5C080911F058C3098F58E2D6AEC75
:108FD0007BE00E94465E31E01C3009F030E0809179
:108FE000BA01817090E0AC01440F551F480F591F22
:108FF0004D53544F8CE36E2D23E0032F39830E9491
:10900000EF5D3981332379F06091BA0161708D2D64
:1090100040E021E00E94981481709091BA019E7FF7
:10902000982B9093BA0148E0E40E6E2D693308F056
:10903000AEC080911F058D3040F50091BA010695B4
:1090400001708E2D69EB7BE00E94465E21E01D30B1
:1090500009F020E08CE36E2D402F0E94AC1B1D30E8
:1090600071F48D2D602F40E021E00E9498148170F2
:10907000880F9091BA019D7F982B9093BA0178E068
:10908000E70E8E2D893308F082C080911F058E3047
:1090900040F50091B001069501708E2D61EB7BE0EB
:1090A0000E94465E21E01E3009F020E08CE36E2D28
:1090B000402F0E94AC1B1E3071F48D2D602F40E0BC
:1090C00021E00E9498148170880F9091B0019D7FDB
:1090D000982B9093B00198E0E90EEE2DE93308F05B
:1090E00056C080911F058F3048F50091B00106955C
:1090F000069501708E2D68EA7BE00E94465E21E0B5
:109100001F3009F020E08CE36E2D402F0E94AC1B35
:109110001F3079F48D2D602F40E021E00E949814DB
:109120008170880F880F9091B0019B7F982B90934E
:10913000B001F8E0EF0E2E2D293348F580911F0580
:10914000803128F580912105882319F421E0103120
:1091500009F020E080E06E2D44E95BE00E941F5E94
:109160001031A9F43D2D303891F41092200589E199
:109170008093210580E80E942B6210923B0682EECC
:1091800090E30E94F51403C022E000E0F3CB0F90BF
:10919000CF91DF911F910F91FF90EF90DF90CF90D3
:1091A000BF90AF9008956F927F928F929F92AF92EF
:1091B000BF92CF92DF92EF92FF920F931F93DF93B4
:1091C000CF930F92CDB7DEB7B82E82E39FE00E9417
:1091D000F61989EA98E06B2D47E020ED37E00AE0C8
:1091E00072E4E72E7FE0F72ECC24C3945CE0A52E3A
:1091F0000E94F11B8090A9088A94D090AA08882D1B
:1092000066E00E94634218E0CC24992487FC909485
:1092100090911F059C0D9C3009F44FC1E92EFF244D
:109220008E149F0439F480912005882329F022E0D0
:10923000A22E04C0AA2402C0AA24A39480E0612F15
:109240004FE25FE022E000E099830E94EF5D9981A8
:10925000993010F048E301C041E3490F8CE0612FE1
:109260000E94EB5DF701EE0FFF1FEE0DFF1DE450B6
:10927000FC4F408187E0489FA00111244453514F87
:10928000DD2011F000E001C00A2D88E1612F27E008
:109290000E94EF5DC701880F991F8E0D9F1D8C5591
:1092A0009E4FFC01E85AFD4F2081253008F4F6C09E
:1092B000FC01EA5AFD4F283008F4F9C040819D2D89
:1092C0009130D1F53BC020E001C02A2D88E4612F08
:1092D0000E942A0FF701EE0FFF1FEE0DFF1DE55054
:1092E000FC4F4081552747FD5095ED2DE23011F0A0
:1092F00020E001C02A2D88E7612F0E94626000E013
:1093000035C020E001C02A2D88E4612F0E94760F2D
:10931000F701EE0FFF1FEE0DFF1DE550FC4F4081E2
:10932000FD2DF23011F020E001C02A2D80E6612FE2
:109330000E94760F01E01AC020E001C02A2D88E4C7
:10934000612F0E942A0FF701EE0FFF1FEE0DFF1D88
:10935000E550FC4F40818D2D823011F020E001C09E
:109360002A2D86E6612F0E942A0F02E080912005B7
:10937000882339F480919C0490919D04009709F40E
:1093800086C0AA2009F483C09D2D9130D1F191307F
:1093900020F0923009F07BC046C03701660C771C84
:1093A0006E0C7F1CECEFF3E06E0E7F1E8B2DF30135
:1093B000608140E02DE00E949814F3018083202F0B
:1093C00030E0853028F0883030F481E090E005C04E
:1093D00080E090E002C082E090E02817390709F4AD
:1093E00056C0C701880F991F8E0D9F1D8C559E4F2B
:1093F000FC01EA5AFD4F1082895A9D4FFC011082F0
:1094000046C0013041F0C701880F991FE80EF91ED0
:109410008AEF93E031C03701660C771C6E0C7F1C1D
:109420008AEF93E01AC0013089F0C701880F991FB5
:109430000230F1F0E80EF91E8BEF93E0E80EF91E12
:109440008B2DF701608143E82DE71DC03701660CC5
:10945000771C6E0C7F1C8BEF93E0680E791E8B2DB2
:10946000F30160814AEE26E10E949814F3010EC0D8
:10947000E80EF91E8BEF93E0E80EF91E8B2DF70135
:10948000608140E024E20E949814F7018083C39435
:10949000185FFC2DF73009F0BBCE0FC08A5A9D4FE4
:1094A000FC014081FD2DF13009F00DCF0ECF408140
:1094B0008D2D813009F025CF26CF0F90CF91DF91F0
:1094C0001F910F91FF90EF90DF90CF90BF90AF90E2
:1094D0009F908F907F906F9008956F927F928F9260
:1094E0009F92AF92BF92CF92DF92EF92FF920F9333
:1094F0001F93CF93DF93982E84E49FE00E94F61988
:109500008BEA98E0692D48E020ED37E00AE014E5A9
:10951000E12E1FE0F12ECC24C394B0E1AB2E0E94CB
:10952000F11B6090AB086A948090AC08862D66E0D1
:109530000E946342A8E0FA2EDD24772467FC709431
:1095400040911F054D0D403109F45DC0A42EBB2490
:109550004F5F80E06F2D20E00E94560FEE24E50162
:10956000CC0FDD1FCE5DDB4F8501000F111F0F5D9E
:109570001B4F6A147B0471F48E1461F480912005F2
:10958000882359F480919C0490919D04009739F4AC
:1095900021E001C020E0CC2405C022E001C021E090
:1095A000CC24C394EE2091F48EE16F2DF80140811C
:1095B0000E94760FCC20D9F0892DF80160814AEE07
:1095C00026E10E949814F801808311C04881552734
:1095D00047FD509580E66F2D0E946260CC2039F0E7
:1095E000892D688143E82DE70E9498148883E394CD
:1095F000FE2DF33009F0BDCFD39488E0F80EED2DA9
:10960000E73009F09DCFDF91CF911F910F91FF902F
:10961000EF90DF90CF90BF90AF909F908F907F9012
:109620006F900895AF92BF92CF92DF92EF92FF9228
:109630000F931F93DF93CF9300D0CDB7DEB7182FD2
:1096400080919301813019F048E1C42E02C03AE1C3
:10965000C32E2BEFB22EBC0C83E29AE00E94F619C7
:1096600088E498E0612F40E024EE37E006E0EC2C3F
:109670000E947A1FF0904808D09049088F2D67E02B
:109680000E94634260911F058C2D90E0462F50E0B0
:109690009C01275030404217530761F42F2D30E0D2
:1096A00004972817390714F48FEF01C081E0680F81
:1096B00060931F05113629F1123678F4143409F439
:1096C00048C0153420F4123408F46AC063C015345D
:1096D00019F1103609F064C009C0143608F45AC0F4
:1096E0001436B9F1153609F05BC016C0FF2009F435
:1096F00057C081E090912005911180E08093200572
:109700004FC080912005882309F44AC0109220059B
:1097100081E60E942B6244C02F2D213059F4DD20B8
:1097200049F080912005882329F0809149088150D3
:10973000809349082F2D30E08B2D992787FD909538
:109740002817390769F5DD2059F1809149088150C2
:109750001EC03F2D313061F48D2D893048F4809149
:109760002005882329F0809149088F5F809349085C
:109770002F2D30E08B2D992787FD909528173907DD
:1097800079F49D2D973060F4809149088F5F809324
:10979000490806C080912005882311F410924908D9
:1097A00080911F05882309F089C088E068E17AE08C
:1097B0000E94465EEF2DE13031F481E090E020918F
:1097C0002005222311F080E090E0082F006182E460
:1097D00068E045E951E02AE00E94EF5D80912005B4
:1097E000882359F48091230587FF07C081E0809387
:1097F00020051092230510924908809120058823A6
:1098000081F020912305332727FD30958D2D90E0A1
:109810008217930734F410922005109223051092BA
:109820004908FF2DF13009F04CC0809120058823B4
:1098300009F447C08091490890912305891B8093C2
:10984000490887FF02C010924908809149088A3070
:109850001CF089E08093490810922305AD2CBB24AD
:10986000F501EB56FE4F80810E94FB2D682F209161
:109870009C0430919D042115310541F4123631F0DC
:10988000133621F0123411F0133431F4812F40E0FB
:1098900021E40E94A714682F862F0E940B2E482FC8
:1098A000F501EB56FE4F80838D2D880F8D0D880FAF
:1098B0008E5B68E021E00E942C5D03C098E0E92EF9
:1098C00002C080E1E82E80911F058230A0F5C09093
:1098D0008701C694C694C69427E0C2228E2D61E10A
:1098E0007AE00E94465E91E03F2D323009F090E030
:1098F00046E08C2D849FA00111244A51564F8CE5DF
:109900006E2D26E0092F9A830E94EF5D9A8199239C
:1099100081F0812F6C2D40E026E00E94A714877013
:10992000880F880F880F90918701977C982B9093D0
:10993000870198E0E90E80911F05833058F5C090AB
:1099400093018E2D6BED79E00E94465E91E0EF2D44
:10995000E33009F090E046E0FC2DF49FA0011124D3
:109960004253564F8CE56E2D26E0092F9A830E94B4
:10997000EF5D9A81992341F0812F6C2D40E021E029
:109980000E94A7148093930128E0E20E3E2D393304
:1099900008F0FFC380919301813041F580911F054C
:1099A000843030F58E2D60EC79E00E94465E409167
:1099B00091018F2D843011F421E401C020E486E66A
:1099C0006E2D50E00E9462609F2D943049F4812FEB
:1099D0006091910141E024E60E94A71480939101D7
:1099E000E8E0EE0EFE2DF93318F0D3C304E001C019
:1099F00005E0809193018150823038F580911F05F8
:109A0000801710F58E2D60EB79E00E94465E409144
:109A10009201F01611F421E401C020E486E66E2DD7
:109A200050E00E946260F01649F4812F609192012B
:109A300040E025E00E94A7148093920128E0E20E06
:109A40003E2D393308F0A5C30F5F80911F058017A5
:109A500020F58E2D67EA79E00E94465E4091720102
:109A6000F01611F421E401C020E486E66E2D50E0EA
:109A70000E946260F01659F4812F609172014AE0F1
:109A80002DE20E94A714809372010E94C26088E0B8
:109A9000E80E9E2D993308F07CC3C02EC3948091AC
:109AA0001F058C1508F58E2D67E979E00E94465E4A
:109AB00040917301FC1411F421E401C020E486E616
:109AC0006E2D0E94100FFC1449F4812F60917301D8
:109AD00048E228E70E94A71480937301E8E0EE0EA5
:109AE000FE2DF93308F055C3C39480911F058C15E2
:109AF00060F58E2D66E879E00E94465E409189010E
:109B0000552747FD5095465F5F4FFC1411F421E443
:109B100001C020E486E66E2D0E9462608091A90D4E
:109B20006E2D4DE60E94EB5DFC1449F4812F60918F
:109B3000890146EF2EE60E94A7148093890128E050
:109B4000E20E3E2D393308F024C3C39480911F05E3
:109B50008C1550F58E2D6BE779E00E94465E91E002
:109B6000FC1090E040918B0150E0440F551F440FD2
:109B7000551F4259564F86E66E2D24E0092F9A83D1
:109B80000E94EF5D9A81992349F0812F60918B01AA
:109B900040E022E00E94A71480938B0188E0E80E49
:109BA0009E2D993308F0F5C2C39480911F058C1542
:109BB000C8F480918A01817021E0FC1020E06E2DB4
:109BC0004DE559E0012F0E94152E817090918A0178
:109BD0009E7F982B90938A01E8E0EE0EFE2DF933DC
:109BE00008F0D7C2C39480911F058C15D8F48091DA
:109BF0008A018695817021E0FC1020E06E2D41E500
:109C000059E0012F0E94152E8170880F90918A01D2
:109C10009D7F982B90938A0128E0E20E3E2D3933E8
:109C200008F0B7C2C39480911F058C15E8F48091A9
:109C30008A0186958695817021E0FC1020E06E2DCA
:109C400042E459E0012F0E94152E8170880F880F81
:109C500090918A019B7F982B90938A0188E0E80E6F
:109C60009E2D993308F095C2C39480911F058C15E1
:109C7000F8F480918A01869586958695817021E019
:109C8000FC1020E06E2D44E359E0012F0E94152EB8
:109C90008170880F880F880F90918A01977F982B89
:109CA00090938A01E8E0EE0EFE2DF93308F071C2C0
:109CB000C39480911F058C1500F58E2D67E279E025
:109CC0000E94465E01E0FC1000E080E66E2D4091AF
:109CD0007501202F0E94760F002349F0812F60919B
:109CE00075014AEE26E10E94A7148093750128E0D1
:109CF000E20E3E2D393308F04CC2C394BB24809150
:109D00001F058C1508F048C0BB2019F467E179E005
:109D100002C067E079E08E2D0E94465EBB2019F4F8
:109D2000A0908C0102C0A0909401AA20A9F08A2DD5
:109D300095E0899FA0011124FC1411F421E401C0D5
:109D400020E486E66E2D0E9462608091A90D6E2D42
:109D500043E70E94EB5D0AC001E0FC1000E086E6EC
:109D60006E2D43E059E023E00E94EF5DFC1439F4CE
:109D7000812F6A2D40E028E70E94A714A82EBB205F
:109D800019F4A0928C0102C0A0929401E8E0EE0EBA
:109D9000FE2DF93308F0FDC1C394B3942B2D22306E
:109DA00009F0ADCF80911F058C15F8F480918A01E0
:109DB00082958F708095817021E0FC1020E06E2DDF
:109DC00045EF58E0012F0E94152E809581708295F5
:109DD000807F90918A019F7E982B90938A0138E032
:109DE000E30E8E2D893308F0D4C1C39480911F05F2
:109DF0008C15F8F48091900182958F708095817018
:109E000021E0FC1020E06E2D49EE58E0012F0E9469
:109E1000152E809581708295807F909190019F7E14
:109E2000982B9093900198E0E90EEE2DE93308F01D
:109E3000B0C1C39480911F058C15D8F4809187011F
:109E40008095817021E0FC1020E06E2D48ED58E0F7
:109E5000012F0E94152E80958170909187019E7F21
:109E6000982B90938701F8E0EF0E2E2D293308F000
:109E700090C1C39480911F058C15E8F480918701EF
:109E800086958095817021E0FC1020E06E2D49ECD4
:109E900058E0012F0E94152E80958170880F9091B7
:109EA00087019D7F982B9093870138E0E30E8E2DDC
:109EB000893308F06EC1C39480911F058C1508F09A
:109EC00086C08E2D6EEB78E00E94465E92E4AA2456
:109ED000BB24A5014B54574FE0919F01F0E00A2CA1
:109EE00002C0F595E7950A94E2F7E170F070892FCA
:109EF0006E2D21E00E2F9A830E94EF5D0894A11C25
:109F0000B11C9A819A5F923721F7FC1409F059C06D
:109F10008091490890912305891B8093490887FF08
:109F200002C010924908809149088A301CF089E0EB
:109F300080934908109223058D2D880F8D0D880F71
:109F40004D2D50E04455574F8E5B6E2D21E002E0C1
:109F50000E94EF5D103631F080919C0490919D0439
:109F6000009779F1812F0E942B621092200581E0E9
:109F700090E002C0880F991FDA94E2F790919F0158
:109F8000982790939F01803151F0803271F0883092
:109F900099F493FF02C09F7C0DC098600BC094FFA2
:109FA00002C0977D07C0906105C095FF02C0977EF3
:109FB00001C0906290939F0181E00E9410580E941E
:109FC000AC5898E0E90EEE2DE93308F0E2C0C394F6
:109FD00080911F058C15F8F48091870186958695F0
:109FE0008095817021E0FC1020E06E2D4DE958E055
:109FF000012F0E94152E80958170880F880F9091F7
:10A0000087019B7F982B90938701F8E0EF0E2E2D10
:10A01000293308F0BEC0C39480911F058C1500F54C
:10A0200090918701991F9927991F81E0891B21E051
:10A03000FC1020E06E2D4FE858E0012F0E94152EF5
:10A040008095879588278795909187019F77982B92
:10A050009093870138E0E30E8E2D893308F099C084
:10A06000C39480911F058C1508F580918A01829513
:10A07000869587708095817021E0FC1020E06E2D20
:10A0800045E858E0012F0E94152E80958170829539
:10A09000880F807E90918A019F7D982B90938A01F2
:10A0A00098E0E90EEE2DE93308F073C0C394809177
:10A0B0001F058C1518F580918A01829586958695E5
:10A0C00083708095817021E0FC1020E06E2D4DE7BB
:10A0D00058E0012F0E94152E809581708295880F7F
:10A0E000880F807C90918A019F7B982B90938A01A6
:10A0F000F8E0EF0E2E2D293308F04BC0C394809169
:10A100001F058C1508F045C086E06E2D48E758E025
:10A110000E944E5E3E2D383390F434E290E0832F5F
:10A120006E2D45E857E0292F00E039839A830E947D
:10A13000CD5C9A819F5F3981385E943081F788E0E9
:10A14000E80E9E2D993328F5DD24D394FC10DD24F0
:10A15000409188014F5C82E16E2D2D2D0E942C5D77
:10A1600094E200E00F5F892F6E2D402F20E09A834C
:10A170000E942A0F9A81985E0430A1F7DD2049F0F1
:10A18000812F6091880140E023E00E94A714809312
:10A1900088010F900F90CF91DF911F910F91FF9049
:10A1A000EF90DF90CF90BF90AF9008958F929F92E5
:10A1B000AF92BF92CF92DF92EF92FF920F931F93D5
:10A1C000DF93CF930F92CDB7DEB7C82E8DE79FE018
:10A1D0000E94F6198DEA98E06C2D49E020ED37E0F9
:10A1E0000AE0FAE0EF2E0E947A1F1091AD0811509C
:10A1F000812F66E00E9463422C2D203899F480E87C
:10A200000E942B6289E180932105193019F40E9484
:10A21000EA6205C0183018F4812F0E945C6381E067
:10A220000E94EA6DDD24E8E0FE2EA12EBB24A7FCEF
:10A23000B09480911F058D0D883081F1882E99246E
:10A2400094012F5F3F4F442737FD4095542FA814AA
:10A25000B90411F401E101C000E182E16F2D72E067
:10A26000E72E0E942C5FF401EE0FFF1FEF5FF54E0B
:10A2700085919491AC0180912105882321F421E0FE
:10A28000A814B90409F020E088E16F2D0E941F5E38
:10A2900038E0F30ED3948D2D873059F6EF2DE93346
:10A2A00008F04FC080912105882321F4DD24D39448
:10A2B000183009F0DD2486E06F2D4FE65FE00E9444
:10A2C0004E5E9AE556E0A52EB12CE0918D01F0E0AE
:10A2D000E852FB4F449150E00A2C02C05595479537
:10A2E0000A94E2F7437050704659504F892F6F2DF2
:10A2F00021E00D2D99830E94EF5D2EEF3FEFA20E1E
:10A30000B31E99819A5F923701F7DD2049F08C2DB9
:10A3100060918D0140E027E10E94A71480938D0198
:10A320006F2D685F693368F480912105882319F4E3
:10A3300021E0193009F020E086E046E55FE00E9468
:10A340001F5E0F90CF91DF911F910F91FF90EF90C3
:10A35000DF90CF90BF90AF909F908F9008954F92D5
:10A360005F926F927F928F929F92BF92CF92DF9275
:10A37000EF92FF920F931F93DF93CF9300D0CDB74F
:10A38000DEB7182F8BEB9FE00E94F61981EC98E066
:10A39000612F46E020ED37E00AE050E1E52E0E9413
:10A3A0007A1F6090C1086A94862D66E00E9463421D
:10A3B000103611F0143641F467FC06C06092A6080E
:10A3C0008CE493E30E94F514CC24DD24EE24E39482
:10A3D00018E0F12E772467FC709430911F053C0D36
:10A3E000BB24B394383028F4BB248E2D883028F059
:10A3F00074C09E2D973008F070C0032F10E091E0DC
:10A400006016710609F090E0DD2019F0DD24D39488
:10A4100001C0D92E80E06F2D48EB5FE0292F3A83F1
:10A4200099830E941F5E3A819981393010F482E14C
:10A4300001C087E1A8014F5F5F4F6F2D292F0E9458
:10A440006260BB2079F0085010402801B3E0440C52
:10A45000551CBA95E1F7400E511EE2EBF3E04E0EAB
:10A460005F1E0BC02801440C551C440C551C400EAB
:10A47000511E8AE893E0480E591E42010AE2F40197
:10A4800041914F01552747FD5095802F6F2D20E0BA
:10A490000E9462600B5E033991F7F8E0FF0EE394CF
:10A4A000BB20B1F085E090E0480E591E0AE2F201AF
:10A4B00041912F01552747FD5095802F6F2D20E0AA
:10A4C0000E9462600B5E0E3791F7F8E0FF0EE39496
:10A4D000C3948C2D873009F080CFDD2029F4809142
:10A4E0001F058F5F80931F050F900F90CF91DF9115
:10A4F0001F910F91FF90EF90DF90CF90BF909F90B2
:10A500008F907F906F905F904F900895AF92BF9221
:10A51000CF92DF92EF92FF920F931F93CF93DF932F
:10A52000F82E87EA98E06F2D4DE00E94EB20809195
:10A530009F08882319F080EC9EE002C086EB9EE025
:10A540000E94F619182F8091A0080E94890EEC0134
:10A55000812F8A5F60E0488120E00E94560FA09022
:10A56000A7088A2D66E00E94634218E0EE24BB240F
:10A57000A7FCB09420911F052E0D822F90E0DD24C2
:10A58000D394A816B90609F0DD24263009F4FAC0E0
:10A59000273090F4223009F457C0233030F42223BE
:10A5A00009F1213009F0E8C134C0243009F499C020
:10A5B000253008F0BAC069C02A3009F46BC12B30CD
:10A5C00038F4283009F420C1293008F044C1F1C022
:10A5D0002C3009F49CC12C3008F47AC12D3009F0DC
:10A5E000CBC1B2C18CE0612F4FEA5EE00E944E5EAB
:10A5F00084E5612F49812D2D0E942A0FDD2009F469
:10A60000BBC18F2D698141E024E20E9498148983A7
:10A61000B3C18CE0612F48EA5EE00E944E5E4A8141
:10A62000552747FD50952D2D206484E5612F0E940C
:10A630006260DD2009F4A0C18F2D6A8143E82DE717
:10A640000E9498148A8398C18F8186FF03C04EE9C7
:10A650005EE002C047E95EE08CE0612F0E944E5E42
:10A660004885552747FD50952D2D206484E5612FA1
:10A670000E946260DD2009F47FC18F2D688543E868
:10A680002DE70E949814888777C1CF80C294C69422
:10A69000C694E3E0CE2281E0C8228CE0612F4CE832
:10A6A0005EE00E944E5E43E09C2D949FA001112429
:10A6B0004B57514F84E5612F23E00D2D0E94EF5D34
:10A6C000DD2009F459C18F2D6C2D40E021E00E945E
:10A6D000981481708295880F880F807C9F819F7B62
:10A6E00090C08CE0612F40E85EE00E944E5E8F815A
:10A6F000817090E0AC01440F551F480F591F475817
:10A70000514F84E5612F23E00D2D0E94EF5DDD2088
:10A7100009F432C16F8161708F2D40E021E00E9409
:10A72000981481709F819E7F6CC08CE0612F42E7FE
:10A730005EE020E00E941F5E4C8183E0489FA00104
:10A7400011244A51504F84E5612F23E00D2D0E94C2
:10A75000EF5DDD2009F410C18F2D6C8140E026E112
:10A760000E9498148C83873008F406C19F2D903680
:10A7700009F002C187508093A6088CE493E30E94FD
:10A78000F514FAC08CE0612F4BE65EE00E944E5E4D
:10A790008EE4612F4B812D2D0E94760FDD2009F470
:10A7A000EBC08F2D6B814AEE26E10E9498148B83BB
:10A7B000E3C08CE0612F43E65EE00E944E5E0F81B5
:10A7C0000295037049F02D2D206484E5612F402F00
:10A7D00050E00E94626007C084E5612F4FE55EE0B3
:10A7E0002D2D0E941F5EDD2009F4C6C08F2D602F25
:10A7F00040E023E00E94981483708295807F9F81BF
:10A800009F7C982B9F83B8C08CE0612F48E55EE069
:10A810000E944E5E4F814695477050E063E0440FC2
:10A82000551F6A95E1F7415C514F84E5612F28E09F
:10A830000D2D0E94EF5DDD2009F49EC06F816695AD
:10A8400067708F2D40E022E00E9498148770880F77
:10A850009F81917FD6CF8CE0612F44E35EE00E9420
:10A860004E5E4D8142954F7080E6612F50E02D2D58
:10A870000E946260DD2009F47FC06D8162956F7077
:10A880008F2D40E02FE00E9498148295807F9D815B
:10A890009F701BC08CE0612F4BE25EE00E944E5E19
:10A8A0004D814F7080E6612F50E02D2D0E94626037
:10A8B000DD2009F461C06D816F708F2D40E02FE0C5
:10A8C0000E9498148F709D81907F982B9D8354C017
:10A8D0008CE0612F40E25EE00E944E5E4E81429528
:10A8E0004F7080E6612F50E02D2D0E946260DD20C8
:10A8F00009F442C06E8162956F708F2D40E02FE0A9
:10A900000E9498148295807F9E819F701AC08CE06F
:10A91000612F47E15EE00E944E5E4E814F7080E6FF
:10A92000612F50E02D2D0E946260DD2029F16E81A3
:10A930006F708F2D40E02FE00E9498148F709E81E1
:10A94000907F982B9E8318C08CE0612F45E05EE0DD
:10A950002D2D0E941F5EDD2079F08F2D803861F44F
:10A960000E942B628091A0080E94082381E00E942F
:10A97000EA6D80E00E94C014E394185F9E2D97302A
:10A9800009F0F8CDDF91CF911F910F91FF90EF90DB
:10A99000DF90CF90BF90AF9008955F926F927F92BB
:10A9A0008F929F92AF92BF92CF92DF92EF92FF92DF
:10A9B0000F931F93CF93DF93D82E8FE99FE00E94D0
:10A9C000F6198FEB98E06D2D45E020ED37E00AE0B9
:10A9D00076EAE72E7FE0F72E51E1C52E11E1A12E98
:10A9E0000E94F11BF090BF08FA948090C0088F2D50
:10A9F00066E00E9463428D2D803821F59F2D9031B5
:10AA000008F5EF2DFF27E7FDF09580911F05E81B66
:10AA1000F109EE0FFF1FEB5DFA4FC081D1818F2D41
:10AA20000E94990EFC01882069F48281882319F024
:10AA3000D095C195DF4FD483C38382E00E94105824
:10AA40000E94AC5818E09924552453946F2C772415
:10AA500067FC709400911F05090D003109F4E1C0F5
:10AA6000802F0E94990EEC018A816B817C81882362
:10AA700019F0709561957F4FA02EBB24F501EE0F64
:10AA8000FF1FEB5DFA4F20813181261B370B2333EB
:10AA9000310524F0F501E155F74F08C09FEF2E3C3A
:10AAA00039072CF4F501E155F74F85258083402FB8
:10AAB0004F5F80E0612F20E00E94560FF501E155C5
:10AAC000F74F8081882311F04FE701C04EE78BE4F8
:10AAD000612F20E00E942C5DEE246A147B0471F447
:10AAE0008E1461F480912005882359F480919C0490
:10AAF00090919D04009739F401E001C000E0CC245E
:10AB000005C002E001C001E0CC24C3948E2D823048
:10AB100009F43FC0833009F45DC08130C1F04B813E
:10AB20005C81202F206280E3612F0E946260CC2034
:10AB300009F46BC06B817C818D2D48E15CEF28EEC0
:10AB400033E002E00E94D4139C838B835EC0488173
:10AB50004456552747FD509588E4612F202F0E94C9
:10AB60006260CC2009F451C068816456688380918A
:10AB7000BA0181FF04C08D2D43E82DE703C08D2D60
:10AB80004CE924E60E949814888388818C59888334
:10AB90003CC049814C59552747FD509586E6612FA9
:10ABA000202F0E946260CC2081F169816C596983F9
:10ABB0008091BA0181FF04C08D2D43E82DE703C0C9
:10ABC0008D2D4CE924E60E9498148983898184564E
:10ABD00089831BC08A8190E0AC01440F551F480F48
:10ABE000591F4856504F8CE6612F23E00E94EF5DBD
:10ABF000CC2059F08D2D6A8140E021E00E9498140C
:10AC000091E0882309F490E09A83E3949E2D943098
:10AC100009F063CF9394185F892D873009F01ACF1C
:10AC20001FC001E09F2D903109F000E080912105C7
:10AC3000882311F020E001C0202F82E1612F47E836
:10AC40005FE00E941F5E002359F08D2D803841F493
:10AC500089E18093210580E80E942B620E94093FD0
:10AC6000DF91CF911F910F91FF90EF90DF90CF90E8
:10AC7000BF90AF909F908F907F906F905F9008955E
:10AC8000F8942091D70D3091D80D7894C90108958A
:10AC9000CF93DF93C4E4D1E080E6FE0111928A9560
:10ACA000E9F78AE08093440189E1809372018AE5A3
:10ACB0008093730181E0809388012196FE0120E05A
:10ACC00032E080E891E02193319395878487938FD8
:10ACD000828F41E0E335F407B1F785E991E068E858
:10ACE00070E14AE050E00E94106F80E090E029910E
:10ACF0003991820F931FE1E0CD35DE07C1F79093C4
:10AD0000700180936F01DF91CF9108951F93CF93CE
:10AD1000DF938AEC98E060E00E946C5A64E471E092
:10AD200080E6FB0111928A95E9F78AEC98E040E60B
:10AD300050E00E94F85A182FC5E9D1E088810E949E
:10AD4000FB2D0E940B2E8993F1E0CF39DF07B1F77D
:10AD5000809144018A3028F480918104816080933D
:10AD600081048AE0809344011D3468F0E5E4F1E059
:10AD700020E030E081919191280F391F81E0ED357D
:10AD8000F807C1F702C020E030E081E040916F0198
:10AD9000509170014217530709F080E0DF91CF9185
:10ADA0001F9108951F93182FE4EAF1E025EA32E09D
:10ADB000DF01C9011D920197E9F7CF016DE770E14D
:10ADC0004AE050E00E94106F812F90E001966AE007
:10ADD00070E00E94BA6E605D6093A901805D80930F
:10ADE000AA018AE08093AE0180E00E945C631F911B
:10ADF0000895CF92DF92EF92FF920F931F93DF930C
:10AE0000CF930F92CDB7DEB76B01803160F5682F1D
:10AE10006F5F8AEC98E049830E946C5A4981042F45
:10AE200010E0C60160E270E050E00E94316F8AECF1
:10AE300098E0B6014AE050E00E94F85A8A30910545
:10AE400091F48AEC98E00E945E5AF601E00FF11F3F
:10AE50002AE030E006C0B9010E94A66E805D8293B0
:10AE6000CB010097C1F70F90CF91DF911F910F9108
:10AE7000FF90EF90DF90CF9008958F5F0E94EF5981
:10AE800008951F93CF93DF93182F803168F5682FB3
:10AE90006F5F8AEC98E00E946C5A64EA71E025EAE0
:10AEA00032E0FB01C90111920197E9F78AEC98E0C1
:10AEB00045EA52E00E94F85A8F3F910509F018F4D4
:10AEC000812F0E94D256C4EAD1E088810E94FB2DD6
:10AED0000E940B2E899391E0CE3AD907B1F78AE010
:10AEE0008093AE010E943415DF91CF911F91089598
:10AEF0000F931F93DF93CF93CDB7DEB760970FB655
:10AF0000F894DEBF0FBECDBF682F6F5F062F0AC05B
:10AF1000102F1F5F812F688B0E94EF59688988234B
:10AF200029F0012F0031A0F3003139F18AEC98E0CB
:10AF30000E946C5A602F6F5F83ED98E042E028E535
:10AF400032E00E94DE5B8E010F5F1F4F06C083ED73
:10AF500098E0B8010E94595BA8958AEC98E0B80186
:10AF60004FE050E00E94875A482F882381F783EDF5
:10AF700098E00E94075C81E001C080E060960FB617
:10AF8000F894DEBF0FBECDBFCF91DF911F910F911F
:10AF90000895EF920F931F930E94DA59882341F08E
:10AFA0000E94455987FD04C00E948656882381F57A
:10AFB0008DE690E161E00E94A3128BE590E10E9492
:10AFC0008A120E94B4590E9448568AEC98E060E0C8
:10AFD00041E024E431E000E610E078ECE72E0E9446
:10AFE000365C8036910529F08CE490E160E00E94A7
:10AFF000A31280E00E94D2568AEC98E061E042E021
:10B0000024EA31E005EA12E058ECE52E0E94365CB5
:10B01000809171010E9441571F910F91EF90089507
:10B02000882359F09091E608982B9093E6080E94A7
:10B03000810E9093E8088093E7080895EF920F93AC
:10B040001F93CF93DF931091E608112309F47EC07C
:10B05000882309F076C00E94810E2091E708309184
:10B06000E808AC01421B530B4436510508F46EC08E
:10B0700068C081E08093E508812F90E0EC01C47006
:10B08000D07012FF03C023E02093E5081092E60879
:10B0900080FF1CC08CED98E061E141E024E431E0E8
:10B0A00000E610E0F4E1EF2E0E94365C8036910558
:10B0B00011F480E020C08091E208823021F4809178
:10B0C000E608816029C08CE390E135C081FF36C07D
:10B0D0008CED98E061E142E024EA31E005EA12E01B
:10B0E000E4E1EE2E0E94365C52E0853A950739F491
:10B0F000809171018F5F61E10E94FD591FC08091B5
:10B10000E2088230A1F48091E608982F9260909333
:10B11000E608209719F086608093E6080E94810E69
:10B12000845690409093E8088093E70807C02097E2
:10B1300029F48CE290E160E00E94A3121092E508ED
:10B1400005C08091E508882309F493CFDF91CF9162
:10B150001F910F91EF9008950AC081E00E941E5840
:10B1600080916B0E833019F4A89510926B0E80912C
:10B17000E608882391F70895DF93CF930F92CDB718
:10B18000DEB7682F70E084E0660F771F8A95E1F7DD
:10B19000CE01019641E050E00E94386F89810F9006
:10B1A000CF91DF910895DF93CF930F92CDB7DEB7A4
:10B1B0006983682F70E094E0660F771F9A95E1F736
:10B1C000CE01019641E050E00E94FF600F90CF91C8
:10B1D000DF91089589EE98E060E070E040E450E08F
:10B1E0000E94FF6008958BEE98E062E070E041E01D
:10B1F00050E00E94FF6008950F931F93182F082FAF
:10B2000004C0802F0E94BC58082F802F0E94BC5879
:10B210008823B9F7802F6091EB080E94D3581093D0
:10B22000EB080E94F3581F910F9108951F931091FE
:10B23000EB08112359F0812F0E94BC588093EB0832
:10B240000E94F358812F60E00E94D358812F1F91F4
:10B250000895F8942091D70D3091D80D7894C901B4
:10B260000895EF92FF92CF93DF938091EB08C0E0B7
:10B27000D0E003C02F960E94BC588823D9F7CE0196
:10B28000DF91CF91FF90EF900895CF92DF92EF92F0
:10B29000FF920F931F93CF93DF9380E8E9E2F9E0E9
:10B2A000DF011D928A95E9F70DEE18E0C0E0D0E0CD
:10B2B0008C2FC43139F4D090EB083BEEE32E38E00C
:10B2C000F32E0BC07E01EE0CFF1CEC0EFD1E2DEECE
:10B2D00038E0E20EF31ED801DC9090E0C82EC39453
:10B2E0001DC08D2D84508C3738F4ED2DF0E0E75DD6
:10B2F000F64F8081882361F0992329F0892F60E03F
:10B300000E94D3580DC0F70110820E94EA5808C06D
:10B31000C0828D2D0E94BC589D2DD82EDD2009F7AE
:10B3200021960D5F1F4FC531D10511F604E0E02FC6
:10B33000F0E0E75DF64F8081882349F4802F60912B
:10B34000EB080E94D3580093EB080E94F3580F5F5C
:10B35000003869F780E0DF91CF911F910F91FF9046
:10B36000EF90DF90CF9008951F9380E4E9EEF8E02E
:10B37000DF01982F1D929A95E9F794E09093E908E0
:10B380008093EA0880E18093EC0884E001C0812F7B
:10B39000182F1F5F612F0E94D3581038C1F78FE715
:10B3A00060E00E94D35884E08093EB080E94EA5842
:10B3B0001F91089589EE98E060E070E040E450E06D
:10B3C0000E94386F8091E908843039F481E09091CF
:10B3D000EA08903419F080E0089580E0089590E044
:10B3E000FC01EE0FFF1FE80FF91FE751F74F81E057
:10B3F0009481992309F480E00895DF93CF9300D0DE
:10B400000F92CDB7DEB790E0FC01EE0FFF1FE80F03
:10B41000F91FDE011196E351F74F23E001900D92E1
:10B420002150E1F770E0DC01AA0FBB1FA80FB91F84
:10B43000FB01EE0FFF1FE60FF71FA351B74FE351BC
:10B44000F74F83E001900D928150E1F7FB01EE0F81
:10B45000FF1FE60FF71FE351F74FDE01119683E060
:10B460000D9001928150E1F70E94EA580F900F90E1
:10B470000F90CF91DF910895DF93CF930F92CDB7C7
:10B48000DEB790E09C01220F331F280F391FF9010E
:10B49000E751F74F84812351374F93E0D9011D9233
:10B4A0009A95E9F789830E94EA588981882311F0E7
:10B4B0000E94FC580F90CF91DF910895FC0180818C
:10B4C00090E0FC01EE0FFF1FE80FF91FE251F74F6C
:10B4D000918180819F700895FC01608312821182A6
:10B4E00070E0CB01880F991F860F971FDC01A751D1
:10B4F000B74F14962C9114972383148215821682C9
:10B500008151974FFC01808182958F7008958F92B1
:10B510009F92AF92BF92CF92DF92EF92FF920F93E2
:10B520001F93DF93CF930F92CDB7DEB78C015B01F2
:10B53000FC01808190E0FC01EE0FFF1FE80FF91F76
:10B54000E251F74F80812181922F9F70F801218174
:10B550003281821B930BE42EF52E8E159F0508F485
:10B560007C0167014E010894811C911C25C0F801E3
:10B570006381662321F184818F5F848370E0B4E06E
:10B58000660F771FBA95E1F7680F711DC40141E09E
:10B5900050E00E94386F8981F50181935F01F801C5
:10B5A00084818F3030F0148283810E94BC58F8016E
:10B5B00083830894C108D108C114D104C1F6F801ED
:10B5C000818192818E0D9F1D8C199D0992838183AB
:10B5D0008E2D8C190F90CF91DF911F910F91FF90BD
:10B5E000EF90DF90CF90BF90AF909F908F90089595
:10B5F0008F929F92AF92BF92DF92EF92FF920F9342
:10B600001F93CF93DF938C015B017A01C0E0D0E000
:10B6100045E0842E912C880E991E3BC0F80185814F
:10B6200090E08F779070009741F4C801B40141E039
:10B6300050E00E94875A813079F5F80145813FE753
:10B64000D32ED4222D2D30E0C7018C1B9D0B8217E9
:10B65000930710F4DE2CDC1AB5016C0F7D1F47FF39
:10B6600008C0CB0160E070E04D2D50E00E94316FCA
:10B670000AC0C8014D2D50E00E94875A8D1519F05F
:10B68000C80FD11D09C0CD0DD11DF80185818D19BF
:10B690008583CE15DF0510F2CE01DF91CF911F918A
:10B6A0000F91FF90EF90DF90BF90AF909F908F90A1
:10B6B00008959F92AF92BF92CF92DF92EF92FF9246
:10B6C0000F931F93CF93DF93EC018B01C42E8B81DB
:10B6D000882389F489819A81009769F4E880FF249E
:10B6E0000E9416598B83F701EE0FFF1FEE0DFF1D11
:10B6F000E751F74F8483DC2C6FE0962E44C0EF8037
:10B70000F8840E94810EE81AF90AF7FE02C082E06E
:10B7100004C08B81882319F481E08E8337C09C811B
:10B720009F3080F01C820E94BC58882339F4EB8043
:10B730000E941659682F8E2D0E94D3588B810E942B
:10B74000BC588B838B81882339F36C81992D961B90
:10B75000ED2C9D1508F4E92EAE2CBB2470E06F5F34
:10B760007F4F90E054E0880F991F5A95E1F7680FDA
:10B77000791FC801A5010E94FF600A0D1B1D8C8165
:10B780008E0D8C83DE18DD2009F0B9CF2C2D30E032
:10B790002D19310989819A81820F931F9A83898398
:10B7A0008C2D8D19DF91CF911F910F91FF90EF900C
:10B7B000DF90CF90BF90AF909F9008950F931F930D
:10B7C000CF93DF93EC01890168831A82198270E0BC
:10B7D000CB01880F991F860F971FFC01E751F74F88
:10B7E00024812B831C821D821E82FC01E251F74FB3
:10B7F00010824295407F41830E94810E080F191FDD
:10B8000018870F83DF91CF911F910F9108951F9398
:10B81000CF93DF93EC01888190E0FC01EE0FFF1FD6
:10B82000E80FF91FE251F74F898180839A819F7059
:10B830008181807F892B81838B81882389F00E947D
:10B84000BC58182F882361F08B8160E00E94D35888
:10B850000E94EA58112331F0812F0E94FC5802C047
:10B8600010E0F6CFDF91CF911F9108954F925F9234
:10B870006F927F929F92AF92BF92CF92DF92EF92A0
:10B88000FF920F931F93DF93CF930F92CDB7DEB745
:10B890005C01290168012E2D30E00E94DE5B1982D7
:10B8A000720100E010E081E03E010894611C711C0F
:10B8B000F70191917F01992341F4882349F4908104
:10B8C000992349F4992493941EC0882371F403C0EA
:10B8D0009924939401C0992499819F3718F40C15E9
:10B8E0001D0561F5882379F001C099248981882399
:10B8F00021F180688983C501B30141E00E94595B51
:10B900008130D1F025C089818823B9F0C501B30108
:10B9100041E00E94595B8130D9F44981B801641B30
:10B920007109640D751DC5010E94595B99818917C4
:10B9300019F0981B99830CC01982892D99819F5FFA
:10B9400099830F5F1F4FC016D10608F0B1CF05C015
:10B9500089818F776801C81AD108C5010E94075CE8
:10B96000C6010F90CF91DF911F910F91FF90EF9043
:10B97000DF90CF90BF90AF909F907F906F905F903F
:10B980004F90089580E094E0E9EAF9E0DF019C013E
:10B990001D9221503040E1F708950F931F93CF93EC
:10B9A000DF93DA011196FA014491ED012196FD0130
:10B9B000A491B0E0179613E0B595A7951A95E1F715
:10B9C0001A2FDE011196FE019491929FE00111243D
:10B9D000AC0FBD1F00FD08C001FF08C09091D90D3C
:10B9E00051E096FD04C002C051E001C050E06695F0
:10B9F0006695669570E09B013695322F2227379524
:10BA0000279590E0280F391F610F711D7695762FCD
:10BA1000662777956795680F791F042F10E014C08B
:10BA2000E901C755D64F80E090E008C0FD01E80F5E
:10BA3000F91FE4915111E095E99301968417B0F351
:10BA4000A00FB11F20583F4F2617370749F7DF9146
:10BA5000CF911F910F910895FF920F931F93CF9352
:10BA6000DF93942F46313CF4440F490F440F22FFDB
:10BA7000ABC0440FA9C0482F4A5F092F112707FD0B
:10BA8000109520FD09C021FF0AC03091D90DFF2477
:10BA9000F39436FD05C003C0FF24F39401C0FF24D6
:10BAA00066956695669570E07695762F662777950C
:10BAB0006795680F711DEB01C755D64F22FF4FC028
:10BAC0009E3209F04A5FC801809760E170E00E94F1
:10BAD000BA6E80EA90E0689F9001699F300D789F70
:10BAE000300D1124C801880F991F53E0000F111F5A
:10BAF0005A95E1F7800F911F280F391F275C3E4EA2
:10BB000085E0882369F0F9019491E056FF4F549144
:10BB10002F5F3F4FF9016491E056FF4F749104C0CD
:10BB200060E050E090E070E0FF2021F0909560959B
:10BB300050957095DE01AF57BF4FFDE0A93ABF07A2
:10BB400040F498836983FE01E058FF4F50837C9353
:10BB5000229681508F3FC1F12F5F3F4FD2CF23FFFD
:10BB60000DC0FF2011F08FEF01C080E06755764FC8
:10BB7000FB01808321964F5F91E001C090E0980126
:10BB8000220F331F220F331F200F311F2A50304F37
:10BB900085E0F9012F5F3F4FE491992311F0843044
:10BBA00039F0FDE0C93ADF0718F4F110E095E993A8
:10BBB000815079F75DE0C93AD50730F4FF2011F0E4
:10BBC0008FEF01C080E08883842FDF91CF911F9198
:10BBD0000F91FF90089520E00E942C5D0895CF9270
:10BBE000DF92EF92FF920F931F93CF93DF93162F65
:10BBF000F22EF0E1EF2EE022C42EE6016E01D52EEA
:10BC0000E6010CC0EE2011F0488102C0FE01449113
:10BC1000612F202F0E942C5DFA942196FF2091F72E
:10BC2000DF91CF911F910F91FF90EF90DF90CF9018
:10BC300008950F9300E00E94EF5D0F910895CF9259
:10BC4000DF92FF920F931F93CF93DF93162F022F54
:10BC5000A0E1FA2EF222C42EE6016E01D52EE601F5
:10BC6000FF2011F0488102C0FE0144912196442337
:10BC700029F0612F202F0E942C5DF2CFDF91CF9110
:10BC80001F910F91FF90DF90CF900895982FAB01F7
:10BC900080E0692F20E00E941F5E089520E00E944E
:10BCA0001F5E0895EF92FF920F931F93DF93CF9340
:10BCB0000F92CDB7DEB7182F062F7A01982F9C5E12
:10BCC00095504E2D4F704A301CF0495C28E002C060
:10BCD000405D20E0892F602F99830E942C5D99811F
:10BCE000911731F0B4E0F694E794BA95E1F7E8CF14
:10BCF0000F90CF91DF911F910F91FF90EF900895DA
:10BD0000E62FE695E695E695F0E0F695FE2FEE2710
:10BD1000F795E795E80FF11DE755F64F8DE0E93A05
:10BD2000F80758F4677081E090E002C0880F991F0F
:10BD30006A95E2F7208128272083089547FF02C0F3
:10BD4000840F4195E62FE695E695E695F0E0F695A9
:10BD5000FE2FEE27F795E795E80FF11DE755F64F13
:10BD60006770A1E0B0E001C0AA0F6A95EAF711C0C0
:10BD70008DE0E93AF80778F4822F90E09C01359540
:10BD8000279580FF04C080818A27808320684150E6
:10BD90003196442369F708952FEF0E949E5E08951F
:10BDA0000F931F93CF93DF93C82FD0E0E62FE69534
:10BDB000E695E695F0E0F695FE2FEE27F795E795E8
:10BDC000EC0FFD1FE755F64F062F10E0242F332709
:10BDD00027FD3095200F311FC90168E070E00E94F7
:10BDE000BA6E7695762F6627779567956C0F7D1FCF
:10BDF0006755764F0770107081E090E002C0880FA1
:10BE0000991F0A95E2F781959081892708C0E0582B
:10BE1000FF4F8DE0E93AF807D0F480818095808368
:10BE2000E617F707A0F38DE0E93AF80780F4C901B7
:10BE300068E070E00E94BA6E21E030E002C0220F9C
:10BE4000331F8A95E2F72195808182278083DF91D5
:10BE5000CF911F910F9108952F923F924F925F9231
:10BE60006F927F928F929F92AF92BF92CF92DF920A
:10BE7000EF92FF920F931F93DF93CF9300D00F9217
:10BE8000CDB7DEB7182F662E59016A01F02E802F2C
:10BE900005FF04C004FF04C002E003C000E001C0CD
:10BEA00001E0E7FE04C0E1942224239401C022248F
:10BEB000D7FE0BC0D094C094B094A094A11CB11C28
:10BEC000C11CD11C4424439401C0442482FF06C0F9
:10BED0009CE09093A90D3AE0932E05C096E09093D4
:10BEE000A90D25E0922E86FF2FC04110190D28EED6
:10BEF000A21623E0B20620E0C20620E0D20614F02B
:10BF0000190D06C034E6A316B104C104D10414F01F
:10BF1000190D06C08AE0A816B104C104D1040CF0C2
:10BF2000190D002391F0023039F4E4E6AE16B104A5
:10BF3000C104D10454F4190DFAE0AF16B104C104E0
:10BF4000D1041CF4190D01C0191B8091A90D810F9A
:10BF50008093A90D023011F420EFF20E5524539472
:10BF600092E0792E88242E2D332727FD3095862DBB
:10BF70008A5F89833B832A8370C0C601B5012AE0AA
:10BF800030E040E050E00E94EF6EE62E80E3382E75
:10BF90003E0C812F662D432D2F2D0E942C5D051503
:10BFA000D9F5F2FE23C08E2D8150833008F47394AE
:10BFB000C601B5012AE030E040E050E00E94EF6E9B
:10BFC000CA01B9012AE030E040E050E00E94EF6E83
:10BFD000623011F06430C1F4E32DE43319F4812EA2
:10BFE000839413C0812E8A9473940FC01250812FB2
:10BFF0008F5FF0FE05C0662D47E00E94D05E05C051
:10C0000069810E94805E01C0812EFAE0AF16B10402
:10C01000C104D1040CF000E0C601B5012AE030E013
:10C0200040E050E00E94EF6E59016A012115310590
:10C030004105510581F4002331F0023059F4252DDA
:10C04000223040F408C0F4FE10C0222021F430EF6A
:10C05000F30E01C000E019195394852D90E0EA8198
:10C06000FB81E817F9070CF088CF882061F0662D76
:10C07000645F882D472D0E94CC5E662D635F882DFE
:10C08000472D0E94CC5E442039F0812F8919662DFE
:10C090004DE22F2D0E942C5D0F900F900F90CF91AD
:10C0A000DF911F910F91FF90EF90DF90CF90BF90A5
:10C0B000AF909F908F907F906F905F904F903F9048
:10C0C0002F900895EF920F93022FFA019F014427BA
:10C0D00037FD4095542F75E0E72E0E942C5F0F919D
:10C0E000EF90089520E00E9462600895A998AB98AF
:10C0F000AC988BBBAD9AAD98AB9AA99A089520E005
:10C1000030E006C045E04A95F1F700002F5F3F4F51
:10C1100028173907BCF30895AA9885E08A95F1F7A6
:10C12000000085E08A95F1F70000AA9A8CED95E071
:10C130000E947F6082EE0E9476608EEA0E947660A6
:10C1400081EA0E94766086EA0E94766084EA0E9414
:10C15000766082EA0E94766080EC0E9476608FE2D0
:10C160000E94766085E20E94766081E80E94766097
:10C1700082E20E9476608FEA0E94766082E280937B
:10C18000720108951F93182F81E80E947660812F15
:10C190000E9476601F9108951F93CF93DF9310E064
:10C1A000C9EAD9E084E00E94766080E10E9476606E
:10C1B000812F806B0E947660A998AB9AAC98FE01A3
:10C1C00080E290819BBBAD9AAD9891819BBBAD9A6B
:10C1D000AD9892819BBBAD9AAD9893819BBB3496F1
:10C1E000AD9AAD98815069F7C058DF4FAB9AA99AC4
:10C1F0001F5F1830B9F6DF91CF911F910895BF925C
:10C20000CF92DF92EF92FF920F931F93CF93DF9322
:10C21000EA01E82EF92E062F172F21C0F701B19061
:10C220007F0168010894C11CD11C04C0009739F03B
:10C230000E94BB188091E50890E082709070E199AF
:10C24000F5CF1FBB0EBBE09A8DB3B81631F0BDBA67
:10C250008FB7F894E29AE19A8FBF219786012097D1
:10C26000E9F6DF91CF911F910F91FF90EF90DF9052
:10C27000CF90BF9008958093DA0D08958091DA0DE4
:10C280001092DA0D0895FC018081982F990F9E700D
:10C29000807F892B8083662321F09160807F892BAA
:10C2A000808381818F5F81839281992391F02081A6
:10C2B0002F7079F4933659F0242F20622093DA0DF1
:10C2C000903111F4803118F080818F7C808311824D
:10C2D00012828281883009F443C0893058F4813059
:10C2E00009F446C08130A0F08230D1F1843009F0E9
:10C2F00052C036C08F3549F1803620F4803109F0C4
:10C300004AC02EC0813689F0823609F044C03DC053
:10C310008081982F9F709F30F1F591E692839181F3
:10C320009131E0F08F7C808319C040664093DA0D34
:10C330009081892F82958F708F5F83708295807F27
:10C340009F7C982B90838FE508C08181883111F400
:10C35000406818C08832F9F480E182831182089520
:10C360009181903328F090E0959587958283118292
:10C37000828190E00197218130E08223932300970E
:10C3800051F440644093DA0D08958181803418F0AF
:10C3900088E08283118208958E3091056CF4FC014F
:10C3A000EE0FFF1FE80FF91FE355F24F90819F70CA
:10C3B00081E09F30E9F53FC0823131F1833160F493
:10C3C0008F30C9F0803118F48E3091F52AC0803159
:10C3D00061F0813169F513C0843151F08431D0F0BE
:10C3E0008531E1F0863121F51EC091B194701DC0F8
:10C3F00093B390781AC090916300917016C0909199
:10C4000063009095987011C08091630083FF12C003
:10C4100091B102C091B19095907407C091B19071A3
:10C4200004C093B3F9CF91B1907281E0992319F4CC
:10C4300080E0089580E008958F708E3058F490E089
:10C44000FC01EE0FFF1FE80FF91FE355F24F82E6E4
:10C450008283118208958F708E3068F490E0FC0121
:10C46000EE0FFF1FE80FF91FE355F24F83E68283BB
:10C4700080818F7C808308950F931F93CF93DF93E8
:10C480008091D70D9091D80D01969093D80D8093FF
:10C49000D70D8091D90D8F5F8093D90D06B300958C
:10C4A00040E050E010E001C0AE01EA012196CA016F
:10C4B000880F991F840F951FB8010C2E02C0759527
:10C4C00067950A94E2F7617070708355924F50E05F
:10C4D0000E944361C630D10539F700B30095C0E032
:10C4E000D0E0FE01E750F64EE4919E012A5F3F4FF7
:10C4F000C901880F991F820F931F8355924FE02324
:10C5000061E009F460E09E012A5F422F50E00E9442
:10C5100043612196C830D10521F7DF91CF911F915A
:10C520000F910895FF920F931F93CF93DF93F82EEF
:10C53000EEEBF1E080E090E0582F9C014081F41692
:10C5400038F0442329F001963A9681329105A1F7FB
:10C550005032B9F1E901CC0FDD1FC901A3E0880F0A
:10C56000991FAA95E1F7C80FD91F8E0102541E4FDB
:10C57000A9014F5F5F4FCA01880F991FE3E0440F85
:10C58000551FEA95E1F7840F951F20953095205EA1
:10C590003F4FA901440F551F63E0220F331F6A95D7
:10C5A000E1F7420F531F82549E4FB8010E941F6F44
:10C5B0008AE0D8011D928A95E9F7CC55DE4FFA8EB4
:10C5C00002C00EEB11E0C801DF91CF911F910F91D6
:10C5D000FF90089580E491E0EEEBF1E0DF019C0133
:10C5E0001D9221503040E1F70895EAE8F3E088E237
:10C5F000DF011D928A95E9F7B89688E4DF011D9264
:10C600008A95E9F70895282F30E08830C0F4462F46
:10C61000572FDA01F901EE0FFF1FEE0FFF1FE20F98
:10C62000F31FE657FC4F95E0899FC0011124815705
:10C630009C4F2D912193E817F907D9F70895462FBC
:10C64000572FDA0128503040F90193E0EE0FFF1F19
:10C650009A95E1F7E20FF31FEE54FC4F99E0899FA2
:10C66000C00111248D589C4F2D912193E817F90793
:10C67000D9F7089590E00197FC01EE0FFF1FE80F36
:10C68000F91FEC55FE4FDF01A85ABD4F6C93DF0137
:10C69000AA5ABD4F4C93E95AFD4F20830895E0916B
:10C6A0008801F0E0EE0FFF1FEE0FFF1FE80FF11DF6
:10C6B000E151FB4F849108958F929F92AF92BF9268
:10C6C000CF92DF92EF92FF920F931F93DF93CF935E
:10C6D000CDB7DEB76D970FB6F894DEBF0FBECDBFF6
:10C6E000F82EDE011596E6E2F1E085E001900D926C
:10C6F0008150E1F7DE011A96E1E2F1E085E0019078
:10C700000D928150E1F7DE011F96ECE1F1E085E04A
:10C7100001900D928150E1F7DE015496E7E1F1E0DE
:10C7200085E001900D928150E1F7DE015996E2E13A
:10C73000F1E085E001900D928150E1F719821A82B3
:10C740001B821C82E0918D01F0E0E852FB4F26E055
:10C7500030E011E0E491CE2EDD24BE016F5F7F4F0B
:10C760000FC04F5F5F4FA417B50711F4FC01108392
:10C7700044305105B1F71F5F22503040153081F031
:10C7800040E050E0C601022E02C0959587950A94BC
:10C79000E2F783709070DC011196860F971FE1CF4E
:10C7A000FF2041F50E94EA6289810E9492628C0119
:10C7B00081E00E944F63F801818374E6F72EF282D4
:10C7C0008A810E9492628C0182E00E944F63F8018C
:10C7D0008183F2828B810E9492628C0183E00E94AD
:10C7E0004F63F8018183F2828C810E9492628C01F6
:10C7F00084E07EC0FF2DF13071F48B810E94926243
:10C80000FC0188E081838CE98283F3828781817FC8
:10C8100084608783D7C18F2D8230E9F58B810E9498
:10C820009262FC0108E001836CE9F62EF28285E158
:10C8300083838781817F846087838EE00E949262F8
:10C84000FC0182E2818314E612838EE00E949262F0
:10C85000FC010183F28284E183838781817F84608C
:10C8600087838EE00E949262FC010183128381E043
:10C8700083838781817F8460878383E00E944F6305
:10C88000482F8BE062E02DE90E943A638CE061E082
:10C8900042E220E095C1EF2DE33081F50E94EA628B
:10C8A000E9808E2D0E9492628C0181E00E944F638C
:10C8B000F801818354E6F52EF2828E2D0E94926259
:10C8C0008C0182E00E944F63F80181838CE98283AE
:10C8D000EA808E2D0E9492628C0181E00E944F635B
:10C8E000F8018183F2828E2D0E9492628C0182E097
:10C8F0000E944F63F8018183F28264C1FF2DF430FE
:10C9000081F50E94EA62EA808E2D0E9492628C017B
:10C9100082E00E944F63F801818344E6F42EF282A4
:10C920008E2D0E9492628C0184E00E944F63F80178
:10C930008183F282EC808E2D0E9492628C0182E0D3
:10C940000E944F63F8018183F2828E2D0E949262D1
:10C950008C0184E00E944F63F80181838CE982831B
:10C9600031C1FF2DF53009F0D0C00E94EA620E946B
:10C97000F56281E00E949262FC013AE0C32EC1821E
:10C9800024E6B22EB28282E00E949262FC019BE019
:10C99000D92ED182B28283E00E949262FC018CE0A7
:10C9A000E82EE182B28284E00E9492628C0181E0F2
:10C9B0000E944F63F8018183B28285E00E949262F7
:10C9C0008C0183E00E944F63F8018183B28204E00E
:10C9D000A02EA38287E0848387818160878385E09E
:10C9E0000E9492628C0183E00E944F63F801818370
:10C9F000B282F38218E0812E8482878181608783EE
:10CA000085E00E9492628C0183E00E944F63F801EE
:10CA10008183B282B6E0BB2EB382A9E09A2E9482C3
:10CA200087818160878385E00E949262FC01818218
:10CA30008CE9828381E083838781817F846087831F
:10CA400086E00E949262FC0191828EE1828388EFEF
:10CA500083838BE00E9492628C0183E00E944F638B
:10CA6000F801818376E4972E9282A382C482878123
:10CA7000816087838BE00E9492628C0183E00E9438
:10CA80004F63F80181839282F382D482878181602F
:10CA900087838BE00E9492628C0183E00E944F6347
:10CAA000F80181839282B382E482878181608783E7
:10CAB0008091BA018F7180628093BA018FE1809377
:10CAC000BB0180E0BE016B5F7F4F0E94036381E08A
:10CAD000BE01665F7F4F0E94036382E0BE01615F1B
:10CAE0007F4F0E94036383E0BE016C5E7F4F0E9414
:10CAF00003638E01075E1F4F84E0B8010E94036349
:10CB000085E0B8010E9403635DC0FF2DF630B1F4EB
:10CB100086E00E949262FC01F18282E3828388EFC8
:10CB2000838314E6108786E00E949262FC01F18202
:10CB30008EEC828388E08383108744C08F2D8730FA
:10CB400009F040C08FE00E949262FC0184E2818380
:10CB500084E6828388E8868380E10E949262FC01F9
:10CB600089E081830EE602838AE0838380E10E946C
:10CB70009262FC0118E0118382E982838BE0838357
:10CB80008781817F8460878380E10E949262FC01BB
:10CB9000118302838CE083838781817F8460878314
:10CBA00081E06BE043E224E20E943A6382E061E0CC
:10CBB00043E229E60E943A6383E062E043E227E928
:10CBC0000E943A6382E00E9410580E94AC586D9611
:10CBD0000FB6F894DEBF0FBECDBFCF91DF911F918E
:10CBE0000F91FF90EF90DF90CF90BF90AF909F900C
:10CBF0008F9008956F927F928F929F92AF92BF9283
:10CC0000CF92DF92EF92FF920F931F93CF93DF9318
:10CC10008091BA0181FF03C060E075E002C060E06E
:10CC200074E09091B70184E69802C0011124885AFB
:10CC30009D4FE091BD01FF27E7FDF09548EE53E0E1
:10CC4000E49F9001E59F300DF49F300D112428538F
:10CC50003045AA24BB24A81AB90A281B390BF5E2CF
:10CC6000EF2EF5E0FF2E4091B401440F485F50E0F5
:10CC7000440F551F440F551F4552524FEBEDFDE039
:10CC8000CC24DD24C61AD70AA8E5B2E0A81BB90B4C
:10CC90001CC0E701699079907E014B01661677060A
:10CCA0000CF4430184018C149D040CF48601005A99
:10CCB000164FE501C01BD10B2C0F3D1F0A0F1B1F88
:10CCC00011830083938382833496E417F50709F771
:10CCD000318320839383828315821482DF91CF91E5
:10CCE0001F910F91FF90EF90DF90CF90BF90AF908A
:10CCF0009F908F907F906F900895E0912B01F0911D
:10CD00002C018193F0932C01E0932B010895FF9265
:10CD10000F931F93CF93DF93B9E0FB2E90E120E0B8
:10CD2000C82FD0E08E0101701070201711F4905FB1
:10CD300007C0892F90E001970E947D66202F90E127
:10CD4000FA9431F0D595C795AE014068842FE8CFAD
:10CD5000892F90E00F960E947D66DF91CF911F9101
:10CD60000F91FF9008951F93CF93DF93182F2BED12
:10CD70003DE030932C0120932B0180913101877489
:10CD800071F08091B401882319F0813029F402C038
:10CD900080E803C080E901C088E980933101809177
:10CDA000310187FF0BC086E190E00E94CC618823AF
:10CDB00029F4809131018F77809331018091310185
:10CDC00087FD5AC085E160E040E00E94541088234E
:10CDD00009F452C0809131018062809331018091C9
:10CDE00071018F5F80933201E3E3F1E0A5E2B5E0EA
:10CDF00080E01CC02D913D913595279520503E4FE8
:10CE000037FD05C093E02F3F390724F405C020E02B
:10CE100030E002C02FEF33E0932F9370482F440F80
:10CE2000440F942B908321838F5F3296811711F7E3
:10CE3000C1E3D1E089910E94876681E0CF33D807B2
:10CE4000C9F780912B0190912C01019790932C01AF
:10CE500080932B018FEF90E00E947D6680E090E050
:10CE60000E947D668BED9DE09093300180932F01B1
:10CE7000DF91CF911F910895809131018F7DADCFCA
:10CE80001F920F920FB60F9211242F938F939F939F
:10CE9000EF93FF9388B391E0892788BBE0912F013E
:10CEA000F09130012191F0933001E0932F01822F16
:10CEB00090E097BD86BD293C08F0C09A80916B0E2A
:10CEC000816080936B0EFF91EF919F918F912F91D5
:10CED0000F900FBE0F901F9018951F920F920FB6D4
:10CEE0000F9211242F933F938F939F93EF93FF9370
:10CEF00088B391E0892788BBE0912B01F0912C0148
:10CF0000208130E020FD04C088B599B5809603C02B
:10CF100088B599B5409699BD88BDC9019595879505
:10CF2000009791F4CF01019690932C0180932B01EF
:10CF30008181882351F48091780090917900805309
:10CF4000984F99BD88BD01C0808380916B0E816030
:10CF500080936B0EFF91EF919F918F913F912F9155
:10CF60000F900FBE0F901F901895EDE7F0E08081B5
:10CF7000857E808317981F9AAAE8B0E01C921092D1
:10CF80008B0082E88C938081806280830895EDE736
:10CF9000F0E080818F7D8083179AAAE8B0E01C9230
:10CFA00010928B008AE08C93808188618083089541
:10CFB0001F920F920FB60F9211248F939F93AF93EE
:10CFC000BF93EF93FF938091770E882321F01F9AF0
:10CFD0001092770E04C01F9881E08093770EA09185
:10CFE0002D01B0912E01FD018191919190938700C7
:10CFF00080938600F0932E01E0932D0180916E0EB8
:10D0000090916F0E909385008093840012968D917D
:10D010009C911397009759F483E29EE090932E0120
:10D0200080932D018091BA0181708093770E809159
:10D030006B0E816080936B0EFF91EF91BF91AF916A
:10D040009F918F910F900FBE0F901F901895AF92E8
:10D05000BF92CF92DF92EF92FF920F931F93CF93E5
:10D06000DF938091BA0181FF03C040E055E002C028
:10D0700040E054E0F090B401FF0C80E1F80E209104
:10D08000B70184E6280290011124285A3D4FE0910F
:10D09000BD01FF27E7FDF09568EE73E0E69FC00154
:10D0A000E79F900DF69F900D112488539045CC2456
:10D0B000DD24C21AD30A821B930B68EFE62EEF0C15
:10D0C000E3E2FEE000271127041B150B68E572E080
:10D0D000621B730B21C0AE2DB0E0AA0FBB1FAB5D6E
:10D0E000BA4FAC901196BC90D5014A175B070CF46F
:10D0F000DA01A017B1070CF4D801A05AB64FE60127
:10D10000CA1BDB0B8C0F9D1F31832083A60FB71F1B
:10D11000B383A2833496E394EF14E8F2318320833F
:10D1200093838283885E934090936F0E80936E0EFC
:10D1300015821482DF91CF911F910F91FF90EF9094
:10D14000DF90CF90BF90AF9008951F920F920FB6CF
:10D150000F9211242F933F934F935F936F937F937D
:10D160008F939F93AF93BF93EF93FF9378940E9415
:10D170002768FF91EF91BF91AF919F918F917F9120
:10D180006F915F914F913F912F910F900FBE0F9034
:10D190001F9018952091740E3091750E90E08227A3
:10D1A00093279070880F991F8B59954EFC014591DC
:10D1B0005491232F3327422753275093750E4093C2
:10D1C000740E08959091700E96959695982B909365
:10D1D000700E8091710E8F5F8093710E843068F0B5
:10D1E000E091720EF091730E9193F093730EE093B1
:10D1F000720E1092700E1092710E089503C080E0AE
:10D200000E94E2688091710E8823C9F7E091720E46
:10D21000F091730E10820895882339F08091760E74
:10D220008F5F8093760E80E803C01092760E80ECBC
:10D230000E94E2688091760E8530B8F708950F93CA
:10D240001F93182F0E94CA6808E0812F81700E94E6
:10D250000C6916950150C9F71F910F91089580EC44
:10D260000E94E26880E80E94E26880E80E94E2682A
:10D2700080E80E94E26880E80E94E26880E80E94FC
:10D28000E26880E80E94E26880EC0E94E26808950B
:10D29000AF92BF92CF92DF92EF92FF920F931F93C4
:10D2A000CF93DF938BED9DE090932C0180932B0126
:10D2B0009093730E8093720E1092750E1092740EEE
:10D2C0001092700E1092710E1092760E0E942F69BD
:10D2D0008091B4010E941F6980916D0E0E941F69A8
:10D2E00080E00E941F6910926D0E05E215E054E087
:10D2F000C52ED12CF80120813181C901880F991FD9
:10D30000820F931FB6010E94BA6EEB012281338116
:10D31000C901880F991F820F931FB6010E94BA6E30
:10D3200060507C4FC050DC4FF8E0C030DF0710F099
:10D33000CFEFD7E07B0128E06030720720F0AFEF3D
:10D34000EA2EA7E0FA2E8C2F0E941F695E019B2D0A
:10D350009F708E2D8295807F892B0E941F69C70147
:10D36000F4E096958795FA95E1F70E941F690C5FA6
:10D370001F4F25E00533120709F0BCCF0091750E51
:10D380008091740E0E941F69802F0E941F690E9465
:10D390002F690E94FE688091780090917900805CEE
:10D3A00093469093790080937800C09ADF91CF9153
:10D3B0001F910F91FF90EF90DF90CF90BF90AF90B3
:10D3C00008958091B30190916C0E981709F494C060
:10D3D00080936C0E8130F9F0813030F08230F1F1C1
:10D3E000833009F089C05EC00E94B5671EBC80E42E
:10D3F0009CE99BBD8ABD1DBC1CBC87B7837C87BFD5
:10D400008CE386BF8FE380937C0087B7806187BF02
:10D410001FBC8AE021C00E94B5671EBC1DBC1CBC9D
:10D4200080E797E199BD88BD80EA9FE090937900FD
:10D430008093780087B7837C87BF8CE386BF8FE3B8
:10D4400080937C0087B7886087BF80917D00816072
:10D4500080937D001FBC82E08EBD4EC00E94B567E8
:10D460001EBC88EC90E090937900809378008CE269
:10D4700091E09DBD8CBD80EE9BEA97BD86BD87B7D0
:10D48000837C87BF8CE386BF8FE380937C0087B764
:10D49000806287BF80917D00816080937D001FBC8A
:10D4A0008AE1DACF1EBC80E49CE99BBD8ABD1DBC2D
:10D4B0001CBC87B7837C87BF80917D008E7F809363
:10D4C0007D008CE386BF8FE380937C0087B780610B
:10D4D00087BF1FBC8AE08EBD0E94276880E593EC61
:10D4E000909387008093860088E893E1909385006D
:10D4F000809384000E94C7678091B301813051F00E
:10D50000813028F0823051F0833079F40CC00E94D1
:10D51000FA65089578940E9448690895789486E0A1
:10D520000E94B36608950E94FA6508951F920F92B3
:10D530000FB60F9211242F933F934F935F936F93E6
:10D540007F938F939F93AF93BF93EF93FF938091BC
:10D55000B3018230C1F480E492EA97BD86BD809128
:10D560007800909179008F3F910538F488E598E92B
:10D57000909379008093780008C088EC90E09093B5
:10D580007900809378000E94E169FF91EF91BF914B
:10D59000AF919F918F917F916F915F914F913F914B
:10D5A0002F910F900FBE0F901F9018951F920F9202
:10D5B0000FB60F9211242F933F934F935F936F9366
:10D5C0007F938F939F93AF93BF93EF93FF938CB50C
:10D5D0009DB52091780E222321F0C09A1092780EEA
:10D5E00004C0C09821E02093780EA0913F01B09133
:10D5F0004001FD01219131913BBD2ABDF0934001D5
:10D60000E0933F012091C5063091C60628173907DF
:10D6100020F49093C6068093C50620910C013091AA
:10D620000D018217930720F490930D0180930C0154
:10D6300012968D919C9113970097D9F48BED9DE0F4
:10D640009093400180933F018091BA018095817051
:10D650008093780E87B78F7E87BF0E94E1698091A3
:10D66000B301882311F0833021F487B7806187BF2D
:10D67000789480916B0E816080936B0EFF91EF9197
:10D68000BF91AF919F918F917F916F915F914F91DA
:10D690003F912F910F900FBE0F901F901895909172
:10D6A00087019873903121F463E00E949A6E089587
:10D6B000983111F486950895983211F4880F0895E1
:10D6C000903319F4982F990F890F0895FC01A5E65E
:10D6D000B0E08C918B7F8C93148215821082118222
:10D6E00016A617A608950E94666B089521E0FC0116
:10D6F0008481882309F420E0822F0895FC01818130
:10D700009081891B877098E0981B81E0933008F422
:10D7100080E00895FC0184818823F9F0815084839E
:10D7200082819381890F828386A5882309F44CC066
:10D7300087A5982F915097A7882331F08091650095
:10D740008460809365000895809165008B7F80934D
:10D7500065008091920187A708951B9880916500CC
:10D760008B7F809365008581882319F081508583A4
:10D77000089580819181891739F190E0DF01A80F28
:10D78000B91F16962C911697228356962C91569770
:10D7900024831E962C911E9723835E962C915E9770
:10D7A0002583D0962C91D09726A717A696962C91D4
:10D7B0009697322F315096963C939697222321F4D8
:10D7C000019687709070808308958F929F92AF9298
:10D7D000BF92CF92EF92FF920F931F93DF93CF935D
:10D7E00000D0CDB7DEB74C01122F4A8369830E9467
:10D7F0007E6B4A816981882331F18091870188732A
:10D8000011F1F401A180BB24C501019697E0F92E26
:10D81000F8228081F816B9F0662329F080919101F1
:10D82000865F860F01C080E0A80CB91CF5018683D5
:10D83000842F0E944F6BF501868B168FE0AA06A3FA
:10D84000C686F401F1820F900F90CF91DF911F9166
:10D850000F91FF90EF90CF90BF90AF909F908F90DF
:10D860000895AF92BF92CF92EF920F93DF93CF9331
:10D8700000D00F92CDB7DEB75C012B834A8369835A
:10D880000E947E6B2B814A816981882329F18091D6
:10D890008701887309F1662329F080919101865FE1
:10D8A000860F01C080E0F5018283842F2B834A8399
:10D8B00069830E944F6BF50184832B812583E6A643
:10D8C00017A6C382808181834A816981002321F068
:10D8D0000150C5010E94E56B0F900F900F90CF9102
:10D8E000DF910F91EF90CF90BF90AF900895CF92BE
:10D8F000EF920F93CF93DF93EC0180918701869590
:10D9000086958695877028819981291709F05CC1D1
:10D91000E62FF0E0E132F10508F056C1EA5BFF4F77
:10D92000EE0FFF1F0590F491E02D0994CE0166E4FF
:10D930004AE0DEC0CE0166E444E1DAC0CE0166E42E
:10D940004EE1D6C0CE0164E64AE022E002E0EE24D9
:10D95000E39452E0C52E36C1CE016FE545E022E0EA
:10D960000AE0EE24E394CC240E94E56BCE016FE53F
:10D9700045E02AE001E00E94E56BCE016FE545E05D
:10D9800022E00AE01FC1CE0160E54AE023E002E0A8
:10D99000EE24CC24CA940E94E56BCE016CE34AE0ED
:10D9A00023E0CC24C3940E94E56BCE0166E44AE0F8
:10D9B00021E000E032E0E32E96C0CE0166E445E0CF
:10D9C00021E001E0EE24E394CC240E94E56BCE013B
:10D9D00062E34FE022E00E94E56BCE0160E54FE09C
:10D9E00022E0F0C0CE016EE645E021E002E0EE2448
:10D9F000E394CC240E94E56BCE016CE745E021E086
:10DA00002AC0CE0162E345E025E000E0EE24CC240C
:10DA10000E94E56BCE016AE545E025E00E94E56BDA
:10DA2000CE016EE643E024E002E0CCC0CE0160E52A
:10DA300045E02AE003E0EE24E394CC240E94E56B69
:10DA4000CE0160E545E024E101E00E94E56BCE01F6
:10DA500060E545E02AE003E0B5C0CE016AE044E1BC
:10DA600025E002E0EE24E394CC24C394ABC0CE01C5
:10DA700062E344E02AE002E0EE24E394CC240E9436
:10DA8000E56BCE0166E448E024E101E00E94E56B2D
:10DA9000CE0162E348E02AE002E00E94E56BCE019D
:10DAA00066E444E024E101E08DC0CE0168E745E092
:10DAB0002AE00AE016C0CE0168E745E022E30AC08A
:10DAC000CE0160E044E12AE001E00BC0CE0160E05D
:10DAD00044E12AE002E005C0CE0160E044E12AE032
:10DAE00003E0EE24E394CC246DC0CE0166E448E26A
:10DAF00021E000E048C0813009F466C0CE016BE44B
:10DB000005C0813009F460C0CE0161E44AE021E043
:10DB100000E041C0CE01642F46E0F9CFCE0166E4BB
:10DB20004AE022E0E6CF813009F44EC0CE0166E43F
:10DB30004AE022E0EDCFCE0168E7E8CFCE0168E70A
:10DB40004AE021E01FC0CE016AE74AE021E00FC0B1
:10DB5000CE016CE74AE021E004C0CE0168E74FE067
:10DB600023E003E010C0CE0168E74FE023E002E0CD
:10DB70000AC0CE0168E74FE023E004C0CE0166E4AE
:10DB800044E129E101E0EE24E39406C0CE0166E41D
:10DB90004AE022E002E0EE24CC240E94316C14C062
:10DBA000CE016CE344E123E002E0EE24CC24C394F4
:10DBB0000E94E56BCE0160E544E123E0EE24E394AE
:10DBC000CC24CA940E94E56BDF91CF910F91EF9026
:10DBD000CF900895682F89E494E046E40E94776C22
:10DBE00008951F920F920FB60F9211242F933F9317
:10DBF0008F939F93EF93FF938BB19AB12CB18C715C
:10DC000021F491FD0DC02E3F29F41092990E10922F
:10DC10009A0E19C02F3FB9F481E08093990E13C07A
:10DC200030919A0E303278F4832F90E03F5F2F3D91
:10DC300021F48758914F20E402C08758914FFC018E
:10DC4000208330939A0EFF91EF919F918F913F9196
:10DC50002F910F900FBE0F901F90189580EF90E0BE
:10DC6000909342018093410110981898109290006F
:10DC700087E689B9599886E38093950084E08AB94C
:10DC800001C08CB15F99FDCF089553980895539AC0
:10DC90000895549857980895549A579A08955D9BFB
:10DCA000FECF509890FD509A8CB908955D9BFECFA1
:10DCB000509A8CB90895EF92FF92CF93DF93E82E9C
:10DCC000E7017E01F92EE70102C00E94566E89919C
:10DCD0008823D9F7DF91CF91FF90EF9008955D9B56
:10DCE000FECF50988EEF8CB908955D9BFECF509873
:10DCF0008FEF8CB90895629FD001739FF001829FCE
:10DD0000E00DF11D649FE00DF11D929FF00D839FCA
:10DD1000F00D749FF00D659FF00D9927729FB00D67
:10DD2000E11DF91F639FB00DE11DF91FBD01CF017A
:10DD300011240895991B79E004C0991F961708F0E3
:10DD4000961B881F7A95C9F780950895AA1BBB1B5F
:10DD500051E107C0AA1FBB1FA617B70710F0A61BEB
:10DD6000B70B881F991F5A95A9F780959095BC010C
:10DD7000CD01089597FB092E07260AD077FD04D020
:10DD8000E5DF06D000201AF4709561957F4F089565
:10DD9000F6F7909581959F4F0895A1E21A2EAA1B40
:10DDA000BB1BFD010DC0AA1FBB1FEE1FFF1FA2174B
:10DDB000B307E407F50720F0A21BB30BE40BF50B48
:10DDC000661F771F881F991F1A9469F760957095D1
:10DDD000809590959B01AC01BD01CF01089597FB03
:10DDE000092E05260ED057FD04D0D7DF0AD0001C1F
:10DDF00038F450954095309521953F4F4F4F5F4FE8
:10DE00000895F6F790958095709561957F4F8F4FA7
:10DE10009F4F0895EE0FFF1F0590F491E02D099498
:10DE2000FB01DC014150504048F005900D9200206C
:10DE3000C9F701C01D9241505040E0F7089568179E
:10DE4000790768F4FB01DC01E40FF51FA40FB51F8F
:10DE500002C002900E9241505040D8F708950C94A1
:10DE6000486FDC0101C06D9341505040E0F70895C8
:10DE7000DC01CB01FC01E199FECF06C0FFBBEEBB8C
:10DE8000E09A31960DB20D9241505040B8F7089586
:10DE9000FB01DC0102C001900D9241505040D8F7C7
:06DEA0000895F894FFCF85
:10DEA60086038703880389034AF0004DFF0722048F
:10DEB6007C5E9CCE003264E2F1003264645A505AB1
:10DEC6006450463C46649CEC1E465ADB0D230EDB32
:10DED6000DFF0000AA05FF09FF0DFF135414AADB6E
:04DEE6000DF000003B
:00000001FF
